:020000040800F2
:1000000000060020E1010008E3010008E301000808
:10001000E3010008E3010008E3010008E301000830
:10002000E3010008E3010008E3010008752F000860
:10003000E3010008E3010008E3010008E301000810
:10004000E3010008E3010008E3010008E301000800
:10005000E3010008E30100081D32000845320008F2
:100060006D32000895320008BD320008E301000837
:10007000E3010008E3010008E3010008E3010008D0
:10008000E3010008E3010008E3010008E3010008C0
:10009000E3010008E3010008E3010008E53200087D
:1000A000E3010008E3010008E3010008E3010008A0
:1000B000B9330008E3010008E3010008E301000888
:1000C000E3010008E3010008E3010008E301000880
:1000D000E3010008E3010008E3010008E301000870
:1000E00049330008E3010008E3010008E3010008C8
:1000F000E3010008E3010008E3010008E301000850
:10010000E3010008E3010008E3010008E30100083F
:10011000E3010008E3010008E3010008E30100082F
:10012000E3010008E3010008E3010008E30100081F
:10013000E3010008E3010008E3010008E30100080F
:10014000E3010008E3010008E30100082927000893
:10015000E3010008E3010008E3010008E3010008EF
:10016000E3010008E3010008E3010008E3010008DF
:10017000E3010008E3010008E3010008E3010008CF
:10018000E3010008E3010008E3010008E3010008BF
:10019000E3010008E3010008E3010008E3010008AF
:1001A000E3010008E3010008E3010008E30100089F
:1001B000E3010008E3010008E3010008E30100088F
:1001C000E3010008E3010008E3010008E30100087F
:1001D000E3010008E3010008E3010008E30100086F
:1001E00002E000F000F8FEE772B6374880F30888B6
:1001F000364880F3098836483649086040F20000E6
:10020000CCF200004EF63471CEF200010860BFF36C
:100210004F8FBFF36F8F40F20000C0F2F0004EF638
:100220008851CEF200010860BFF34F8FBFF36F8F8C
:100230004FF00000E1EE100A4EF63C71CEF20001E4
:100240000860062080F31488BFF36F8F01F034FF3D
:1002500002F02EFE4FF055301F491B4A91423CBF21
:1002600041F8040BFAE71D49184A91423CBF41F896
:10027000040BFAE71A491B4A1B4B9A423EBF51F83E
:10028000040B42F8040BF8E700201849184A914281
:100290003CBF41F8040BFAE701F012FF02F05CFEEC
:1002A000144C154DAC4203DA54F8041B8847F9E7A7
:1002B00000F042F8114C124DAC4203DA54F8041B22
:1002C0008847F9E701F0FABE00060020002200206E
:1002D0000000000808ED00E00000002000060020FB
:1002E0008837000800220020402200204022002001
:1002F000602E0020E0010008E0010008E001000895
:10030000E00100082DE9F04F2DED108AC1F80CD066
:10031000C3689D46BDEC108ABDE8F08F002383F3CF
:1003200011882846A047002001F074FAFEE701F08A
:1003300003FA00DFFEE7000038B500F0BFFB01F074
:100340008BFE054601F0AEFE0446C8B90E4B9D4239
:1003500018D001339D4218BF044641F2883504BFCE
:1003600001240025002001F081FE0CB100F074F89A
:1003700000F002FD284600F0C3F800F06DF8F9E740
:100380000025EFE70546EDE7010007B008B500F0EE
:1003900067FBA0F120035842584108BD07B541F260
:1003A0001203022101A8ADF8043000F077FB03B07E
:1003B0005DF804FB38B5302383F3118817480368D0
:1003C0000BB101F0F3FA164A144800234FF47A7186
:1003D00001F0E2FA002383F31188124C236813B171
:1003E0002368013B2360636813B16368013B63606A
:1003F0000D4D2B7833B963687BB9022000F026FCE1
:10040000322363602B78032B07D163682BB902205A
:1004100000F01CFC4FF47A73636038BD402200206A
:10042000B50300086023002058220020084B1870F4
:1004300003280CD8DFE800F008050208022000F0CD
:10044000FDBB022000F0F0BB024B00225A60704757
:100450005822002060230020244B254A10B51C465A
:100460001968013140D004339342F9D16268214BBD
:100470009A4239D9204B9B6803F1006303F580331E
:100480009A4231D2002000F033FB0220FFF7CEFF6A
:100490001A4B1A6C00221A64196E1A66196E596C7E
:1004A0005A64596E5A665A6E5A6942F080025A610D
:1004B0005A6922F080025A615A691A6942F0005260
:1004C0001A611A6922F000521A611B6972B64FF064
:1004D000E0233021C3F8084DD4E9003281F31188BC
:1004E0009D4683F30888104710BD00BF0000010837
:1004F00020000108FFFF0008002200200038024011
:100500002DE9F04F93B0AA4B00902022FF210AA8BA
:100510009D6800F0DBFBA74A1378A3B9A648012128
:1005200003601170302383F3118803680BB101F06D
:100530003DFAA24AA04800234FF47A7101F02CFA48
:10054000002383F31188009B13B19D4B009A1A601E
:100550009C4A009C1378032B1EBF00231370984AFB
:100560004FF0000A18BF5360D3465646D1460120CB
:1005700000F064FB24B1924B1B68002B00F0118249
:10058000002000F06DFA0390039B002BF2DB0120AA
:1005900000F04AFB039B213B162BE8D801A252F83E
:1005A00023F000BF0106000829060008BD06000868
:1005B0006F0500086F0500086F0500084707000871
:1005C000170900083108000893080008BB08000854
:1005D000E10800086F050008F30800086F0500082F
:1005E00065090008A10600086F050008A9090008B0
:1005F0000D060008A10600086F0500089308000812
:100600000220FFF7C3FE002840F0F581009B022185
:10061000BAF1000F08BF1C4605A841F21233ADF82D
:10062000143000F03BFAA2E74FF47A7000F018FAA9
:10063000071EEBDB0220FFF7A9FE0028E6D0013FF2
:10064000052F00F2DA81DFE807F0030A0D101336F8
:1006500005230593042105A800F020FA17E054486B
:100660000421F9E758480421F6E758480421F3E744
:100670004FF01C08404600F03DFA08F104080590D0
:10068000042105A800F00AFAB8F12C0FF2D10120DC
:1006900000FA07F747EA0B0B5FFA8BFB4FF00009F4
:1006A00000F060FB26B10BF00B030B2B08BF0024FE
:1006B000FFF774FE5BE746480421CDE7002EA5D086
:1006C0000BF00B030B2BA1D10220FFF75FFE0746B7
:1006D00000289BD0012000F00BFA0220FFF7A6FEB5
:1006E00000261FFA86F8404600F012FA044690B140
:1006F0000021404600F01CFA01360028F1D1BA462C
:10070000044641F21213022105A8ADF814303E460A
:1007100000F0C4F92BE70120FFF788FE2546244BA3
:100720009B68AB4207D9284600F0E4F9013040F05D
:1007300067810435F3E7234B00251D70204BBA4633
:100740005D603E46ACE7002E3FF460AF0BF00B035C
:100750000B2B7FF45BAF0220FFF768FE322000F026
:100760007FF9B0F10008FFF651AF18F003077FF4EE
:100770004DAF0F4A926808EB050393423FF646AF30
:10078000B8F5807F3FF742AF124B0193B84523DDA8
:100790004FF47A7000F064F90390039A002AFFF690
:1007A00035AF019B039A03F8012B0137EDE700BF3A
:1007B000002200205C23002040220020B503000816
:1007C000602300205822002004220020082200205C
:1007D0000C2200205C220020C820FFF7D7FD07462E
:1007E00000283FF413AF1F2D11D8C5F12002424558
:1007F0000AAB25F0030028BF424683490192184402
:1008000000F03EFA019A8048FF2100F05FFA4FEABB
:10081000A8037D490193C8F38702284600F05EFAD9
:10082000064600283FF46DAF019B05EB830537E7D3
:100830000220FFF7ABFD00283FF4E8AE00F0A4F97A
:1008400000283FF4E3AE0027B846704B9B68BB42DC
:1008500018D91F2F11D80A9B01330ED027F003039C
:1008600012AA134453F8203C05934046042205A9DC
:1008700000F0ACFA04378046E7E7384600F03AF972
:100880000590F2E7CDF81480042105A800F006F9E0
:1008900006E70023642104A8049300F0F5F800287B
:1008A0007FF4B4AE0220FFF771FD00283FF4AEAE36
:1008B000049800F051F90590E6E70023642104A8AC
:1008C000049300F0E1F800287FF4A0AE0220FFF7C7
:1008D0005DFD00283FF49AAE049800F04DF9EAE778
:1008E0000220FFF753FD00283FF490AE00F05CF9C2
:1008F000E1E70220FFF74AFD00283FF487AE05A993
:10090000142000F057F904210746049004A800F0D1
:10091000C5F83946B9E7322000F0A2F8071EFFF605
:1009200075AEBB077FF472AE384A926807EB0903D5
:1009300093423FF66BAE0220FFF728FD00283FF4FC
:1009400065AE27F003074F44B9453FF4A9AE4846CA
:1009500000F0D0F80421059005A800F09FF809F1F7
:100960000409F1E74FF47A70FFF710FD00283FF417
:100970004DAE00F009F9002844D00A9B01330BD09A
:1009800008220AA9002000F0A9F900283AD0202264
:10099000FF210AA800F09AF9FFF700FD1C4800F0BB
:1009A0003FFF13B0BDE8F08F002E3FF42FAE0BF0E9
:1009B0000B030B2B7FF42AAE0023642105A80593BB
:1009C00000F062F8074600287FF420AE0220FFF70F
:1009D000DDFC804600283FF419AEFFF7DFFC41F252
:1009E000883000F01DFF059800F0EEF9464600F053
:1009F000B9F93C46BBE5064652E64FF0000905E66C
:100A0000BA467EE637467CE65C22002000220020C3
:100A1000A086010070B50F4B1B780133DBB2012BB0
:100A20000C4611D80C4D29684FF47A730E6AA2FB5C
:100A30000332014622462846B047844204D1074B80
:100A400000221A70012070BD4FF4FA7000F0E8FE29
:100A50000020F8E710220020082600209423002020
:100A600007B50023024601210DF107008DF807307C
:100A7000FFF7D0FF20B19DF8070003B05DF804FB3D
:100A80004FF0FF30F9E700000A4608B50421FFF7F0
:100A9000C1FF80F00100C0B2404208BD30B4054C37
:100AA0002368DD69044B0A46AC460146204630BC4B
:100AB000604700BF08260020A086010070B501F045
:100AC000D1F9094E094D30800024286833888342CB
:100AD00008D901F0C1F92B6804440133B4F5803F13
:100AE0002B60F2D370BD00BF962300206823002046
:100AF00001F066BA00F1006000F5803000687047D0
:100B000000F10060920000F5803001F0F1B90000C2
:100B1000054B1A68054B1B889B1A834202D9104467
:100B200001F09AB900207047682300209623002026
:100B300038B5084D044629B128682044BDE838403E
:100B400001F0AAB92868204401F08EF90028F3D0FA
:100B500038BD00BF6823002010F003030AD1B0F5B0
:100B6000047F05D200F10050A0F51040D0F8003805
:100B7000184670470023FBE700F10050A0F5104035
:100B8000D0F8100A70470000064991F8243033B1BC
:100B90000023086A81F824300822FFF7B1BF012042
:100BA000704700BF6C230020014B1868704700BFDE
:100BB000002004E070B5194B1D68194B0138C5F3CE
:100BC0000B0408442D0C04221E88A6420BD15C683D
:100BD0000A46013C824213460FD214F9016F4EB10E
:100BE00002F8016BF6E7013A03F10803ECD1814208
:100BF0000B4602D22C2203F8012B0A4A0524168840
:100C0000AE4204D1984284BF967803F8016B013C50
:100C100002F10402F3D1581A70BD00BF002004E0B5
:100C20009C34000888340008022802BF024B4FF4AD
:100C300000129A61704700BF00040240022802BF00
:100C4000014B20229A61704700040240022801BF34
:100C5000024A536983F02003536170470004024045
:100C600070B504464FF47A764CB1412C254628BF26
:100C7000412506FB05F000F0D3FD641BF4E770BDD1
:100C800010B50023934203D0CC5CC4540133F9E780
:100C900010BD000010B5013810F9013F3BB191F9CA
:100CA00000409C4203D11AB10131013AF4E71AB174
:100CB00091F90020981A10BD1046FCE70346024641
:100CC000D01A12F9011B0029FAD1704702440346D9
:100CD000934202D003F8011BFAE770472DE9F8436D
:100CE0001F4D144695F824200746884652BBDFF86E
:100CF00070909CB395F824302BB92022FF214846F0
:100D00002F62FFF7E3FF95F82400C0F10802A2422A
:100D100028BF2246D6B24146920005EB8000FFF77D
:100D2000AFFF95F82430A41B1E44F6B2082E1744DA
:100D30009044E4B285F82460DBD1FFF725FF00285A
:100D4000D7D108E02B6A03EB82038342CFD0FFF7B1
:100D50001BFF0028CBD10020BDE8F8830120FBE772
:100D60006C230020024B1A78024B1A70704700BFA8
:100D7000942300201022002010B5104C104800F0E1
:100D8000B5F821460E4800F0DDF82468626DD2F80F
:100D9000043843F00203C2F804384FF47A70FFF7C6
:100DA0005FFF0849204600F0D3F9626DD2F804389D
:100DB00023F00203C2F8043810BD00BF68350008F4
:100DC00008260020703500087047000030B5094D36
:100DD0000A4491420DD011F8013B5840082340F3DA
:100DE0000004013B2C4013F0FF0384EA5000F6D1CD
:100DF000EFE730BD2083B8ED02684368114301601E
:100E000003B118477047000013B5446BD4F894340D
:100E10001A681178042915D1217C022912D1197977
:100E2000128901238B4013420CD101A904F14C001B
:100E300001F0FAFED4F89444019B2179024620681F
:100E400000F0D0F902B010BD143001F07DBE0000FA
:100E50004FF0FF33143001F077BE00004C3001F04A
:100E60004FBF00004FF0FF334C3001F049BF00008E
:100E7000143001F04BBE00004FF0FF31143001F090
:100E800045BE00004C3001F01BBF00004FF0FF32A8
:100E90004C3001F015BF00000020704710B5D0F8AD
:100EA00094341A6811780429044617D1017C022968
:100EB00014D15979528901238B4013420ED1143039
:100EC00001F0DEFD024648B1D4F894444FF480733B
:100ED00061792068BDE8104000F072B910BD0000D3
:100EE000406BFFF7DBBF0000704700007FB5124B7F
:100EF000036000234360C0E90233012502260F4B43
:100F0000057404460290019300F18402294600967C
:100F10004FF48073143001F08FFD094B0294CDE93A
:100F2000006304F523724FF48073294604F14C00EA
:100F300001F056FE04B070BDBC340008E10E00089C
:100F4000090E00080B68302282F311880A7903EB3E
:100F5000820290614A79093243F822008A7912B1FB
:100F600003EB820398610223C0F8941403740020F9
:100F700080F311887047000038B5037F044613B131
:100F800090F85430ABB9201D01250221FFF734FF42
:100F900004F1140025776FF0010100F069FC84F87A
:100FA000545004F14C006FF00101BDE8384000F0EE
:100FB0005FBC38BD10B5012104460430FFF71CFFAB
:100FC0000023237784F8543010BD000038B5044660
:100FD0000025143001F048FD04F14C00257701F0A4
:100FE00017FE201D84F854500121FFF705FF20460D
:100FF000BDE83840FFF752BF90F8443003F060037B
:10100000202B07D190F84520212A4FF0000303D868
:101010001F2A06D800207047222AFBD1C0E90E33D0
:1010200003E0034A82630722C2630364012070471E
:101030001122002037B5D0F894341A6811780429A9
:1010400004461AD1017C022917D11979128901238A
:101050008B40134211D100F14C05284601F098FE57
:1010600058B101A9284601F0DFFDD4F89444019B52
:1010700021790246206800F0B5F803B030BD0000C9
:10108000F0B500EB810385B09E6904460D46FEB1C4
:10109000302383F3118804EB8507301D0821FFF707
:1010A000ABFEFB685B691B6806F14C001BB101904D
:1010B00001F0C8FD019803A901F0B6FD024648B150
:1010C000039B2946204600F08DF8002383F3118806
:1010D00005B0F0BDFB685A691268002AF5D01B8A7A
:1010E000013B1340F1D104F14402EAE7093138B57C
:1010F00050F82140DCB1302383F31188D4F89424D4
:101100001368527903EB8203DB689B695D6845B124
:1011100004216018FFF770FE294604F1140001F065
:10112000B9FC2046FFF7BAFE002383F3118838BDCF
:101130007047000001F018B8012303700023C0E9D4
:101140000133C36183620362C36243620363704716
:1011500038B50446302383F311880025C0E90355D0
:10116000C0E90555416001F00FF80223237085F3B3
:101170001188284638BD000070B500EB8103054694
:101180005069DA600E46144618B110220021FFF7AC
:101190009DFDA06918B110220021FFF797FD31468F
:1011A0002846BDE8704001F0B9B80000826802F03E
:1011B000011282600022C0E90422826101F03AB982
:1011C000F0B400EB81044789E4680125A4698D40EF
:1011D0003D43458123600023A2606360F0BC01F0C1
:1011E00055B90000F0B400EB81040789E4680125DB
:1011F00064698D403D43058123600023A2606360E4
:10120000F0BC01F0CFB9000070B502230025044600
:101210000370C0E90255C0E90455C564856180F8D2
:10122000345001F017F863681B6823B12946204643
:10123000BDE87040184770BD0378052B10B5044613
:101240000AD080F850300523037043681B680BB147
:10125000042198470023A36010BD000001780529F0
:1012600006D190F85020436802701B6803B11847FC
:101270007047000070B590F83430044613B1002375
:1012800080F8343004F14402204601F0F5F8636838
:101290009B68B3B994F8443013F0600535D0002151
:1012A000204601F095FB0021204601F087FB636892
:1012B0001B6813B1062120469847062384F8343072
:1012C00070BD204698470028E4D0B4F84A30E26B5D
:1012D0009A4288BFE36394F94430E56B002B4FF0EA
:1012E000300380F20381002D00F0F280092284F89F
:1012F000342083F311880021D4E90E232046FFF720
:1013000071FF002383F31188DAE794F8452003F096
:101310007F0343EA022340F20232934200F0C58089
:1013200021D8B3F5807F48D00DD8012B3FD0022BB8
:1013300000F09380002BB2D104F14C02A263022290
:10134000E2632364C1E7B3F5817F00F09B80B3F5CE
:10135000407FA4D194F84630012BA0D1B4F84C3092
:1013600043F0020332E0B3F5006F4DD017D8B3F568
:10137000A06F31D0A3F5C063012B90D8636894F8B7
:1013800046205E6894F84710B4F848302046B047CD
:10139000002884D04368A3630368E3631AE0B3F5CD
:1013A000106F36D040F6024293427FF478AF5C4B28
:1013B000A3630223E3630023C3E794F84630012BC1
:1013C0007FF46DAFB4F84C3023F00203C4E90E553E
:1013D000A4F84C30256478E7B4F84430B3F5A06F36
:1013E0000ED194F8463084F84E30204600F08AFF43
:1013F00063681B6813B101212046984703232370BB
:101400000023C4E90E339CE704F14F03A3630123D7
:10141000C3E72378042B10D1302383F311882046AF
:10142000FFF7C4FE85F311880321636884F84F50E9
:1014300021701B680BB12046984794F84630002B6A
:10144000DED084F84F300423237063681B68002BC0
:10145000D6D0022120469847D2E794F848301D069E
:1014600003F00F0120460AD500F0F8FF012804D050
:1014700002287FF414AF2B4B9AE72B4B98E700F030
:10148000DFFFF3E794F84630002B7FF408AF94F8C1
:10149000483013F00F01B3D01A06204602D501F0F0
:1014A000ABFAADE701F09EFAAAE794F84630002BBC
:1014B0007FF4F5AE94F8483013F00F01A0D01B066E
:1014C000204602D501F084FA9AE701F077FA97E70F
:1014D000142284F8342083F311882B462A462946A7
:1014E0002046FFF76DFE85F31188E9E65DB1152210
:1014F00084F8342083F311880021D4E90E23204698
:10150000FFF75EFEFDE60B2284F8342083F311889A
:101510002B462A4629462046FFF764FEE3E700BF34
:10152000EC340008E4340008E834000838B590F8DA
:1015300034300446002B3ED0063BDAB20F2A34D8B2
:101540000F2B32D8DFE803F0373131082232313146
:101550003131313131313737C56BB0F84A309D42C6
:1015600014D2C3681B8AB5FBF3F203FB12556DB9A5
:10157000302383F311882B462A462946FFF732FE93
:1015800085F311880A2384F834300EE0142384F89C
:101590003430302383F3118800231A46194620463D
:1015A000FFF70EFE002383F3118838BD036C03B1EF
:1015B00098470023E7E70021204601F009FA0021BF
:1015C000204601F0FBF963681B6813B10621204631
:1015D00098470623D7E7000010B590F83430142B55
:1015E000044629D017D8062B05D001D81BB110BD51
:1015F000093B022BFBD80021204601F0E9F900212C
:10160000204601F0DBF963681B6813B10621204610
:101610009847062319E0152BE9D10B2380F83430C5
:10162000302383F3118800231A461946FFF7DAFDA9
:10163000002383F31188DAE7C3689B695B68002B9A
:10164000D5D1036C03B19847002384F83430CEE73A
:1016500000230375826803691B6899689142FBD275
:101660005A68036042601060586070470023037539
:10167000826803691B6899689142FBD85A680360C5
:10168000426010605860704708B50846302383F305
:1016900011880B7D032B05D0042B0DD02BB983F3C0
:1016A000118808BD8B6900221A604FF0FF338361F7
:1016B000FFF7CEFF0023F2E7D1E9003213605A6052
:1016C000F3E70000FFF7C4BF054BD9680875186839
:1016D00002681A60536001220275D860FEF712BEDC
:1016E0009823002030B50C4BDD684B1C87B00446B6
:1016F0000FD02B46094A684600F04EF92046FFF706
:10170000E3FF009B13B1684600F050F9A86907B0E9
:1017100030BDFFF7D9FFF9E79823002089160008AC
:10172000044B1A68DB6890689B68984294BF00205D
:101730000120704798230020084B10B51C68D8681A
:1017400022681A60536001222275DC60FFF78EFF69
:1017500001462046BDE81040FEF7D4BD9823002086
:1017600038B5074C074908480123002523706560F8
:1017700001F046FB0223237085F3118838BD00BFBA
:1017800000260020F43400089823002000F044B91B
:10179000034A516853685B1A9842FBD8704700BFF0
:1017A000001000E08B60022308618B8208467047BE
:1017B0008368A3F1840243F8142C026943F8442C93
:1017C000426943F8402C094A43F8242CC26843F884
:1017D000182C022203F80C2C002203F80B2C044ACC
:1017E00043F8102CA3F12000704700BF1D03000830
:1017F0009823002008B5FFF7DBFFBDE80840FFF79E
:1018000061BF0000024BDB6898610F20FFF75CBFEF
:1018100098230020302383F31188FFF7F3BF0000E3
:1018200008B50146302383F311880820FFF75AFFDB
:10183000002383F3118808BD064BDB6839B1426889
:1018400018605A60136043600420FFF74BBF4FF0ED
:10185000FF307047982300200368984206D01A682A
:101860000260506099611846FFF72CBF7047000076
:1018700038B504460D462068844200D138BD03685F
:1018800023605C608561FFF71DFFF4E710B5036816
:101890009C68A2420CD85C688A600B604C60216036
:1018A000596099688A1A9A604FF0FF33836010BDBF
:1018B0001B68121BECE700000A2938BF0A2170B52B
:1018C00004460D460A26601901F094FA01F080FAE8
:1018D000041BA54203D8751C2E460446F3E70A2EC6
:1018E00004D9BDE87040012001F0CABA70BD000003
:1018F000F8B5144B0D46D96103F1100141600A2A75
:101900001969826038BF0A22016048601861A8180E
:10191000144601F061FA0A2701F05AFA431BA34268
:10192000064606D37C1C281901F064FA2746354682
:10193000F2E70A2F04D9BDE8F840012001F0A0BA6F
:10194000F8BD00BF98230020F8B506460D4601F00B
:101950003FFA0F4A134653F8107F9F4206D12A469A
:1019600001463046BDE8F840FFF7C2BFD169BB6809
:10197000441A2C1928BF2C46A34202D92946FFF746
:101980009BFF224631460348BDE8F840FFF77EBF83
:1019900098230020A823002010B4C0E903230023CB
:1019A0005DF8044B4361FFF7CFBF000010B5194C41
:1019B000236998420DD0D0E90032816813605A60E3
:1019C0009A680A449A60002303604FF0FF33A361D2
:1019D00010BD2346026843F8102F536000220260B6
:1019E00022699A4203D1BDE8104001F0FDB9936825
:1019F00081680B44936001F0EBF92269E169926818
:101A0000441AA242E4D91144BDE81040091AFFF774
:101A100053BF00BF982300202DE9F047DFF8BC80BA
:101A200008F110072C4ED8F8105001F0D1F9D8F871
:101A30001C40AA68031B9A423ED81444D5E90032E0
:101A40004FF00009C8F81C4013605A60C5F80090B8
:101A5000D8F81030B34201D101F0C6F989F31188EA
:101A6000D5E9033128469847302383F311886B6901
:101A7000002BD8D001F0ACF96A69A0EB04094A4503
:101A800082460DD2022001F0FBF90022D8F8103076
:101A9000B34208D151462846BDE8F047FFF728BFBA
:101AA000121A2244F2E712EB090938BF4A462946C6
:101AB0003846FFF7EBFEB5E7D8F81030B34208D050
:101AC0001444211AC8F81C00A960BDE8F047FFF7CC
:101AD000F3BEBDE8F08700BFA823002098230020B4
:101AE00000207047FEE70000704700004FF0FF3015
:101AF0007047000002290CD0032904D001290748AF
:101B000018BF00207047032A05D8054800EBC20023
:101B10007047044870470020704700BFCC3500086C
:101B2000202200208035000870B59AB0054608468E
:101B300001A9144600F0C2F801A8FFF7BFF8431C42
:101B40005B00C5E900340022237003236370C6B232
:101B500001AB02341046D1B28E4204F1020401D826
:101B60001AB070BD13F8011B04F8021C04F8010C34
:101B70000132F0E708B5302383F311880348FFF7FB
:101B800059FA002383F3118808BD00BF08260020FE
:101B900090F8443003F01F02012A07D190F8452045
:101BA0000B2A03D10023C0E90E3315E003F06003D4
:101BB000202B08D1B0F848302BB990F84520212AC5
:101BC00003D81F2A04D8FFF717BA222AEBD0FAE766
:101BD000034A82630722C26303640120704700BF87
:101BE0001822002007B5052917D8DFE801F01916DB
:101BF00003191920302383F31188104A0190012121
:101C0000FFF7BAFA01980E4A0221FFF7B5FA0D481C
:101C1000FFF7DCF9002383F3118803B05DF804FBC0
:101C2000302383F311880748FFF7A6F9F2E7302342
:101C300083F311880348FFF7BDF9EBE7203500086F
:101C4000443500080826002038B50C4D0C4C0D49D1
:101C50002A4604F10800FFF767FF05F1CA0204F104
:101C600010000949FFF760FF05F5CA7204F118007A
:101C70000649BDE83840FFF757BF00BFD02A002013
:101C800020220020003500080A350008153500081C
:101C900070B5044608460D46FFF710F8C6B2204658
:101CA000013403780BB9184670BD32462946FEF759
:101CB000F1FF0028F3D10120F6E700002DE9F047FD
:101CC00005460C46FEF7FAFF2C49C6B22846FFF738
:101CD000DFFF08B10C36F6B229492846FFF7D8FFD6
:101CE00008B11036F6B2632E0BD8DFF89080DFF81B
:101CF0009090244FDFF898A02E7846B92670BDE862
:101D0000F08729462046BDE8F04701F09FBB252E0D
:101D100030D1072241462846FEF7BCFF80B91A4B56
:101D2000224603F1100153F8040B42F8040B8B42D6
:101D3000F9D119889B781180937007351334DBE74C
:101D4000082249462846FEF7A5FF98B90F4BA21C6A
:101D5000197809090232C95D02F8041C13F8011B45
:101D600001F00F015345C95D02F8031CF0D118348E
:101D70000835C1E704F8016B0135BDE7EC35000813
:101D80001535000808360008F4350008107AFF1FE2
:101D90001C7AFF1FBFF34F8F024AD368DB03FCD4CA
:101DA000704700BF003C024008B5094B1B7873B96F
:101DB000FFF7F0FF074B1A69002ABFBF064A5A60B7
:101DC00002F188325A601A6822F480621A6008BDF3
:101DD0002E2D0020003C02402301674508B50B4B27
:101DE0001B7893B9FFF7D6FF094B1A6942F00042FE
:101DF0001A611A6842F480521A601A6822F48052FA
:101E00001A601A6842F480621A6008BD2E2D002004
:101E1000003C02400B28F0B516D80C4C0C49237836
:101E20007BB90C4D0E460C234FF0006255F8047B35
:101E300046F8042B013B13F0FF033A44F6D101238B
:101E4000237051F82000F0BD0020FCE7602D002039
:101E5000302D00201C360008014B53F8200070473D
:101E60001C3600080C2070470B2810B5044601D919
:101E7000002010BDFFF7CEFF064B53F82430184466
:101E8000C21A0BB90120F4E712680132F0D1043B09
:101E9000F6E700BF1C3600080B2810B5044621D811
:101EA000FFF778FFFFF780FF0F4AF323D360C300EB
:101EB000DBB243F4007343F002031361136943F48C
:101EC00080331361FFF766FFFFF7A4FF074B53F85A
:101ED000241000F0D9F8FFF781FF2046BDE810403C
:101EE000FFF7C2BF002010BD003C02401C360008B6
:101EF000F8B512F00103144642D18218B2F1016F15
:101F000057D82D4B1B6813F0010352D02B4DFFF710
:101F10004BFFF323EB60FFF73DFF40F20127032C5B
:101F200015D824F001046618244C401A40F2011719
:101F3000B142236900EB010524D123F001032361A1
:101F4000FFF74CFF0120F8BD043C0430E7E78307AE
:101F5000E7D12B6923F440732B612B693B432B6141
:101F600051F8046B0660BFF34F8FFFF713FF036850
:101F70009E42E9D02B6923F001032B61FFF72EFF6E
:101F80000020E0E723F44073236123693B4323618E
:101F90000B882B80BFF34F8FFFF7FCFE2D8831F8A5
:101FA000023BADB2AB42C3D0236923F001032361EE
:101FB000E4E71846C7E700BF00380240003C024093
:101FC000084908B50B7828B11BB9FFF7EDFE0123CE
:101FD0000B7008BD002BFCD0BDE808400870FFF76F
:101FE000FDBE00BF2E2D002010B50244064BD2B21C
:101FF000904200D110BD441C00B253F8200041F8BB
:10200000040BE0B2F4E700BF502800400F4B30B59E
:102010001C6F240407D41C6F44F400741C671C6FED
:1020200044F400441C670A4C236843F48073236023
:102030000244084BD2B2904200D130BD441C00B2E1
:1020400051F8045B43F82050E0B2F4E70038024056
:10205000007000405028004007B5012201A900206F
:10206000FFF7C2FF019803B05DF804FB13B5044607
:10207000FFF7F2FFA04205D0012201A90020019440
:10208000FFF7C4FF02B010BD70470000034B1A6891
:102090001AB9034AD2F874281A607047642D0020D8
:1020A0000030024008B5FFF7F1FF024B1868C0F39B
:1020B000407008BD642D002070470000FEE700005E
:1020C0000A4B0B480B4A90420BD30B4BDA1C121AEB
:1020D000C11E22F003028B4238BF00220021FEF70E
:1020E000F5BD53F8041B40F8041BECE7C8370008A3
:1020F000602E0020602E0020602E002070B5D0E9F8
:1021000015439E6800224FF0FF3504EB4213510146
:10211000D3F800090028BEBFD3F8000940F0804082
:10212000C3F80009D3F8000B0028BEBFD3F8000B9A
:1021300040F08040C3F8000B013263189642C3F8A8
:102140000859C3F8085BE0D24FF00113C4F81C38FB
:1021500070BD0000890141F02001016103699B0607
:10216000FCD41220FFF714BB10B5054C2046FEF737
:10217000E3FF4FF0A0436365024BA36510BD00BFB2
:10218000682D00207036000870B50378012B0546D5
:1021900050D12A4B446D98421BD1294B5A6B42F0C7
:1021A00080025A635A6D42F080025A655A6D5A692C
:1021B00042F080025A615A6922F080025A610E216F
:1021C00043205B6900F022FC1E4BE3601E4BC4F809
:1021D00000380023C4F8003EC02323606E6D4FF426
:1021E0000413A3633369002BFCDA012333610C2051
:1021F000FFF7CEFA3369DB07FCD41220FFF7C8FAE9
:102200003369002BFCDA0026A6602846FFF776FF2C
:102210006B68C4F81068DB68C4F81468C4F81C68FC
:102220004BB90A4BA3614FF0FF336361A36843F0DE
:102230000103A36070BD064BF4E700BF682D0020CA
:10224000003802404014004003002002003C30C02F
:10225000083C30C0F8B5446D054600212046FFF724
:1022600079FFA96D00234FF001128F68C4F834384C
:102270004FF00066C4F81C284FF0FF3004EB431207
:1022800001339F42C2F80069C2F8006BC2F8080926
:10229000C2F8080BF2D20B686A6DEB65636210231B
:1022A0001361166916F01006FBD11220FFF770FAC1
:1022B000D4F8003823F4FE63C4F80038A36943F46B
:1022C000402343F01003A3610923C4F81038C4F875
:1022D00014380A4BEB604FF0C043C4F8103B084B76
:1022E000C4F8003BC4F81069C4F80039EB6D03F181
:1022F000100243F48013EA65A362F8BD4C3600086F
:1023000040800010426D90F84E10D2F8003823F44F
:10231000FE6343EA0113C2F8003870472DE9F84321
:1023200000EB8103456DDA68166806F00306731E3C
:10233000022B05EB41130C4680460FFA81F94FEA58
:1023400041104FF00001C3F8101B4FF0010104F1E0
:10235000100398BFB60401FA03F391698EBF334EA0
:1023600006F1805606F5004600293AD0578A04F156
:102370005801490137436F50D5F81C180B43C5F875
:102380001C382B180021C3F8101953690127611E4E
:10239000A7409BB3138A928B9B08012A88BF5343A3
:1023A000D8F85C20981842EA034301F1400205EB9B
:1023B0008202C8F85C00214653602846FFF7CAFE37
:1023C00008EB8900C3681B8A43EA845348346401DC
:1023D0001E432E51D5F81C381F43C5F81C78BDE8A4
:1023E000F88305EB4917D7F8001B21F40041C7F823
:1023F000001BD5F81C1821EA0303C0E704F13F03D2
:1024000005EB83030A4A5A6028462146FFF7A2FEDD
:1024100005EB4910D0F8003923F40043C0F8003927
:10242000D5F81C3823EA0707D7E700BF0080001063
:1024300000040002826D1268C265FFF75FBE0000F3
:102440005831436D49015B5813F4004004D013F434
:10245000001F0CBF02200120704700004831436D6F
:1024600049015B5813F4004004D013F4001F0CBF63
:10247000022001207047000000EB8101CB68196A3F
:102480000B6813604B6853607047000000EB8103DA
:1024900030B5DD68AA691368D36019B9402B84BFD1
:1024A000402313606B8A1468426D1C44013CB4FBEA
:1024B000F3F46343033323F0030302EB411043EAD5
:1024C000C44343F0C043C0F8103B2B6803F0030340
:1024D000012B09B20ED1D2F8083802EB411013F4E7
:1024E000807FD0F8003B14BF43F0805343F000538B
:1024F000C0F8003B02EB4112D2F8003B43F004432A
:10250000C2F8003B30BD00002DE9F041244D6E6D56
:1025100006EB40130446D3F8087BC3F8087B380762
:102520000AD5D6F81438190706D505EB84032146D9
:10253000DB6828465B689847FA071FD5D6F8143839
:10254000DB071BD505EB8403D968CCB98B69488AB6
:102550005A68B2FBF0F600FB16228AB91868DA68EE
:1025600090420DD2121AC3E90024302383F311885C
:102570000B482146FFF78AFF84F31188BDE8F081FC
:10258000012303FA04F26B8923EA02036B81CB680F
:10259000002BF3D021460248BDE8F041184700BFA8
:1025A000682D002000EB810370B5DD68436D6C6918
:1025B0002668E6604A0156BB1A444FF40020C2F870
:1025C00010092A6802F00302012A0AB20ED1D3F8D8
:1025D000080803EB421410F4807FD4F8000914BFFC
:1025E00040F0805040F00050C4F8000903EB421264
:1025F000D2F8000940F00440C2F80009D3F83408CA
:10260000012202FA01F10143C3F8341870BD19B96F
:10261000402E84BF4020206020682E8A8419013C0F
:10262000B4FBF6F440EAC44040F000501A44C6E758
:102630002DE9F8433B4D6E6D06EB40130446D3F88D
:102640000889C3F8088918F0010F4FEA40171AD01B
:10265000D6F81038DB0716D505EB8003D9684B692F
:102660001868DA68904230D2121A4FF000091A60E6
:10267000C3F80490302383F3118821462846FFF7DE
:1026800091FF89F3118818F0800F1CD0D6F83438E8
:102690000126A640334216D005EB84036D6DD3F8B6
:1026A0000CC0DCF814200134E4B2D2F800E005EBF1
:1026B00004342F445168714515D3D5F8343823EAD2
:1026C0000606C5F83468BDE8F883012303FA04F26E
:1026D0002B8923EA02032B818B68002BD3D0214660
:1026E00028469847CFE7BCF81000AEEB01038342C1
:1026F00028BF0346D7F8180980B2B3EB800FE2D8A1
:102700009068A0F1040959F8048FC4F80080A0EB88
:1027100009089844B8F1040FF5D818440B449060A8
:102720005360C7E7682D00202DE9F74FA24C656D77
:102730006E69AB691E4016F480586E6107D0204662
:10274000FEF762FD03B0BDE8F04F00F047BC002E7D
:1027500012DAD5F8003E98489B071EBFD5F8003E18
:1027600023F00303C5F8003ED5F8043823F0010335
:10277000C5F80438FEF772FD370505D58E48FFF71A
:10278000BDFC8D48FEF758FDB0040CD5D5F80838CF
:1027900013F0060FEB6823F470530CBF43F410538F
:1027A00043F4A053EB6031071BD56368DB681BB9AA
:1027B000AB6923F00803AB612378052B0CD1D5F866
:1027C000003E7D489A071EBFD5F8003E23F0030364
:1027D000C5F8003EFEF742FD6368DB680BB1764842
:1027E0009847F30274D4B70227D5D4F85490DFF891
:1027F000C8B100274FF0010A09EB4712D2F8003B9D
:1028000003F44023B3F5802F11D1D2F8003B002B05
:102810000DDA62890AFA07F322EA0303638104EB03
:102820008703DB68DB6813B1394658469847A36DC8
:1028300001379B68FFB29F42DED9F00617D5676D5E
:102840003A6AC2F30A1002F00F0302F4F012B2F572
:10285000802F00F08580B2F5402F08D104EB830370
:102860000022DB681B6A07F5805790426AD130036B
:10287000D5F8184813D5E10302D50020FFF744FE30
:10288000A20302D50120FFF73FFE630302D5022019
:10289000FFF73AFE270302D50320FFF735FE750345
:1028A0007FF550AFE00702D50020FFF7C1FEA1077A
:1028B00002D50120FFF7BCFE620702D50220FFF718
:1028C000B7FE23077FF53EAF0320FFF7B1FE39E7E0
:1028D000636DDFF8E4A0019300274FF00109A36DB9
:1028E0009B685FFA87FB9B453FF67DAF019B03EB3F
:1028F0004B13D3F8001901F44021B1F5802F1FD1FB
:10290000D3F8001900291BDAD3F8001941F09041DF
:10291000C3F80019D3F800190029FBDB5946606D94
:10292000FFF718FC218909FA0BF321EA030323813D
:1029300004EB8B03DB689B6813B1594650469847FC
:102940000137CCE7910708BFD7F80080072A98BF66
:1029500003F8018B02F1010298BF4FEA182884E7BF
:10296000023304EB830207F580575268D2F818C08F
:10297000DCF80820DCE9001CA1EB0C0C00218842EB
:102980000AD104EB830463689B699A6802449A60E5
:102990005A6802445A606AE711F0030F08BFD7F87B
:1029A00000808C4588BF02F8018B01F1010188BFCE
:1029B0004FEA1828E3E700BF682D0020436D03EBC2
:1029C0004111D1F8003B43F40013C1F8003B7047BC
:1029D000436D03EB4111D1F8003943F40013C1F802
:1029E00000397047436D03EB4111D1F8003B23F4EC
:1029F0000013C1F8003B7047436D03EB4111D1F860
:102A0000003923F40013C1F80039704700F1604326
:102A100003F561430901C9B283F80013012200F0F4
:102A20001F039A4043099B0003F1604303F5614390
:102A3000C3F880211A60704730B5039C01720433DB
:102A400004FB0325C0E90653049B03630021059B97
:102A5000C160C0E90000C0E90422C0E90842C0E941
:102A60000A11436330BD0000416A0022C0E904112D
:102A7000C0E90A22C2606FF00101FEF7F9BE000052
:102A8000D0E90432934201D1C2680AB9181D7047D7
:102A90000020704703691960C2680132C260C269D0
:102AA000134482690361934224BF436A0361002196
:102AB000FEF7D2BE38B504460D46E3683BB1626905
:102AC000131D1268A3621344E362002007E0237A17
:102AD00033B929462046FEF7AFFE0028EDDA38BDAF
:102AE0006FF00100FBE70000C368C269013BC360EF
:102AF0004369134482694361934224BF436A43613B
:102B000000238362036B03B11847704770B530230D
:102B1000044683F31188866A3EB9FFF7CBFF05466A
:102B200018B186F31188284670BDA36AE26A13F8CB
:102B3000015BA362934202D32046FFF7D5FF002337
:102B400083F31188EFE700002DE9F84F04460E46A5
:102B5000174698464FF0300989F311880025AA4698
:102B6000D4F828B0BBF1000F09D141462046FFF749
:102B7000A1FF20B18BF311882846BDE8F88FD4E976
:102B80000A12A7EB050B521A934528BF9346BBF1D7
:102B9000400F1BD9334601F1400251F8040B43F8B2
:102BA000040B9142F9D1A36A40334036A362403509
:102BB000D4E90A239A4202D32046FFF795FF8AF30D
:102BC0001188BD42D8D289F31188C9E730465A46E8
:102BD000FEF756F8A36A5B445E44A3625D44E7E7F0
:102BE00010B5029C0172043303FB0421C0E90613F3
:102BF0000023C0E90A33039B0363049BC460C0E95C
:102C00000000C0E90422C0E90842436310BD00008F
:102C1000026AC260426AC0E904220022C0E90A22B4
:102C20006FF00101FEF724BED0E904239A4201D1DE
:102C3000C26822B9184650F8043B0B607047002365
:102C40001846FAE7C368C2690133C3604369134495
:102C500082694361934224BF436A43610021FEF7C6
:102C6000FBBD000038B504460D46E3683BB123695F
:102C70001A1DA262E2691344E362002007E0237A8E
:102C800033B929462046FEF7D7FD0028EDDA38BDD6
:102C90006FF00100FBE7000003691960C268013AA8
:102CA000C260C269134482690361934224BF436ACC
:102CB000036100238362036B03B118477047000070
:102CC00070B530230D460446114683F31188866A99
:102CD0002EB9FFF7C7FF10B186F3118870BDA36A44
:102CE0001D70A36AE26A01339342A36204D3E169CF
:102CF00020460439FFF7D0FF002080F31188EDE76C
:102D00002DE9F84F04460D46904699464FF0300A9B
:102D10008AF311880026B346A76A4FB94946204670
:102D2000FFF7A0FF20B187F311883046BDE8F88F88
:102D3000D4E90A073A1AA8EB0607974228BF1746B4
:102D4000402F1BD905F1400355F8042B40F8042B04
:102D50009D42F9D1A36A4033A3624036D4E90A23E5
:102D60009A4204D3E16920460439FFF795FF8BF3BB
:102D700011884645D9D28AF31188CDE729463A46CB
:102D8000FDF77EFFA36A3B443D44A3623E44E5E772
:102D9000D0E904239A4217D1C3689BB1836A8BB1EF
:102DA000043B9B1A0ED01360C368013BC360C36928
:102DB0001A44836902619A4224BF436A0361002373
:102DC00083620123184670470023FBE700F030B907
:102DD0004FF08043586A70474FF080430022586399
:102DE0001A610222DA6070474FF080430022DA60F5
:102DF000704700004FF0804358637047FEE70000C3
:102E000070B51B4B01630025044686B0586085628F
:102E10000E4600F0BFF804F11003C4E904334FF08C
:102E2000FF33C4E90635C4E90044A560E562FFF755
:102E3000CFFF2B460246C4E9082304F134010D4AB2
:102E4000256580232046FEF7ADFC0123E0600A4A99
:102E50000375009272680192B268CDE90223074BB4
:102E60006846CDE90435FEF7C5FC06B070BD00BF6D
:102E7000002600207C36000881360008FD2D000861
:102E8000024AD36A1843D062704700BF98230020DB
:102E90004B6843608B688360CB68C3600B69436198
:102EA0004B6903628B6943620B68036070470000E3
:102EB00008B5264B26481A6940F2FF110A431A61E9
:102EC0001A6922F4FF7222F001021A611A691A6B60
:102ED0000A431A631A6D0A431A651E4A1B6D11468E
:102EE000FFF7D6FF02F11C0100F58060FFF7D0FF6D
:102EF00002F1380100F58060FFF7CAFF02F15401CA
:102F000000F58060FFF7C4FF02F1700100F58060FA
:102F1000FFF7BEFF02F18C0100F58060FFF7B8FFFC
:102F200002F1A80100F58060FFF7B2FF02F1C401D1
:102F300000F58060FFF7ACFF02F1E00100F5806072
:102F4000FFF7A6FFBDE8084000F0EEB800380240E9
:102F5000000002408836000808B500F059FAFEF774
:102F6000FFFBFFF793F8BDE80840FEF76DBE0000D9
:102F700070470000EFF3098305494A6B22F0010214
:102F80004A63683383F30988002383F31188704709
:102F900000EF00E0302080F3118862B60C4B0D4A40
:102FA000D96821F4E0610904090C0A43DA60D3F816
:102FB000FC20094942F08072C3F8FC200A6842F004
:102FC00001020A602022DA7783F82200704700BFEE
:102FD00000ED00E00003FA05001000E010B530231A
:102FE00083F311880E4B5B6813F4006314D0F1EE89
:102FF000103AEFF30984683C4FF08073E361094BAA
:10300000DB6B236684F30988FEF78AFB10B1064B5D
:10301000A36110BD054BFBE783F31188F9E700BFFF
:1030200000ED00E000EF00E02F030008320300088D
:103030000F4B1A6C42F001021A641A6E42F0010240
:103040001A660C4A1B6E936843F0010393604FF0BD
:10305000804353229A624FF0FF32DA6200229A6173
:103060005A63DA605A6001225A611A60704700BFE1
:1030700000380240002004E04FF0804208B511699A
:10308000D3680B40D9B2C9439B07116107D53023E0
:1030900083F31188FEF77AFB002383F3118808BDC0
:1030A0001F4B1A696FEAC2526FEAD2521A611A694B
:1030B000C2F308021A614FF0FF301A695A69586169
:1030C00000215A6959615A691A6A62F080521A627B
:1030D0001A6A02F080521A621A6A5A6A58625A6A66
:1030E00059625A6A1A6C42F080521A641A6E42F09F
:1030F00080521A661A6E0B4A106840F48070106095
:10310000186F00F44070B0F5007F1EBF4FF48030A0
:1031100018671967536823F40073536000F054B9BB
:103120000038024000700040334B4FF080521A6468
:10313000324A4FF4404111601A6842F001021A60AD
:103140001A689107FCD59A6822F003029A602A4B0C
:103150009A6812F00C02FBD1196801F0F9011960AC
:103160009A601A6842F480321A601A689203FCD599
:103170005A6F42F001025A671F4B5A6F9007FCD5F5
:103180001F4A5A601A6842F080721A601B4A5368DC
:103190005904FCD5184B1A689201FCD5194A9A605B
:1031A000194B1A68194B9A42194B21D1194A1168C7
:1031B000194A91421CD140F205121A60144A136850
:1031C00003F00F03052BFAD10B4B9A6842F0020271
:1031D0009A609A6802F00C02082AFAD15A6C42F4FA
:1031E00080425A645A6E42F480425A665B6E70475F
:1031F00040F20572E1E700BF003802400070004075
:103200000854400700948838002004E0116400202E
:10321000003C024000ED00E041C20F41074A08B502
:10322000536903F00103536123B1054A13680BB1DD
:1032300050689847BDE80840FFF7D0BE003C014009
:10324000E02D0020074A08B5536903F002035361DB
:1032500023B1054A93680BB1D0689847BDE8084090
:10326000FFF7BCBE003C0140E02D0020074A08B536
:10327000536903F00403536123B1054A13690BB189
:1032800050699847BDE80840FFF7A8BE003C0140E0
:10329000E02D0020074A08B5536903F00803536185
:1032A00023B1054A93690BB1D0699847BDE808403E
:1032B000FFF794BE003C0140E02D0020074A08B50E
:1032C000536903F01003536123B1054A136A0BB12C
:1032D000506A9847BDE80840FFF780BE003C0140B7
:1032E000E02D0020164B10B55C6904F478725A6129
:1032F000A30604D5134A936A0BB1D06A98476006B7
:1033000004D5104A136B0BB1506B9847210604D5B6
:103310000C4A936B0BB1D06B9847E20504D5094A70
:10332000136C0BB1506C9847A30504D5054A936CF8
:103330000BB1D06C9847BDE81040FFF74FBE00BFFF
:10334000003C0140E02D0020194B10B55C6904F4ED
:103350007C425A61620504D5164A136D0BB1506D5B
:103360009847230504D5134A936D0BB1D06D984748
:10337000E00404D50F4A136E0BB1506E9847A104B8
:1033800004D50C4A936E0BB1D06E9847620404D5F5
:10339000084A136F0BB1506F9847230404D5054AB0
:1033A000936F0BB1D06F9847BDE81040FFF716BE82
:1033B000003C0140E02D002008B5FFF75DFEBDE8B0
:1033C0000840FFF70BBE0000062108B50846FFF7CE
:1033D0001DFB06210720FFF719FB06210820FFF738
:1033E00015FB06210920FFF711FB06210A20FFF734
:1033F0000DFB06211720FFF709FB06212820FFF708
:1034000005FBBDE8084007211C20FFF7FFBA0000BC
:1034100008B5FFF745FE00F00BF8FDF78BFEFDF752
:1034200063FDFFF7A5FDBDE80840FFF7CFBC000036
:103430000023054A19460133102BC2E9001102F19D
:103440000802F8D1704700BFE02D0020034611F8B4
:10345000012B03F8012B002AF9D1704753544D3347
:1034600032463F3F3F0053544D33324634307800AC
:1034700053544D3332463432780053544D33324630
:103480003434365858000000012033000010410049
:1034900001105A000310590007103100000000000D
:1034A0005C340008130400006634000819040000AE
:1034B00070340008210400007A3400080000000085
:1034C000650E0008510E00088D0E0008790E0008E8
:1034D000850E0008710E00085D0E0008490E0008F8
:1034E000990E00080000000001000000000000002C
:1034F00063300000F0340008F02300200026002094
:103500004172647550696C6F740025424F4152449A
:10351000252D424C002553455249414C25000000C1
:10352000020000000000000081100008ED100008FB
:1035300040004000A02A0020B02A00200200000025
:10354000000000000300000000000000311100082E
:103550000000000010000000C02A00200000000051
:103560000100000000000000682D002001010200A1
:10357000E51B0008F51A0008911B0008751B0008E0
:10358000430000008835000809024300020100C022
:1035900032090400000102020100052400100105A7
:1035A000240100010424020205240600010705820B
:1035B000030800FF09040100020A000000070501DA
:1035C00002400000070581024000000012000000D8
:1035D000D4350008120110010200004009124157C1
:1035E00000020102030100000403090425424F41C7
:1035F000524425006F6D6E69627573663470726F28
:103600002D626473686F740030313233343536376D
:103610003839414243444546000000000040000064
:1036200000400000004000000040000000000100D9
:103630000000020000000200000002000000020082
:103640000000020000000200000002000000000074
:10365000751200082D150008D9150008400040001B
:10366000C82D0020C82D002001000000D82D00200A
:103670008000000040010000030000006D61696EE1
:103680000069646C650000000001804200000000D9
:10369000AAAAAAAA00010040FFFF00000000000043
:1036A00000A00A004005000100000000AAAAAAAA82
:1036B00040020001CFFF00000000000000000000F9
:1036C0000000000000000000AAAAAAAA0000000052
:1036D000FFFF0000000000000000000000000000EC
:1036E00000000000AAAAAAAA00000000FFFF000034
:1036F00000000000000000000000000000000000CA
:10370000AAAAAAAA00000000FFFF00000000000013
:10371000000000000000000000000000AAAAAAAA01
:1037200000000000FFFF000000000000000000009B
:103730000000000000000000AAAAAAAA00000000E1
:10374000FFFF00000000000000000000000000007B
:10375000000000000A00000000000000030000005C
:103760000000000000000000000000000000000059
:103770000000000000000000000000000000000049
:1037800000000000000000008300000000000000B6
:1037900000000F0000000000FF009600000000087D
:1037A000009600000000080004000000E835000852
:1037B0000000000000000000000000000000000009
:1037C0000000000000000000FFFFFFFFFFFFFFFF01
:1037D000FFFFFFFFFFFFFFFFFFFFFFFFFFFFFFFFF9
:1037E000FFFFFFFFFFFFFFFFFFFFFFFFFFFFFFFFE9
:1037F000FFFFFFFFFFFFFFFFFFFFFFFFFFFFFFFFD9
:10380000FFFFFFFFFFFFFFFFFFFFFFFFFFFFFFFFC8
:020000040801F1
:100000000006002099120108118409086D8309086F
:10001000D98309086D830908A58309089B12010883
:100020009B1201089B1201089B12010831000C0869
:100030009B1201089B1201089B1201089B120108E8
:100040009B1201089B1201089B1201089B120108D8
:100050009B1201089B120108C90B0C08F10B0C083C
:10006000190C0C08410C0C08690C0C08EDB00B08BD
:1000700015B10B0841B10B086DB10B0899B10B0814
:10008000C1B10B08EDB10B0871B00B089B12010850
:100090009B1201089B1201089B120108910C0C088D
:1000A000B50D0C08B90D0C08CD0D0C08D10D0C08C0
:1000B000D50D0C08E90D0C08FD0D0C089B1201086C
:1000C0009B12010879B70B0821B90B089B12010894
:1000D0009B120108650D0C089B120108790D0C0894
:1000E000F50C0C089B1201089B120108210E0C084C
:1000F000250E0C08390E0C083D0E0C0819B20B0821
:100100009B1201089B120108110E0C089B1201089A
:100110008D0D0C089B1201089B1201089B1201080F
:1001200045B20B086DB20B0899B20B08C5B20B08AB
:10013000F1B20B089B1201089B1201089B120108E7
:100140009B1201089B1201089B1201085D070C0815
:1001500019B30B0845B30B0871B30B08A10D0C08BC
:100160009B1201089B1201089B1201089B120108B7
:100170009B1201089B1201089B1201089B120108A7
:100180009B1201089B1201089B1201089B12010897
:100190009B1201089B1201089B1201089B12010887
:1001A0009B1201089B1201089B1201089B12010877
:1001B0009B1201089B1201089B1201089B12010867
:1001C0009B1201089B1201089B1201089B12010857
:1001D0009B1201089B1201089B1201089B12010847
:1001E000C9580108097F0208C5F7030831BA050894
:1001F00055C005089133060839980608FD9F060882
:1002000035A30608B1080708E12E070891F0070892
:1002100095500808ED5D080801750908A57A0908D8
:100220003D940A0869EF0A0881160B08A92C0B08EF
:10023000515C0B0831630B08000000000000000057
:1002400081F0004102E000BF83F0004330B54FEA87
:1002500041044FEA430594EA050F08BF90EA020FF4
:100260001FBF54EA000C55EA020C7FEA645C7FEA87
:10027000655C00F0E2804FEA5454D4EB5555B8BFAA
:100280006D420CDD2C4480EA020281EA030382EA1B
:10029000000083EA010180EA020281EA0303362DAD
:1002A00088BF30BD11F0004F4FEA01314FF4801C80
:1002B0004CEA113102D0404261EB410113F0004F92
:1002C0004FEA03334CEA133302D0524263EB430349
:1002D00094EA050F00F0A780A4F10104D5F1200EE7
:1002E0000DDB02FA0EFC22FA05F2801841F1000142
:1002F00003FA0EF2801843FA05F359410EE0A5F116
:1003000020050EF1200E012A03FA0EFC28BF4CF046
:10031000020C43FA05F3C01851EBE37101F00045FC
:1003200007D54FF0000EDCF1000C7EEB00006EEB09
:100330000101B1F5801F1BD3B1F5001F0CD3490893
:100340005FEA30004FEA3C0C04F101044FEA4452EA
:1003500012F5800F80F09A80BCF1004F08BF5FEA71
:10036000500C50F1000041EB045141EA050130BD51
:100370005FEA4C0C404141EB0101013C28BFB1F563
:10038000801FE9D291F0000F04BF01460020B1FAAE
:1003900081F308BF2033A3F10B03B3F120020CDA81
:1003A0000C3208DD02F1140CC2F10C0201FA0CF05F
:1003B00021FA02F10CE002F11402D8BFC2F1200CC4
:1003C00001FA02F120FA0CFCDCBF41EA0C0190407A
:1003D000E41AA2BF01EB0451294330BD6FEA0404C3
:1003E0001F3C1CDA0C340EDC04F11404C4F12002AE
:1003F00020FA04F001FA02F340EA030021FA04F3C0
:1004000045EA030130BDC4F10C04C4F1200220FA16
:1004100002F001FA04F340EA0300294630BD21FA54
:1004200004F0294630BD94F0000F83F4801306BF1A
:1004300081F480110134013D4EE77FEA645C18BF0E
:100440007FEA655C29D094EA050F08BF90EA020FA5
:1004500005D054EA000C04BF1946104630BD91EA9D
:10046000030F1EBF0021002030BD5FEA545C05D1A0
:100470004000494128BF41F0004130BD14F58004DF
:100480003CBF01F5801130BD01F0004545F0FE4153
:1004900041F470014FF0000030BD7FEA645C1ABF88
:1004A000194610467FEA655C1CBF0B46024650EABF
:1004B000013406BF52EA033591EA030F41F40021EB
:1004C00030BD00BF90F0000F04BF0021704730B571
:1004D0004FF4806404F132044FF000054FF0000146
:1004E00050E700BF90F0000F04BF0021704730B507
:1004F0004FF4806404F1320410F0004548BF4042DC
:100500004FF000013EE700BF42004FEAE2014FEA30
:1005100031014FEA02701FBF12F07F4393F07F4F0B
:1005200081F06051704732F07F4208BF704793F00E
:100530007F4F04BF41F40021704730B54FF4607421
:1005400001F0004521F000411CE700BF50EA010224
:1005500008BF704730B54FF000050AE050EA0102CD
:1005600008BF704730B511F0004502D5404261EB3D
:1005700041014FF4806404F132045FEA915C3FF47E
:10058000D8AE4FF003025FEADC0C18BF03325FEA1B
:10059000DC0C18BF033202EBDC02C2F1200300FACC
:1005A00003FC20FA02F001FA03FE40EA0E0021FAF1
:1005B00002F11444BDE600BF70B54FF0FF0C4CF4DF
:1005C000E06C1CEA11541DBF1CEA135594EA0C0F91
:1005D00095EA0C0F00F0DEF82C4481EA030621EACC
:1005E0004C5123EA4C5350EA013518BF52EA033507
:1005F00041F4801143F4801338D0A0FB02CE4FF0B9
:100600000005E1FB02E506F00042E0FB03E54FF0E8
:100610000006E1FB03569CF0000F18BF4EF0010EE0
:10062000A4F1FF04B6F5007F64F5407404D25FEADC
:100630004E0E6D4146EB060642EAC62141EA55518F
:100640004FEAC52040EA5E504FEACE2EB4F1FD0CD1
:1006500088BFBCF5E06F1ED8BEF1004F08BF5FEA4F
:10066000500E50F1000041EB045170BD06F0004601
:1006700046EA010140EA020081EA0301B4EB5C04AE
:10068000C2BFD4EB0C0541EA045170BD41F48011A6
:100690004FF0000E013C00F3AB8014F1360FDEBFCB
:1006A000002001F0004170BDC4F10004203C35DAA7
:1006B0000C341BDC04F11404C4F1200500FA05F32A
:1006C00020FA04F001FA05F240EA020001F00042CB
:1006D00021F0004110EBD37021FA04F642EB060141
:1006E0005EEA430E08BF20EAD37070BDC4F10C046B
:1006F000C4F1200500FA04F320FA05F001FA04F22F
:1007000040EA020001F0004110EBD37041F100011A
:100710005EEA430E08BF20EAD37070BDC4F1200525
:1007200000FA05F24EEA020E20FA04F301FA05F28D
:1007300043EA020321FA04F001F0004121FA04F235
:1007400020EA020000EBD3705EEA430E08BF20EA05
:10075000D37070BD94F0000F0FD101F0004640003F
:1007600041EB010111F4801F08BF013CF7D041EAC1
:10077000060195F0000F18BF704703F000465200C5
:1007800043EB030313F4801F08BF013DF7D043EA96
:100790000603704794EA0C0F0CEA135518BF95EA4C
:1007A0000C0F0CD050EA410618BF52EA4306D1D1D3
:1007B00081EA030101F000414FF0000070BD50EAF2
:1007C000410606BF1046194652EA430619D094EA7C
:1007D0000C0F02D150EA013613D195EA0C0F05D166
:1007E00052EA03361CBF104619460AD181EA0301BA
:1007F00001F0004141F0FE4141F470014FF0000072
:1008000070BD41F0FE4141F4780170BD70B54FF00C
:10081000FF0C4CF4E06C1CEA11541DBF1CEA13558C
:1008200094EA0C0F95EA0C0F00F0A7F8A4EB05046E
:1008300081EA030E52EA03354FEA013100F0888065
:100840004FEA03334FF0805545EA131343EA12632E
:100850004FEA022245EA111545EA10654FEA0026E3
:100860000EF000419D4208BF964244F1FD0404F59C
:10087000407402D25B084FEA3202B61A65EB0305F8
:100880005B084FEA32024FF480104FF4002CB6EBB5
:10089000020E75EB030E22BFB61A754640EA0C0035
:1008A0005B084FEA3202B6EB020E75EB030E22BF75
:1008B000B61A754640EA5C005B084FEA3202B6EBB6
:1008C000020E75EB030E22BFB61A754640EA9C0075
:1008D0005B084FEA3202B6EB020E75EB030E22BF45
:1008E000B61A754640EADC0055EA060E18D04FEA03
:1008F000051545EA16754FEA06164FEAC30343EAA3
:1009000052734FEAC2025FEA1C1CC0D111F4801F6F
:100910000BD141EA00014FF000004FF0004CB6E768
:1009200011F4801F04BF01430020B4F1FD0C88BF07
:10093000BCF5E06F3FF6AFAEB5EB030C04BFB6EB12
:10094000020C5FEA500C50F1000041EB045170BD05
:100950000EF0004E4EEA113114EB5C04C2BFD4EB32
:100960000C0541EA045170BD41F480114FF0000EB6
:10097000013C90E645EA060E8DE60CEA135594EA32
:100980000C0F08BF95EA0C0F3FF43BAF94EA0C0F35
:100990000AD150EA01347FF434AF95EA0C0F7FF4AA
:1009A00025AF104619462CE795EA0C0F06D152EAFE
:1009B00003353FF4FDAE1046194622E750EA4106E2
:1009C00018BF52EA43067FF4C5AE50EA41047FF4F3
:1009D0000DAF52EA43057FF4EBAE12E74FF0FF3C58
:1009E00006E000BF4FF0010C02E000BF4FF0010C29
:1009F0004DF804CD4FEA410C7FEA6C5C4FEA430CA2
:100A000018BF7FEA6C5C1BD001B050EA410C0CBFF0
:100A100052EA430C91EA030F02BF90EA020F002052
:100A2000704710F1000F91EA030F58BF994208BFB9
:100A300090422CBFD8176FEAE37040F00100704776
:100A40004FEA410C7FEA6C5C02D150EA013C07D1CD
:100A50004FEA430C7FEA6C5CD6D152EA033CD3D018
:100A60005DF8040B704700BF8446104662468C4612
:100A70001946634600E000BF01B5FFF7B7FF002845
:100A800048BF10F1000F01BD4DF808EDFFF7F4FF6E
:100A90000CBF012000205DF808FB00BF4DF808EDF9
:100AA000FFF7EAFF34BF012000205DF808FB00BF1C
:100AB0004DF808EDFFF7E0FF94BF012000205DF83E
:100AC00008FB00BF4DF808EDFFF7CEFF94BF0120F3
:100AD00000205DF808FB00BF4DF808EDFFF7C4FFEC
:100AE00034BF012000205DF808FB00BF4FEA410C35
:100AF0007FEA6C5C02D150EA013C0AD14FEA430C18
:100B00007FEA6C5C02D152EA033C02D14FF0000054
:100B100070474FF0010070474FEA410212F5001292
:100B200015D211D56FF47873B3EB625212D94FEA34
:100B3000C12343F0004343EA505311F0004F23FA1E
:100B400002F018BF404270474FF00000704750EA73
:100B5000013005D111F0004008BF6FF00040704730
:100B60004FF00000704700BF4A0011D212F500128A
:100B700011D20DD56FF47873B3EB62520ED44FEAF5
:100B8000C12343F0004343EA505323FA02F0704775
:100B90004FF00000704750EA013002D14FF0FF30B3
:100BA00070474FF0000070474FEA4102B2F1E04356
:100BB00024BFB3F5001CDCF1FE5C0DD901F0004C44
:100BC0004FEAC0024CEA5070B2F1004F40EB830094
:100BD00008BF20F00100704711F0804F21D113F1C0
:100BE0003872BCBF01F00040704741F480114FEAF9
:100BF0005252C2F11802C2F1200C10FA0CF320FA82
:100C000002F018BF40F001004FEAC1234FEAD3239E
:100C100003FA0CFC40EA0C0023FA02F34FEA430308
:100C2000CCE77FEA625307D150EA01331EBF4FF091
:100C3000FE4040F44000704701F0004040F0FE40AC
:100C400040F40000704700BF80F0004002E000BFA9
:100C500081F0004142001FBF5FEA410392EA030FA7
:100C60007FEA226C7FEA236C6AD04FEA1262D2EBF1
:100C70001363C1BFD218414048404140B8BF5B42F6
:100C8000192B88BF704710F0004F40F4000020F08F
:100C90007F4018BF404211F0004F41F4000121F0A5
:100CA0007F4118BF494292EA030F3FD0A2F10102EF
:100CB00041FA03FC10EB0C00C3F1200301FA03F12D
:100CC00000F0004302D5494260EB4000B0F5000F50
:100CD00013D3B0F1807F06D340084FEA310102F10F
:100CE0000102FE2A51D2B1F1004F40EBC25008BFC1
:100CF00020F0010040EA03007047490040EB00008B
:100D0000013A28BFB0F5000FEDD2B0FA80FCACF18B
:100D1000080CB2EB0C0200FA0CF0AABF00EBC250B8
:100D200052421843BCBFD0401843704792F0000FA6
:100D300081F4000106BF80F400000132013BB5E7F9
:100D40004FEA41037FEA226C18BF7FEA236C21D06F
:100D500092EA030F04D092F0000F08BF08467047D4
:100D600090EA010F1CBF0020704712F07F4F04D1A2
:100D7000400028BF40F00040704712F100723CBFB5
:100D800000F50000704700F0004343F0FE4040F4DF
:100D9000000070477FEA226216BF08467FEA23639D
:100DA0000146420206BF5FEA412390EA010F40F488
:100DB000800070474FF0000304E000BF10F00043D4
:100DC00048BF40425FEA000C08BF704743F09643BB
:100DD00001464FF000001CE050EA010208BF7047D6
:100DE0004FF000030AE000BF50EA010208BF70475D
:100DF00011F0004302D5404261EB41015FEA010C72
:100E000002BF84460146002043F0B64308BFA3F169
:100E10008053A3F50003BCFA8CF2083AA3EBC2534B
:100E200010DB01FA02FC634400FA02FCC2F120026A
:100E3000BCF1004F20FA02F243EB020008BF20F0A1
:100E40000100704702F1200201FA02FCC2F1200207
:100E500050EA4C0021FA02F243EB020008BF20EAFC
:100E6000DC7070477BB972B90029BEBF00204FF01B
:100E7000004106E008BF00281CBF6FF000414FF0A2
:100E8000FF3000F007BAADF1080C6DE904CE00297F
:100E900009DB002B1ADB00F095F8DDF804E0DDE952
:100EA000022304B07047404261EB4101002B1BDB81
:100EB00000F088F8DDF804E0DDE9022304B04042E8
:100EC00061EB4101524263EB43037047524263EBD3
:100ED000430300F077F8DDF804E0DDE9022304B015
:100EE000404261EB41017047524263EB430300F023
:100EF00069F8DDF804E0DDE9022304B0524263EB57
:100F00004303704753B94AB9002908BF00281CBFE2
:100F10004FF0FF314FF0FF3000F0BCB9ADF1080CDD
:100F20006DE904CE00F04EF8DDF804E0DDE90223BF
:100F300004B07047430803F05533C01A830803F028
:100F4000333300F03330184400EB101000F00F3052
:100F500000EB002000EB0040000E704707EE900A07
:100F6000F5EEC07AF1EE10FA01D400F00BB8F1EE14
:100F7000677A08B517EE900A00F004F8404261EB7A
:100F8000410108BDD0B5FFF7BFFA0C4B0022064661
:100F90000F46FFF711FBFFF7E7FD0446FFF792FA54
:100FA000074B0022FFF708FB02460B463046394646
:100FB000FFF74AF9FFF7D8FD2146D0BD0000F03D0C
:100FC0000000F0412DE9F047089D04468E46002BB5
:100FD0004DD18A42944669D9B2FA82F252B101FAED
:100FE00002F3C2F1200120FA01F10CFA02FC41EAFD
:100FF000030E94404FEA1C48210CBEFBF8F61FFA82
:101000008CF708FB16E341EA034306FB07F199421C
:101010000AD91CEB030306F1FF3080F01F819942CF
:1010200040F21C81023E63445B1AA4B2B3FBF8F0A9
:1010300008FB103344EA034400FB07F7A7420AD930
:101040001CEB040400F1FF3380F00A81A74240F258
:1010500007816444023840EA0640E41B00261DB1C3
:10106000D4400023C5E900433146BDE8F0878B42F8
:1010700009D9002D00F0EF800026C5E900013046B7
:101080003146BDE8F087B3FA83F6002E4AD18B4291
:1010900002D3824200F2F980841A61EB030301203B
:1010A0009E46002DE0D0C5E9004EDDE702B9FFDE27
:1010B000B2FA82F2002A40F09280A1EB0C014FEAD2
:1010C0001C471FFA8CFE0126200CB1FBF7F307FB2F
:1010D000131140EA01410EFB03F0884208D91CEBD2
:1010E000010103F1FF3802D2884200F2CB8043466F
:1010F000091AA4B2B1FBF7F007FB101144EA01444E
:101100000EFB00FEA64508D91CEB040400F1FF31DC
:1011100002D2A64500F2BB800846A4EB0E0440EACA
:1011200003409CE7C6F12007B34022FA07FC4CEAD3
:10113000030C20FA07F401FA06F31C43F9404FEAC6
:101140001C4900FA06F3B1FBF9F8200C1FFA8CFEDB
:1011500009FB181140EA014108FB0EF0884202FA2F
:1011600006F20BD91CEB010108F1FF3A80F08880F0
:10117000884240F28580A8F102086144091AA4B2AD
:10118000B1FBF9F009FB101144EA014100FB0EFE2E
:101190008E4508D91CEB010100F1FF346CD28E455D
:1011A0006AD90238614440EA0840A0FB0294A1EBEE
:1011B0000E01A142C846A64656D353D05DB1B3EB4B
:1011C000080261EB0E0101FA07F722FA06F3F1407B
:1011D0001F43C5E9007100263146BDE8F087C2F122
:1011E0002003D8400CFA02FC21FA03F3914001439A
:1011F0004FEA1C471FFA8CFEB3FBF7F007FB1036D3
:101200000B0C43EA064300FB0EF69E4204FA02F47E
:1012100008D91CEB030300F1FF382FD29E422DD9D1
:10122000023863449B1B89B2B3FBF7F607FB163306
:1012300041EA034106FB0EF38B4208D91CEB010186
:1012400006F1FF3816D28B4214D9023E6144C91A06
:1012500046EA004638E72E46284605E70646E3E616
:101260001846F8E64B45A9D2B9EB020864EB0C0E20
:101270000138A3E74646EAE7204694E74046D1E72F
:10128000D0467BE7023B614432E7304609E76444DD
:10129000023842E7704700BF02E000F000F8FEE7C6
:1012A00072B6374880F30888364880F30988364894
:1012B0003649086040F20000CCF200004EF634716E
:1012C000CEF200010860BFF34F8FBFF36F8F40F283
:1012D0000000C0F2F0004EF68851CEF20001086026
:1012E000BFF34F8FBFF36F8F4FF00000E1EE100A96
:1012F0004EF63C71CEF200010860062080F314889F
:10130000BFF36F8FAEF0F2FEADF058FF4FF05530E7
:101310001F491B4A91423CBF41F8040BFAE71D49A3
:10132000184A91423CBF41F8040BFAE71A491B4A9C
:101330001B4B9A423EBF51F8040B42F8040BF8E7EE
:1013400000201849184A91423CBF41F8040BFAE7C3
:10135000AEF0D0FEADF086FF144C154DAC4203DA72
:1013600054F8041B8847F9E701F01EF9114C124D9F
:10137000AC4203DA54F8041B8847F9E7AEF0B8BE74
:1013800000060020002200200000010808ED00E017
:10139000000000200006002020A30E0800220020EC
:1013A000002C0020002C0020C05A0120E001010880
:1013B0003802010838020108380201082DE9F04F0F
:1013C0002DED108AC1F80CD0C3689D46BDEC108A83
:1013D000BDE8F08F002383F311882846A047002042
:1013E000ADF072FCFEE7ADF0CFFA00DFFEE70000E3
:1013F00001F0FF01102A2BDB10F0070F08D010F8C6
:10140000013B013A8B422DD010F0070F42B3F6D1C9
:10141000F0B441EA012141EA014122F007047FF0E2
:1014200000070023F0E80256083C85EA010586EA39
:10143000010685FA47F5A3FA87F586FA47F6A5FA75
:1014400087F68EB9EED1F0BC01F0FF0102F0070281
:1014500032B110F8013B013A83EA010313B1F8D12C
:101460000020704701387047002D06BF354603380D
:10147000073815F0010F07D1013015F4807F02BF46
:10148000013015F4C03F0130F0BC0138704700BF97
:1014900010F8012B11F8013B012A28BF9A42F7D01E
:1014A000D01A7047034613F8012B002AFBD1181AF3
:1014B0000138704738B50022002304460D46FFF777
:1014C000EDFA28B920462946BDE8384000F00AB8B0
:1014D000204605F1004100F005F8404261EB410172
:1014E00038BD00BFD0B50C4B002206460F46FFF7B3
:1014F00063F8FFF739FB0446FEF7E4FF074B0022D1
:10150000FFF75AF802460B4630463946FEF79CFE76
:10151000FFF72AFB2146D0BD0000F03D0000F0415E
:10152000036800221B68184710B503685B6804460F
:10153000984708B194F84D0010BD000038B5044636
:101540007DF0BCF80E4B1D680146E86A026812681F
:10155000904753F0C3FEEB6A93F89C1052F0AAFE3A
:1015600094F837305BB186F089FFEB6AD3F8A0308E
:10157000C01AB0F5FA6F24BF002384F8373038BDA5
:101580000C2C002070B50E4605465FF0B1FB5FF0F5
:1015900073FB10B90124204670BD0A4B93F9E23465
:1015A000012BF7D15FF0A4FB437A002BF2D15FF05F
:1015B0009FFB847A002CEDD1034A314628467DF00A
:1015C000A9FAE8E7104C002028840C08034BD3F854
:1015D0004C350BB97DF028B801207047104C002025
:1015E0002DE9F0432DED028BC47F91B006460F46E6
:1015F0008CB990F90430002B00F00681834B1D68F4
:10160000A86A03685B6B9847044650B9804A39461C
:1016100030467DF07FFA204611B0BDEC028BBDE86C
:10162000F083B3684BB933685B6B3946304611B011
:10163000BDEC028BBDE8F0431847E86AFFF774FF82
:1016400004460028E7D1394630467EF023F9DFF81A
:10165000F4810546394630467DF084FA08F2F442BA
:1016600008F59E6392ED007AD3ED007AB4EEE77A46
:101670002840F1EE10FAC5B209D598F9EC34032BE5
:1016800005D0644A394630467DF044FA254608F2D2
:101690009443D3ED007AB0EE088AF4EEC87AF1EE06
:1016A00010FA0BD517EE900AFEF72EFF5A4ACDE935
:1016B0000001394630467DF02DFA002508F5936388
:1016C000D3ED007AF4EEC87AF1EE10FA0BD517EEEE
:1016D000900AFEF719FF514ACDE90001394630461C
:1016E0007DF018FA002508F29C43D3ED007AB8EE9D
:1016F000087AF4EEC77AF1EE10FA0BDD17EE900AD5
:10170000FEF702FF464ACDE90001394630467DF03A
:1017100001FA0025B8F98034042B07DC0522009279
:101720003946404A30467DF0F5F90025D8F8380FA3
:101730005FF03AFB80B198F9E2346BB1D8F8383FEA
:10174000B8F9E424B3F90E309A4205DA364A39463C
:1017500030467DF0DFF90025DFF8EC903946304661
:10176000FFF710FF99F8C131002B46D100EA0504BC
:101770002E484FF4806100F0F9FE78B1D8F8383F78
:10178000B3F90C30A3F2E24292B2B2F5FA7F05D976
:10179000274A394630467DF0BDF9002499F85C3877
:1017A00053B124482DF08EF8054628B9224A39460F
:1017B00030467DF0AFF92C4600212E2204A80DF111
:1017C0000C080391B2F0C8FBD9F8AC0142463221B3
:1017D00008F0F6F9054600287FF41DAFD9F8AC01F2
:1017E00003689B689847154ACDF800800346394640
:1017F00030467DF08FF92C460DE7114A39463046C8
:101800007DF088F90024B3E7012404E70C2C0020C4
:1018100038840C084F840C0872840C0892840C08DD
:10182000B4840C08D6840C08F5840C08102C002015
:1018300030850C086484002058850C0898370D0802
:101840001B850C08104C0020107C002070B505464C
:101850000E46FFF797FE3146044628467DF0C6FE49
:101860002040C0B270BD0000F0B591B005460E46F4
:101870007DF02EFA0446D8B1102128467CF03AFFBC
:10188000B0B100212E2204A803AF0391B2F064FB93
:1018900010F0AAFD32233A46012110F091F80446D7
:1018A00030B9054B00973246102128467CF02AFFBC
:1018B000204611B0F0BD00BF6C850C0870B5054620
:1018C0000E46B1B990F910408CB116480BF02AFBC6
:1018D000DFED157AB0EEC00AB4EEE70AF1EE10FAC9
:1018E00007D4124A012128467DF014F934462046D7
:1018F00070BDAB689BB10E4B1B68D86AFFF714FE36
:10190000044630B15DF000FD0A4A042156F024FE81
:10191000EDE731462846BDE870407DF0A5BC0124C6
:10192000E5E700BF102C00200000003478850C088B
:101930000C2C00208A850C0838B504467EF064F82B
:101940000546A8B10B4805F0CBFB38B10A490B4856
:1019500010F076F910B1074800F0DAFD2046FFF7E5
:10196000EDFD0123064984F8373020467DF062FF03
:10197000284638BD102C0020408F00202040002039
:10198000AC850C08F8B505460E461746C2B12329AA
:1019900001D0012914D81D4807F076FC044668B12F
:1019A00000242046F8BD95F91030022B08D05DF0D8
:1019B000ABFC174A062156F0CFFDF2E7002EF2D01D
:1019C0003A46314628467EF0D5F804460028E7D04E
:1019D000104ED6F8AC2106F178039A4203D006F6F1
:1019E00054002DF0A5FBD6F8AC0103689B6B98471B
:1019F00086F828082846FFF7A1FD4FF0FF33064977
:101A0000C6F8DC3128467DF015FFCAE7102C00200F
:101A1000BC850C08107C0020D4850C08F8B5054660
:101A20000E467CF013FF104B93F9B7740446CFB900
:101A30000E48BD212DF012FB38B10D4B32464FF44C
:101A4000804128467CF05EFE3C460848BC212DF0D3
:101A500005FB38B1074B32464FF4804128467CF0F5
:101A600051FE00242046F8BD104C00206484002064
:101A7000E8850C0814860C0800207047014800F027
:101A8000EDBC00BF102C002003685B681847000005
:101A90000DF004BC65F012BA5FF078B825F008BB11
:101AA00052F08ABD07F024BD50F044BE0AF034BDA8
:101AB0000CF064BC02F04EBE4FF0D8B914F002BD79
:101AC00062F0F2BA61F070BF0CF0BCBC46F01ABE16
:101AD0000BF0A6BA14F054B866F0A4BF5EF078BD5F
:101AE0005CF080BE06F036BF04F0A8BA0AF052B827
:101AF0000AF07CBC0CF08ABA0CF05EBD0BF0C8B8E2
:101B00000CF0AABB01F03CB900F2845016F09ABE6A
:101B100007F05CBA90F8F432B02202FB030390F8AD
:101B2000382393F8D13012B1012B28BF0123184676
:101B300070470000034808602E21117008221A60C7
:101B4000704700BF78890C0870B5044604F5A055AD
:101B500000F5C8403C301035FFF7F0FC0021284666
:101B600010F0C8FB802120460CF08EFF18B127F042
:101B700023F924F0B7FE04F5005303F29C4292EDE2
:101B8000007ADFED226A03F29442D2ED007A67EE2A
:101B9000A67A04F5A052FDEEE77AD2ED976AF8EE48
:101BA000E77A03F64C7367EEA67A05F54570FDEE0D
:101BB000E77A04F5AF4617EE901A43F8041CD2ED0D
:101BC000967AF0EEE77A67EE877A04F5BA51C3EDBC
:101BD000007A08312AF06AF994ED467AD6ED097A4E
:101BE000E7EE007AC6ED097AB0EE670A27F04CFE00
:101BF0004FF4001186ED090A20460CF045FF20B194
:101C00002846BDE870400EF079BE70BD0000C842A5
:101C1000FFF79ABF38B500F5A0450446D5F8AC01EA
:101C200003689B6B984795F8E3373BB930B104F5EF
:101C30003F502030BDE8384082F052B938BD000036
:101C4000FFF7E8BF38B54FF4801104460CF01CFFD5
:101C5000054620B9012120460CF016FF0546022159
:101C600020460CF011FF48B115B9204602F014FDD2
:101C700004F5A05010300EF03FFD01E0002DF7D12B
:101C80004FF4805120460CF0FFFE30B104F5C74000
:101C90003830BDE8384062F02DBB38BDFFF7D2BF09
:101CA00038B54FF4801104460CF0EEFE01210546D4
:101CB00020460CF0E9FE18B115B9204602F0ECFC04
:101CC000102120460CF0E0FE60B1204602F05AFDE3
:101CD0004FF4800120460CF0D7FE18B927F06CF8BD
:101CE00024F0FCFE202120460CF0CEFE28B1204638
:101CF00002F0BCFD204602F0D5FE4FF40051204614
:101D00000CF0C2FE10B1204602F0B4FE8021204645
:101D10000CF0BAFE28B127F04FF8BDE8384024F0A7
:101D200005BE38BDFFF7BCBF00F5A04300F5C540B8
:101D3000D3F8D01114307FF015BB0000FFF7F4BFCB
:101D400010B5044616F06EFE90F921308BB190F874
:101D5000403373B194F9A8355BB1064B1B68DB6A5D
:101D600093F89C302BB904F28450BDE8104016F073
:101D700081BB10BD0C2C0020FFF7E2BF2DE9F8431A
:101D8000434B1B68DB6A93F89C300446002B7DD0E4
:101D900000F5805898F81937002B77D007F074FABF
:101DA000002873D004F5055604F50055103695F853
:101DB0009E1230460EF044F8002867D004F5907764
:101DC0003846FFF7A7FE022860D994F814244FF094
:101DD000B00909FB024292ED837AF1EE007AB4EE8B
:101DE000E77AF1EE10FA51D495F89E1230460EF0D3
:101DF000D7FAB5F9803407EE903AB8EEE77AB4EE48
:101E0000C07AF1EE10FA0CDD94F8143409FB0343A8
:101E1000F8EE677A93ED837AF4EEC77AF1EE10FA72
:101E200034DCD8F80836D5F8482F002BB8BF5B4211
:101E300093422BDC08F20C63D3ED007A9FED156A18
:101E400005F59363D3ED006AF8EEE77A66EE866AED
:101E5000F4EEE67AF1EE10FA18DC05F64C7393ED29
:101E6000007A27EE067AF4EEC77AF1EE10FA0DD476
:101E700094F81414B5F98224B02303FB01713046A1
:101E800001F58271BDE8F8430DF0F0BDBDE8F883BF
:101E90000C2C00200000C842FFF770BF2DE9F04174
:101EA00090F814342D4D00EB03132F68D3F8C48140
:101EB00000F5907604463046FFF72CFE474514D0D7
:101EC000022814D904F5A047C5F8008097F8D4314A
:101ED000012B15D817D104F5C045D5F83833E3B92F
:101EE000D5F83C33CBB905230BE0022810D804F514
:101EF000A04393F8D4215AB1052283F8D42107E0F6
:101F0000013B87F8D43104F5C2500C3011F0ECFBE2
:101F10002046BDE8F0410AF009B8114B1B68D86AA9
:101F200003685B68984780460028ECD194F8141445
:101F3000B02303FB0161DC31204605F043F9D5F8FD
:101F40001C330FCB05F5487605F5507586E80F0074
:101F500085E80F0087F8D481D5E700BF002C00206A
:101F60000C2C0020FFF79ABF10B500F5A04300F538
:101F7000805493F8E3271AB1002384F819370AE054
:101F8000D3F83038042B07D100F5C440083082F074
:101F900045FA84F8190710BD0123EEE710B500F5E6
:101FA000A0442346D4F8AC2178339A4208D000F5F7
:101FB000A1433C339A421CBF4FF0FF33C4F89C3717
:101FC00004F28C73074A1A6004F5F263064A1A6039
:101FD000FFF7CAFFD4F8AC010368BDE810401B69E5
:101FE000184700BF0000C8420000C8C2FFF7D6BFB4
:101FF000F7B500F5A0460446D6F830388B420D46BA
:102000003FD00B1F00F5C447594207F1080759415B
:102010003846019182F0F2F80199384682F0EEF8E4
:10202000042D02D118486DF0F5FBD6F83038012B9D
:1020300018D1032D16D104F5C8403C307CF048FB84
:1020400040B1204607F020F920B104F53B501C3088
:102050006DF0DAFB2046C6F8305803B0BDE8F0401A
:1020600002F06EBC072DF5D104F55B50D6F8AC2715
:102070006423052192FBF3F33030044A56F06CFAE6
:10208000E8E703B0F0BD00BFEC5A0020B8860C08AA
:1020900038B500F5A0450446D5F8AC0103689B6B44
:1020A000984700283FD095F82838E3BBD5F8AC21F5
:1020B0002B4678339A4238D195F8DC372BB9012179
:1020C0002046BDE83840FFF793BFB5F89238152B8E
:1020D00029D104F5C04393F80C1211F0010120D16D
:1020E000D5F83028072A1CD093F982320BB9042185
:1020F000E6E720460AF016FFDFED0F7AB4EEE70AB6
:10210000F1EE10FAF3DB04F5C440083082F0C6F8B3
:102110000028ECD004F55B50084A0621303056F018
:102120001BFA0721CCE70321CAE704F5A1433C339E
:102130009A42F8D138BD00BF0000B442DC860C08DA
:1021400010B5214CD4F8AC2104F178039A422DED5E
:10215000028BB0EE408A03D00020BDEC028B10BD94
:10216000D4F83038042B25D194F8D53133B1174940
:10217000A1F6DC202DF054FA0028EED19FED147A60
:10218000F0EEC87AF4EEC77AF1EE10FA09D49FEDBA
:10219000110A28EE008ABDEEC88A18EE103AC4F87B
:1021A000AC370D4882F07AF80028D5D0002384F8A7
:1021B000DF37D2E7B4F89218A4F5A04006F026FA6B
:1021C0000028D1D1C8E700BF107C0020408F00203C
:1021D000000000340000C842188E002010B52DED1C
:1021E000028B00F5A0430446D3F83038042B0BD102
:1021F00004F0D0F92046B0EE408A04F097FA38EEA9
:10220000400ABDEC028B10BD00F5C04494EDDB0A22
:10221000F7E700002DE9F0412DED028B00F58C650C
:102220008AB00446284612F063FC04F5A05000234F
:1022300007A910300793089309930FF0E7FE0028D1
:1022400000F087809DED090ADFED597A04F5A0457D
:1022500005F2BC7393ED007A20EE270ADFED557A84
:10226000A7EE270A04F5B2404C3083ED000A66F071
:10227000EDFD2046FFF70CFFD5F8AC0103689B6B22
:10228000984795F8E337002B5ED100285CD095F88D
:102290002838002B58D1D5F83038042B70D09FED5A
:1022A000468A204604F064FA04F5C04204F5A143CE
:1022B000C2F8F404D5F8AC111033994204F5005675
:1022C0001AD192F8B033BBB9B6F9143F002B04DC35
:1022D0003A49D1F8D41EC9060ED5D2F81C73D2F8EB
:1022E00024137F680A33C91B64277B438142ACBF38
:1022F0005B181B18C2F8F434D5F83038D2F8F4144F
:10230000D5F8D82105912046049203930CF03AFEAB
:10231000B5F9E68107462046FFF760FFCDE9007872
:1023200006F21C5605F64C0504F53F50F0EE400A47
:10233000DDE90332D6ED001A95ED001A0599B0EEED
:10234000480A203081F070FA0AB0BDEC028BBDE87B
:10235000F08104F59070FFF7DDFB02280AD994F8AC
:102360001434B02202FB034393F8402212B193EDE0
:102370008B0A69E7284612F055FAB1EE400A63E786
:1023800004F5C64604F5C6473036403704F5C64165
:102390003A462031304615F089FC00283FF47FAFE3
:1023A0003946304615F016FDB0EE408A79E700BF99
:1023B000CDCC4C3ECDCC4C3F00000000104C00205A
:1023C000FFF728BF00F5A04300F5A140D3F8AC21EA
:1023D000343082421FBF03F2C47301201B680B60BC
:1023E00008BF00207047000010B500F5A04200F5BE
:1023F000A143D2F8AC2134339A420C4612D000F5F6
:102400004050D0F8180903681B69984707EE900AF6
:102410009FED057AF8EEE77A012067EE877AC4ED42
:10242000007A10BD0020FCE70AD7233C10B500F568
:10243000A04200F5A143D2F8AC2134339A420C46B5
:102440000AD000F54050D0F8180903685B69984736
:10245000012084ED000A10BD0020FCE730B50546E0
:102460000FC985B06C4684E80F0040F279322146EE
:10247000284604F037FD0C4B03F1A002D3F8AC3131
:1024800093420ED19DF8001011F0040102D12046B4
:1024900015F008FA0548214604F0E0FD012005B0DA
:1024A00030BD0020FBE700BF107C0020102C002076
:1024B00000F5A040D0F8AC0103689B6C1847000001
:1024C00000F5A040D0F8AC010368DB6C18470000B1
:1024D00010B500F5A0531033D3F808421460D3F8B8
:1024E00004320B6000F50050D0F8D43E9B050BD4AD
:1024F00000F21C50D0ED006AD2ED007A9FED037A15
:10250000E6EEC77AC2ED007A10BD00BF35FA8E3C08
:1025100038B50D4D044629460C480FF0A3FC04F5D0
:10252000A04305F13C0183F8D50104F5A05010301B
:1025300004F5C0440FF02EFBD4EDDB7AF1EE677AA0
:10254000C4EDDB7A38BD00BF408F00202040002062
:1025500010B5044600F590701EF08AFF2046BDE8D5
:102560001040FFF7D5BF0000FFF7F2BF00F50050A5
:10257000D0F8D43E194214BF01200020704700005B
:1025800010B500F5A0430446D3F8AC0103689B6D79
:102590009847014604F5A1406C30BDE8104084F036
:1025A000F3BA0000FFF7ECBF38B5054B1C68236891
:1025B0000A461D68034B01462046A847002038BD47
:1025C0000C2C0020102C002070B52DED028B044641
:1025D000036804F500559B6D9847D5F8D43E1B065B
:1025E00018D5B5F98034B5F98214CA1A0B4402EB38
:1025F000D27203EBD37352105B1000EE902A00EE00
:10260000103A04F5A050F8EEE00AB8EEC00A103017
:102610000FF07EF85A4BB5F8B2241A7004F5C8458D
:1026200060F058FC3C3560F0A7F800212846FEF722
:10263000D7FF544E0123B0712846F3717CF03EF869
:1026400028B928467DF00AF9B0FA80F040093071C7
:10265000042120460CF018FA20B104F5B2406C3089
:1026600050F01AF928467CF029F8E0B994F81434AF
:1026700004F5C04504EB031341F28832D3F8C4617A
:10268000D5F8B433F31A93420DD904F59070FFF7DF
:1026900041FA022807D9C5F8B463204604F020FDAA
:1026A0000023C5F80832B4F9A4301BB9B4F8A2303D
:1026B000A4F8A430B4F8A430DFED338A07EE903AE2
:1026C000F8EEE77AB7EE008A88EE270AD4ED2B7A87
:1026D000F0EEE77AF4EEE87AF1EE10FA09D5B4F903
:1026E000A23007EE903AF8EEE77A88EE277A84ED8A
:1026F0002B7AD4ED2B0A26F0C9FF20BB50F0DCFF6B
:1027000040F27D124FF4801150F08EFF4EF064FCC9
:102710004EF0CCF804F54A501C30B0EE408A75F00B
:1027200085F804F54F50B0EE480A383075F07EF861
:10273000B0EE480ABDEC028B04F554502C30BDE8D5
:10274000704075F073B8D4ED2B7A94ED460AF0EE34
:10275000E77AF4EEE87AF1EE10FA09D5B4F9A2308E
:1027600007EE903AF8EEE77A88EE277A84ED2B7A36
:10277000D4ED2B0A26F08AFF0028BFD0C6E700BFA1
:102780005C230020AD91002000000034FFF71CBF47
:1027900070B500F5C046044696F98032002B2ADD5C
:1027A00006F072FD38BB04F5C8453C3528467DF07F
:1027B00055F800B328467BF081FFE0B185F05EFE5E
:1027C00004F5A0434FF47A72D3F8CC37C01A96F9C7
:1027D0008032534398420ED301221C212846FFF732
:1027E000D1F840B104F55B50034ABDE870400621C2
:1027F000303055F0B1BE70BDFC860C0830B52DED03
:10280000028B044683B000F5A05001A910300FF0F0
:10281000CFFB002874D004F5AF4595ED0D7ADDEDC2
:10282000017AB4EEE77AF1EE10FA05F1340507D536
:1028300004F5C8403C307BF04BFF08B1019B2B6096
:1028400004F500541820B4F98034052BB8BF0523D3
:1028500007EE903A04F2D443D3ED006AB4F982341F
:1028600007EE103AB8EEC77AF8EEE77A37EE077A55
:10287000C6EE870AB6EE007AF4EE470AF1EE10FAD9
:10288000C8BFF0EE470A9FED2E7A67EE877A9FED7C
:102890002D7A86EEA71AF0EE007AB4EE671AF1EE02
:1028A00010FA48BFB0EE671ADDED017AF4EEC77A90
:1028B000F1EE10FACCBF86EEA70AB0EE410A26F080
:1028C000F7FFB0EE408A20480EF05AFB90B91F483F
:1028D0004021FFF74BFE68B11D4BD3F83038012B78
:1028E00008D1F7EE007AB4EEE78AF1EE10FA58BF9D
:1028F000B0EE678AB0EE480A03B0BDEC028B30BD83
:1029000004F5C8403C307BF0E3FEB7EE008A0028B7
:10291000D9D046205FF080FDB4EEC80ADFED0D7A15
:10292000F1EE10FAD8BFB0EE480A87EE800AAFF099
:1029300063FA2F209FED081ADFED080ABFE700BFFA
:102940003333333F17B7D13820400020102C0020FC
:10295000107C0020000034428FC2D53F9A99193F65
:10296000F8B504465EF0C4F90368DB68984705468D
:1029700010B900252846F8BD204606F015FB04F5E1
:10298000A0460746D6F8AC0103689B6B984780B118
:102990000E4BD3F8AC0103685B6B984748B104F564
:1029A000005494F92935002BE3D0032BE1D03D46A8
:1029B000E0E796F8C031002BDCD004F5005494F920
:1029C000EC54023D18BF0125D4E700BF107C002065
:1029D00073B500F5A0431A46D3F8AC1193ED7D0A08
:1029E0001432914229D100F50052D2F8302FB2F9B9
:1029F0000840003C18BF012400F5495500F58050FF
:102A0000D3F84468D0F8082693F840382435B61A2D
:102A10005BB10B488DED010A4FF40061FFF7A6FD95
:102A20009DED010A80F00100C3B2224631462846DE
:102A300002B0BDE870407DF0B9BD0024DCE700BF06
:102A4000102C002010B5044605F0E0FE98B104F506
:102A5000A042D2F8443803F58C415031C2F84418F2
:102A600004F58051D1F808160029BEBFA3F58C43A8
:102A7000503BC2F844382046FFF7AAFFBDE810409B
:102A800004205FF0B5BC00002DE9F0412DED048B72
:102A900000F5005606F21C5393ED008ADFED358AEF
:102AA00028EE288A00F5A048BDEEC88AD8F8483834
:102AB00098ED7D9A18EE102A1A4408EE102A054661
:102AC00046205FF0A9FC06F2C443D3ED007AD8F8A3
:102AD000AC01B8EEC88A4346A0EE278A1433984268
:102AE000FDEEC87A17EE904A41D1D6F8343FB3F9DB
:102AF0000860003E18BF012603685B699847C0B9AB
:102B0000D8F8AC0103689B6B984790B905F5C047AE
:102B1000D7F8EC34022B0CD128460AF051F840B11A
:102B2000D7ED987A67EEA87AFDEEE77A17EE903A3D
:102B30001CB205F54E5705F580553C37D5F80C36D7
:102B4000E41A98F840383BB10B484FF40061FFF7A6
:102B50000DFD80F00100C3B2B0EE490ABDEC048B5C
:102B6000324621463846BDE8F0417DF05BBA00268A
:102B7000C2E700BF0000C842102C002010B5044678
:102B80000CF04AFB68B100B200EB4000C0EB001350
:102B900000EE103AB8EEC00ABDE8104013205FF016
:102BA00027BC2046FFF770FFF6E7000010B50E487F
:102BB000FFF7D6FEB0B10D4C04205FF02DFCD4F829
:102BC000300F5EF005FB04205FF012FC13205FF075
:102BD00023FCD4F8340F5EF0FBFABDE8104013205C
:102BE0005FF006BC10BD00BF102C0020104C002070
:102BF00070B52DED028B0446FFF7B2FE002875D0AC
:102C000004F5A0452A46D5F8AC31243293426DD064
:102C1000283293426AD02432934267D01C3A9342BE
:102C200064D00832934261D0403A93425ED004F5BA
:102C30000056F6EE008AD6F8300F5EF089F9B4EE51
:102C4000E80AF1EE10FA3EDDB0EE087AFFEE007A07
:102C5000E0EE077AB0EE670AD6F8482FD5F8443888
:102C600007EE902AB8EEE77A07EE903AF8EEE77AA8
:102C70005142E7EE007AFDEEE77A17EE900AC5F8CA
:102C8000440826F0B5FED5F8AC21C5F8440804F593
:102C9000A14318339A4222D0D6F8340F5EF058F987
:102CA000B4EEE80AF1EE10FAB0EE408A21DCFEEE56
:102CB000007AB4EEE70AF1EE10FA22D5B0EE087A07
:102CC000F7EE007A19E0FEEE007AB4EEE70AF1EED4
:102CD00010FAC1D5B0EE087AF7EE007AB8E72648C8
:102CE0004FF48051FFF742FC0028D5D0BDEC028B99
:102CF00070BDB0EE087AFFEE007AE8EE077AB0EE2B
:102D0000678A204605F082FD08B1B1EE488A06F5D3
:102D10009363D3ED006AD5F848389FED186A06F63C
:102D20004C7696ED007AB5EEC08A07EE903AF1EE59
:102D300010FACCBF28EE268A27EE488AF8EEE77A0A
:102D400066EE866AE8EE067A27EE067AFDEEE77A08
:102D5000FDEEE66A17EE903ABDEEC77A16EE902ABF
:102D600017EE101A17EE900AC5F8483826F040FE04
:102D7000C5F84808BAE700BF102C00200000C84280
:102D800070B5044604F5A04585F078FBD5F8BC3154
:102D9000C31AB3F5FA6F064603D9D5F8AC0106F0AD
:102DA00029FF2E4BC5F8BC61D3F8AC01026813684B
:102DB0009847002120460AF0B5F8DFED297AB0EEF9
:102DC000C00AB4EEE70AF1EE10FA45D504F5C043A7
:102DD000D3EDDB7AB1EE047AF0EEE77AF4EEC77A5F
:102DE000F1EE10FA38D504F58C6011F01BFDF6EE0B
:102DF000007AB0EEC00AB4EEE70AF1EE10FA2BD575
:102E000004F5C05595ED057AF0EE087AB4EEE77A50
:102E1000F1EE10FA05F114051ED504F549502430E1
:102E20007DF034FC04F54E503C307DF0ABF904F5F8
:102E3000545014307EF0D8F895ED007AF7EE007A11
:102E4000B4EEE77AF1EE10FA06D504F55A500830E0
:102E5000BDE870407DF01EBE70BD00BF107C00203C
:102E60000000003400F5005090F97734012BC3BF07
:102E700000F57E6090ED290ADFED047A9FED040AEB
:102E8000C8BF20EE270A46205FF0B2BA0000C84251
:102E9000000000002DE9F0412DED028B00F5A04867
:102EA0000546D8ED7D8A09F0A9FC0746D8F8AC01A3
:102EB00003681B6A984705F55456143698B14E4C72
:102EC000D4F80838002B0EDD85F0D8FAD4F808388D
:102ED000C01A40F6B733984205D8B4F9FC473046DB
:102EE0007EF08EF87AE005F5C04305F5005493F8BE
:102EF000E13443B1B4F90835002B04DD05F5405346
:102F000093F92A3513BBD8F8AC3105F5A045143533
:102F1000AB426DD00021B0EE680A30467DF008FE6D
:102F2000054604205FF078FA2AB207EE902A04F2F0
:102F3000BC43F8EEE77A93ED007AE0EE077AFDEE17
:102F4000E77A17EE904A3C4424B2C8E701212846AC
:102F500009F02CFE9FED297AB4F90835C0EE077A06
:102F600008EE103AD8F844389FED250AB8EEC88A22
:102F700028EE278A07EE903AF8EEE77A67EE807A35
:102F80009FED200A27EE800AAEF05AFDB4F9803496
:102F9000DFED1D7A20EE270A07EE903A08F505636B
:102FA00093ED007AF8EEE77A0021B4EEE77AF1EEDD
:102FB00010FA58BFF0EE477A80EE277A3046DFED00
:102FC000137AB0EE480AA7EE270AF0EE680A7DF001
:102FD0000BFFBDEEC00A10EE103A1CB2BDEC028B26
:102FE00020460B49BDE8F04141F2941226F010BD95
:102FF000391E18BF01218EE7107C002000A08C45EF
:103000000AD7233C35FA8E3C0AE81C41E02E654283
:103010006CEEFFFF38B500F540530546D3F81809AC
:103020000368DB689847014605F55A5008307DF083
:1030300013FD04B22846FFF793FC70B107EE904AE7
:1030400005F50055B8EEE70AD5F83C0F5EF0C0F87C
:10305000BDEEC00A10EE103A1CB220460349BDE88E
:10306000384041F2941226F0D3BC00BF6CEEFFFF53
:1030700038B590F81434B02202FB030393ED837A41
:10308000F7EE007AB4EEE77AF1EE10FA054600F5B5
:10309000A0441DD5002109F045FFDFED427AB0EED6
:1030A000C00AB4EEE70AF1EE10FA11D5D4F83038C0
:1030B000012B0DD0072B0BD0002384F8A03704F28E
:1030C000A474002323602846BDE8384009F096BB6D
:1030D00085F0D4F9D4F8A837C4F8A807C31AB3F513
:1030E0007A7F84BF002384F8A037284609F086FB46
:1030F000D4F83038012B07EE100A2DD0072B2BD037
:10310000B8EEC77ADFED286AC7EE267A05F50052D9
:10311000B2F9CC2400EE102AB8EEC00A27EE800ADD
:10312000DFED207AB0EEC07AB4EEE77AF1EE10FA75
:1031300014D4002384F8A03794F8A03705F55A502A
:103140000830DBB97DF070FBBDE83840174900B2AC
:1031500041F2941226F05CBC9FED150A94F8A0276A
:10316000002AE9D10122934284F8A027E4D0072B5A
:103170001EBF04F2A47300221A60DDE704F2A474F7
:1031800094ED007ADFED0B7A67EEC77A9FED0A7A4D
:1031900067EE877AFDEEE77A17EE901A7DF05CFC19
:1031A000D2E700BF0000003400A08C456CEEFFFFAA
:1031B00000000000E02E65420000C84270B52DED11
:1031C000028B00F5C446083682B00546304680F0D2
:1031D00095FF0446E8B905F50053D3F8302FB2F94E
:1031E000082082B905F5C042D2EDDB7A03F5996378
:1031F00093ED007AF0EEE77AF4EEC77AF1EE10FA8A
:103200004CBF01240024304680F08CFF002808BF0A
:103210000024304680F072FF28BB05F5A043D3F8A8
:103220009C37013319D0F4B99FED1A8A2846FFF76D
:1032300031FE07EE900AB8EEE70A8DED010AD4B927
:1032400015205FF0D5F89DED010A1A2002B0BDEC03
:10325000028BBDE870405FF0CBB8002CE4D028466C
:10326000FFF706FF02E02846FFF7D4FE07EE900ABC
:10327000B8EEE78ADAE71A205FF05CFB9DED010A01
:1032800008B9B0EE480A15205FF0B2F8B0EE480A6F
:10329000DBE700BF0000000010B500F5005303F5A8
:1032A0009362D2ED006ADFED137A9FED136A03F6A5
:1032B0004C7292ED007A03F57E6366EEA76A27EE04
:1032C000277AD3ED2A7A67EE867AFDEEE66ABDEEBE
:1032D000C77AFDEEE77A044616EE902A17EE101A2A
:1032E00017EE900A26F084FB04F5A044C4F84808C1
:1032F00010BD00BF0000C842A00CB34510B5044685
:103300000BF0C6FB031E2CDB04F5005191F977246A
:103310009A4226DD04F5A040D0F83048022C20D097
:1033200001F59A61D1ED007ADFED0E6AD31A66EEEF
:10333000E76A07EE102A07EE903AB8EEC77AF8EE81
:10334000E77AD0F8483887EE876A07EE903AF8EEC9
:10335000E77AE6EE867AFDEEE77A17EE903AC0F865
:10336000483810BD0000C842F8B52DED028B00F5BD
:10337000A0459FED440AD5F844389FED437A07EE07
:10338000903AF8EEE77A044667EE807A9FED3F0ABE
:10339000F0EEE76AF4EE476AF1EE10FAC8BFF0EE1D
:1033A000477A27EE800AAEF0BBF926F0A3F9B7EE14
:1033B000008AC8EE007A05F64C0704F50056C7ED02
:1033C000007A96F9A83453B3204605F01FFA30BBB3
:1033D000B6F98034012BB8BF012307EE903A05F50A
:1033E0000562F8EEE77AD2ED006A86EEA77AB4EECF
:1033F000C87AF1EE10FA15D840F6C4122449D5F86F
:10340000440826F0F5FAC5F84408D6F8482F40F6E7
:10341000C4139A42D4BFC6F8482FC6F8483FBDEC43
:10342000028BF8BDD7ED007AB4EEE77AF1EE10FA30
:10343000F5D588EE070A20EE000AAEF02BFBDFED93
:10344000157AD5F8440820EE270ADFED137A20EE2E
:10345000270A40F6C413FDEEC07A17EE904A9C424C
:10346000B8BF1C462246614226F0C2FAC5F844089D
:10347000D6F8483FA342D4BFC6F8483FC6F8484FE5
:10348000CDE700BF0AD7233C0000AA4235FA8E3CA4
:103490003CF6FFFFE02E65420000C84210B500F583
:1034A00040530446D3F8180903681B68984704F58D
:1034B0000053D3F8482F514226F09AFA04F5A0435E
:1034C000C3F844082046BDE81040FFF74DBF000098
:1034D00070470000012070470820704701207047A6
:1034E00070470000014B93F8B4047047104C002063
:1034F000034B93F9C80C003818BF0120704700BF78
:10350000104C0020014B93F9B6047047104C00207A
:1035100013B5064BD3F8AC014B690468009308312E
:103520000EC9646CA04702B010BD00BF107C002023
:1035300070470000002070477047000038B5254DE7
:10354000D5F8AC0103685B6898470F2834D80F287A
:1035500039D8DFE800F008360808080808080838F5
:1035600036363636363610241B4B93F8E92612B120
:1035700093F8E8360BB944F01004184BD5F8AC2199
:103580009A42A3F1080303D09A4218BF44F01004F2
:10359000134991F92915C1B19A4218D0032902D1D2
:1035A000104B9A4201D144F040040F487BF086F85A
:1035B00068B144F080040AE0182814BF01241824DC
:1035C000D2E71824D0E70124CEE79A42EDD144F0A7
:1035D000010038BD107C0020105C0020C47C00205D
:1035E000104C0020887C00204C90002008B5044836
:1035F00005F04AFE00280CBF0120022008BD00BFD4
:10360000102C0020F0B52DED028B8BB005460EF08E
:10361000EBFE4FF48071D0F8047290ED828AD0F8FE
:103620000C6204461448FEF7A1FF30B9134BDFEDDE
:10363000147A93ED007AA7EE678A2D7C84F01EFF42
:10364000D4F81823D4F81C33D4F81413089209932F
:1036500027221C23CDE900320390079103AA1E21E3
:10366000284604978DED058A069655F0A9FF0BB004
:10367000BDEC028BF0BD00BF102C00202C510020AF
:1036800035FA8E3C2DE9F041414E2DED068BD6F8F2
:10369000AC2106F1B4039A428AB073D0A6F5005368
:1036A00090F81080D3F81879D6F844389FED399AFD
:1036B00007EE903AD6F84838B8EEE7AA07EE903A07
:1036C0003B6838469B68F8EEE79A984707EE900A01
:1036D000F8EEE77A384667EE897A2AEE09AAFDEE17
:1036E000E77A69EE899A17EE903A1DB23B681B693A
:1036F000984707EE900AF8EEE77AA6F5A04067EE45
:10370000897AFDEEE77A17EE903A1CB206F2C4739E
:10371000D3ED008ADFED207AF4EEE78AF1EE10FABD
:1037200058BFF0EE678A02F08DFE3B68D6ED78AAAE
:10373000DFED1A7A5B6908EE100A38466AEEA7AA2E
:103740009847FCEEE88AB8EEC88A18EE903AB7229D
:1037500028EE098AADF824301A23CDE900323E2143
:1037600003AA40468DED03AACDED049A8DED058A9E
:10377000CDED06AA8DED070AADF82050ADF8224038
:1037800055F01EFF0AB0BDEC068BBDE8F08100BF0E
:10379000107C00200AD7233C00FF7F470000C8426E
:1037A00008B502480BF074F900B208BD102C0020D7
:1037B00037B50D46134840F2EF2203F093FB2C7807
:1037C00014F004040AD0696803220F4813F0A6FF1E
:1037D0000C4803B0BDE8304002F050BD01AA2146BC
:1037E000284614F06FF80028F2D0DDED017A9FED45
:1037F000077A67EE877A2246FDEEE77A17EE901A8F
:10380000E3E700BF102C0020508F00200000C842CA
:1038100010B5054C012384F8EB3657F0D3FB002399
:1038200084F8EB3610BD00BF105C00205AF07ABE61
:103830002DE9F0412DED028B4FF0000882B0CDE96B
:1038400000281E4F9FED1E8A0C461546B0EE480A12
:10385000B1F90220D7F8301F4FF47A7306465BF0B7
:1038600049F90123CDE90053B4F90020D7F8341FFA
:10387000B0EE480A30464FF47A735BF03BF9B4F986
:103880000420D7F8381F9FED0F0A43463046CDE994
:1038900000585BF02FF9CDE90058B4F90620D7F8AD
:1038A0003C1FB0EE480A4FF47A7330465BF022F9C1
:1038B00002B0BDEC028BBDE8F08100BF104C0020CF
:1038C0000000FA4400007A4438B5C5780B46352D1F
:1038D000044628BF3525352200211846B0F03CFBB0
:1038E0002A4604F10C01BDE83840B0F0EBBA000004
:1038F00010B5074B93F96C2940F24D3440F24D134B
:10390000002A08BF1C4657F0A5F9204310BD00BF90
:10391000107C002010B5044614F004FB204610BDB6
:1039200010B50B4C002384F8DF3758F045F8D4F875
:10393000AC2104F178039A4208D194F858382BB995
:1039400004F65400BDE810402BF0C4BD10BD00BF0C
:10395000107C002013B5124C94F89E1204F5A87048
:103960000CF06EFA78B194F89E1204F5A8700CF081
:10397000D5FC40B194F89E1204F5A87002B0BDE8E1
:1039800010400CF00DBD0EF02FFD01A90EF010FB44
:1039900018B19DED010A02B010BD9FED020AFAE7D1
:1039A000104C00200000000008B5084BD3F8B82EDA
:1039B000002A03DCBDE8084057F0C4B803F6D8502D
:1039C00054F046F990ED000A08BD00BF104C0020ED
:1039D00008B51148D0F8AC2100F1AC039A4214D0DC
:1039E000B0F9C4319BB990F8693783B990F8C13107
:1039F0006BB990F8193863B9A0F5A04005F044FC04
:103A000000280CBF0320042008BD0220FCE705208D
:103A1000FAE70620F8E700BF107C002030B5224C02
:103A2000D4F8AC2104F1B4039A4291B0054638D0E1
:103A3000002304F59A50029313F05AFE014620B970
:103A400002AA04F59A5013F09FFE2C7C84F016FD18
:103A5000164BDDED027A9FED167AD3E9D22305935A
:103A60000023F8EEE77A0793089309930A930B93E0
:103A70000C930D930E934FF6F853ADF83C300023A2
:103A8000CDE9030267EE877A96228DF83E30332324
:103A9000CDE90032572103AA2046CDED067A55F034
:103AA0008FFD11B030BD00BF107C0020108C0020B5
:103AB0000AD7233C10B557F0C7FA044678B909482D
:103AC000D0F8AC2180F8DF4700F178039A4206D1A4
:103AD00090F858381BB900F654002BF0FBFC204638
:103AE00010BD00BF107C00200120704708B5034BBB
:103AF000D3F8AC0103685B68984708BD107C0020D0
:103B000030B587B005460EF06FFC04462D7C84F07E
:103B1000A9FCD4F88422D4F88832049205930021B9
:103B20001023CD22CDE900320290039102AA42F681
:103B30000C31284655F044FD07B030BD30B52DEDB1
:103B4000028B89B005460EF04FFC00F55A7393E8DE
:103B5000070002AC84E80700DDED020A9DED030AD0
:103B60002D7CF1EE600AB1EE400AADF0FBFF20467D
:103B7000B0EE408A28F080FDDFED0B7A049B0793BE
:103B800028EE278A0C230122CDE90032A82105AABC
:103B900028468DED058A8DED060A55F011FD09B018
:103BA000BDEC028B30BD00BFE02E6542282938B540
:103BB000054623D007D824292BD0272911D01B292B
:103BC00008D1012413E0432937D008D84029F8D080
:103BD000422928D02846BDE838405BF0E7B8532991
:103BE000EEE7122154F0EAFE044610B90024204604
:103BF00038BD297C13484DF08FFDF8E7162154F0AD
:103C0000DDFE04460028F1D0297C0E484DF05EFE12
:103C1000EDE70C2154F0D2FE04460028E6D02846F9
:103C2000FFF78CFFE3E7102154F0C8FE044600289C
:103C3000DCD02846FFF764FFD9E7017C024880F01A
:103C40005BFABEE77C850020188E0020F0B52DEDD4
:103C5000028B05468DB01646B0EE408A0C46002910
:103C600030D0007C55F042FC0746287C56F042FBE1
:103C700000F121039F4207D2287C0DB0BDEC028BDE
:103C8000BDE8F04054F088BE63690893636A226916
:103C9000CDF82530236AA069E1680792CDF8293074
:103CA0006222212327680590CDE900320691287C05
:103CB0000397192303AAC2218DED048A8DF824608D
:103CC00055F07EFC0DB0BDEC028BF0BD70B52D4DF6
:103CD000D5F8AC2105F1B4039A42044650D0A5F5BD
:103CE0004056B6F85A35DB0708D5A5F5005393EDD5
:103CF000E40A012203F56371FFF7A8FFB6F85A350D
:103D0000980708D520490B4693ED000A0439022292
:103D10002046FFF79BFFB6F85A35590708D51B49CF
:103D20000B4693ED000A043903222046FFF78EFF6D
:103D3000B6F85A351A0708D515490B4693ED000A0F
:103D4000043905222046FFF781FFB6F85A35DB0615
:103D500016D5D5F83038042B12D10EF045FB0546A8
:103D60000C4880F0F9F995EDC70ADFED0B7A0146B2
:103D700020EE270A20460622BDE87040FFF766BF06
:103D800070BD00BF107C0020FC600020706200202D
:103D9000CC620020188E0020E02E654270B50446EB
:103DA0000E461DF0A3FB90F8F412B02303FB0101B3
:103DB000DC31204603F006FA054698B13EB10EF01C
:103DC00013FB90F87C3243F0020380F87C3204F558
:103DD000A04304F5A144D3F8AC011034A04201D1B2
:103DE00005F054FE284670BD73B516460191044691
:103DF0000EF0FAFA01990DF023FF054698B13EB195
:103E00000EF0F2FA90F87C3243F0020380F87C3234
:103E100004F5A043D3F8AC0104F5A1431033984254
:103E200001D105F033FE284602B070BD30B505461D
:103E300085B00C46D1E9040125F0F0FF40B1684699
:103E400013F066FC6A46214628465AF0C3FD08B9BD
:103E5000022067E0344840F24F32694603F042F8EE
:103E6000D4ED037AF4EE677AF1EE10FA22D69FEDE4
:103E70002F7AF0EEE77AF4EEC77AF1EE10FA54BF3B
:103E8000012200229DF80030294962F3410368466F
:103E90008DF8003013F0A6FD0028D9D125486946D9
:103EA00069F074FD40B951F019FA0522162150F05D
:103EB000CDFFCDE70022E5E7D4ED017AFDEEE77A0C
:103EC00017EE903ADB0706D41B4B03F1A002D3F8A0
:103ED000AC31934225D11949134802220AF0EAFB7A
:103EE0009DF8001011F0040102D1684613F0DAFCCD
:103EF0000D48694603F0B2F894ED020AB4EE400AA8
:103F0000F1EE10FA0BD6B5EEC00AF1EE10FA06DDAE
:103F10009DF800100948C1F3400106F031FE002071
:103F200000E0042005B030BD102C0020000000345B
:103F3000408F0020304F0020107C0020B07C0020FB
:103F400010B52DED028BD1ED017A91ED008AFCEEDA
:103F5000E77A8AB0CDED037A9DF80C1005AA0446E5
:103F60005AF022FDC8B1DFED0E7A059B009368EE92
:103F7000277A0022FDEEE77A114617EE903A06A85E
:103F800013F0E6FB23682046D3F8CC3006A9984707
:103F900000200AB0BDEC028B10BD0220F9E700BF83
:103FA0000000C84237B5124DD5F8AC0103681B6A52
:103FB0000C46984740B9D5F8AC2105F178039A42F0
:103FC00002D0042003B030BDD4ED007AD4ED020A53
:103FD00094ED010A0748FCEEE77ACDED017A9DF8F1
:103FE000041003F0A3FE0028EBD00020EAE700BF96
:103FF000107C0020102C002008B5D1ED007A9FED38
:10400000087A0848F0EEE77AF4EEC77AF1EE10FA93
:1040100054BF0121002104F0F3FB002008BD00BFC4
:1040200000000034102C002010B5D1ED007AFCEE19
:10403000E77A17EE903A9CB2012C02D0022C06D0FF
:1040400084B91148214664F06FFE002010BD0F486E
:1040500090F860395B0707D55BF056F90C4A0521EB
:1040600054F07AFA0420F1E790F94C391BB95BF06F
:104070004BF9084AF3E7A0F5A04008F07FFA0028C2
:1040800014BF00200420E1E75C850020107C0020A4
:10409000188D0C08338D0C0838B58B8BC02B05465A
:1040A0000C4631D8B12B0BD8112B00F09480142B77
:1040B00000F0948021462846BDE838405BF06ABF96
:1040C000B23B0E2BF6D801A151F823F03B41010879
:1040D000B5400108B5400108B5400108B5400108E8
:1040E000B5400108B5400108B5400108314101085B
:1040F000B5400108554101088D410108B54001084E
:104100004541010827410108D42B08D0B3F5967F1B
:1041100047D0D02BCED1BDE83840FFF785BFBDE8F2
:104120003840FFF769BF2146BDE83840FFF77EBE43
:104130002146BDE83840FFF703BF2146BDE83840BF
:10414000FFF730BF94ED000A2748FDF7F9FFD8B11B
:1041500000201AE0254C94F8D531ABB1244904F67F
:1041600054002BF0B5FA78B1012384F88D3802227F
:1041700004F17801A4F5A0400AF09CFA0028E7D1E8
:104180001A4B002283F88D28042038BD174C94F870
:10419000D531002BF8D0164904F654002BF01CFA48
:1041A000E1E7D1ED007A9FED137AF0EEE77AF4EED5
:1041B000C77AF1EE10FA14D5D1ED017AF0EEE77A74
:1041C000F4EEC77AF1EE10FA0BD50B49022206483D
:1041D0000AF070FABCE709490222F8E7084902220E
:1041E000F5E70220D1E700BF102C0020107C002052
:1041F000408F002000000034887C0020A87C002034
:10420000A07C0020F0B5414CD4F8AC2104F1A0030F
:104210009A428FB00D4677D1CE78272E28BF272619
:104220002722002104A8AFF097FE324605F10C01C9
:1042300004A8AFF047FE059B9DF836500093069BFF
:104240000193ED43079B0293EDB2089B03938DF816
:10425000365084F013F915F0810F05F087070646F4
:1042600001D1802F12D1684627F06EF9DFED287A50
:10427000C4F8006820EE270ADFED267A20EE270A30
:10428000BDEEC00A10EE103AC4F8F43715F0820FF4
:1042900001D1802F12D1684627F070F9DFED1C7A2A
:1042A000C4F8046820EE270ADFED1A7A20EE270A08
:1042B000BDEEC00A10EE103AC4F8F83715F0840FBE
:1042C00001D1802F12D1684627F068F9DFED107A0E
:1042D000C4F8086820EE270ADFED0E7A20EE270AE0
:1042E000BDEEC00A10EE103AC4F8FC376B060BD5D1
:1042F000DDED0C7A9FED077AC4F8106867EE877AD7
:1043000004F60C03C3ED007A0FB0F0BD107C002062
:10431000E02E65420000C84230B51F4C91B00846FF
:1043200002A9FFF7D1FAD4F8AC2104F1A0039A4214
:104330002FD19DF83C30072B2BD104F58054D4EDC0
:10434000D17ADDED056A9FED157AF8EEE77AE6EEB3
:10435000C77AFDEEE77AC4EDD17A5AF0D5FFD4F8EA
:104360001C23D4F8443352689FED0D7A9B1A07EE54
:10437000903AF8EEE77A054667EE877A17EE900AEC
:10438000FCF7C2F8074ACDE900010621284654F09F
:10439000E3F811B030BD00BF107C00200000C8421F
:1043A0000AD7233C4C8D0C0810B51D4B03F1A0021D
:1043B000D3F8AC319342044696B008460FD108A911
:1043C000FFF782FA9DF8541003AA20465AF0ECFA3F
:1043D00038B95AF099FF134A042154F0BDF816B0C9
:1043E00010BDBDF8503023F004039BB2002BF6D073
:1043F000DDED0B7A9FED0C7A039B009367EE877AD5
:104400000022FDEEE77A114617EE903A04A813F069
:104410009FF9236804A9D3F8CC3020469847DEE7FB
:10442000107C0020608D0C080000C84230B48D7AEA
:104430004B7A43EA0523CD7A43EA0543562B0446DB
:104440000A461BD008D8522B12D0542B13D020462A
:10445000114630BC5AF078BF03F18073863B23F0DD
:104460007F43012BF3D8017C064830BC4DF0F6BAEF
:1044700030BCFFF7C7BE30BCFFF74EBF30BCFFF704
:1044800093BF00BF7C85002000207047C820704784
:1044900001207047002070470020704790F89C3042
:1044A0008B4286BF283150F8210000207047000061
:1044B00090F89C308B4286BF283150F821000020B4
:1044C0007047000003207047014B93F8B204704717
:1044D000104C002070B504464C4808F01DFD18B182
:1044E000E36A43F40003E362484808F015FD88B12D
:1044F00046205DF091FFDFED467AB4EEE70AF1EE7B
:1045000010FA07D8236B43F400032363636B43F46F
:1045100000036363E36A43F4F843E3623D4BD3F87B
:10452000AC0103685B6898470138172814D8DFE8A6
:1045300000F03A420C4442424242133A3A3A3A3A82
:104540003A13131313131313133A334A92F8E8363A
:104550008BB392F8E9268AB3304B93F80432012BDF
:104560003DD0022B44D02E4B1D68DDB12D4E284688
:1045700096F8221F47F06EFFA0B1E36A43F4807300
:10458000E36296F958351BB1236B43F480732363C0
:1045900096F8221F284647F095FF18B1636B43F445
:1045A0008073636370BDD4E90C2342F4E04243F4AA
:1045B000E04322636363012300E00023216B41F4A5
:1045C00080622263626B42F480606063002BC3D020
:1045D00041F4406142F4406221636263BCE7E36AF4
:1045E00043F48003E362236B43F480032363BAE75D
:1045F000E36A43F48003E362236B43F480032363A1
:10460000636B43F480036363ADE700BF102C0020AD
:10461000000000B4107C0020105C0020108C0020F2
:1046200058920020104C002013B54FF44470CDE98F
:10463000002113F06FFC044628B1DDE900215BF096
:10464000A5F8024B2360204602B010BD608F0C0815
:1046500000207047002070470020704700207047FE
:1046600000F514501430704700487047E8B40C0847
:1046700000F5A040D0F8AC0103685B681847000063
:1046800000F5A0431846D3F8AC3178301B1A5842D5
:10469000584170479B20704730B500F5A04303F6A2
:1046A000480353F8042CDFED2A6A07EE902AB8EE8F
:1046B000E77AD3ED007AF8EEE77A85B0044627EE84
:1046C000267A67EEA67A00F5A050002301A91030E3
:1046D00003938DED017ACDED027A04F58F550CF040
:1046E00033F804F54E520C32692128464FF0C2FCD3
:1046F00004F5535228326A2128464FF0BBFC04F5DA
:10470000405393F92A2542B903F5A463D3ED007A07
:10471000F5EEC07AF1EE10FA06DD04F559521C32BE
:104720006B2128464FF0A6FC04F55A540834204665
:104730007CF0B4F928B104F130026D2128464FF025
:1047400099FC0DF051FE0DF077FB05B030BD00BFB8
:104750000AD7233C10B54FF4801104460AF094F9AF
:1047600010B12046FFF798FF4FF4800120460AF071
:104770008BF928B124F020FBBDE8104022F0AEB93F
:1047800010BD000070B500F5A05590B000231035A5
:10479000029302A9002304460DF1070228468DF872
:1047A00007300DF00BFC03A928460CF039FC08B9C2
:1047B0002C4B03933022002104A8AFF0CDFB04F56D
:1047C000A046A3238DF8103095238DF8113083F087
:1047D0005DFED6F84438ADF81B3004F58053CDF8B3
:1047E0001300D3F80826ADF81D20D3F80C36D6F800
:1047F0004828CDF817104620ADF81F20ADF821301D
:104800005DF00AFE10EE103A1520CDF823305DF071
:1048100003FE10EE103ACDF8273004F53F539FED1C
:10482000127AD3ED317A67EE877A284617EE903AFE
:10483000CDF82B30029BCDF82F309DF807308DF846
:104840003330039B0D930DF0BFFDD6F8E8318DEDAD
:104850000E0A302204A904F58F500F934FF046FD45
:1048600010B070BD2292CA7F0000C84270B58EB0F1
:104870003522044600216846AFF06EFBA3238DF875
:10488000003095238DF80130012304F5A0468DF802
:10489000023083F0FBFD04F5405506F2C473CDF8F9
:1048A00003001B68D5F81809CDF80710CDF80B30B8
:1048B00003681B699847ADF80F00D5F8180903681D
:1048C0009B689847ADF811001C4801F0BBFDADF89E
:1048D0001300D5F8180903685B69984710EE103A81
:1048E000D5F81809CDF8153003689B69984710EE84
:1048F000103ACDF81930D6F8E031CDF81D3004F576
:10490000C0433522D3F84813CDF82110D3F84C1307
:10491000CDF82510D3F84413D3F8F434CDF829108A
:10492000CDF82D306946D6F8D831CDF8313004F5C0
:104930008F504FF0DBFC0EB070BD00BF102C00207C
:1049400030B587B01622044600216846AFF004FB5C
:10495000A3238DF8003095238DF8013002238DF8C4
:10496000023083F093FD04F5A045CDF80300204606
:10497000CDF8071004F088FC05F634038DF80B0021
:104980001B680393124B1B68D86A90F89C308DF813
:1049900010300368DB69984795F819388DF81230A4
:1049A0008DF8110024F008FA23F0FCF9D5F830381E
:1049B0008DF813008DF81430162295F81A388DF8FA
:1049C0001530694604F58F504FF090FC07B030BDAC
:1049D0000C2C002010B58AB027220446002168461E
:1049E000AFF0BAFAA3238DF8003095238DF801308B
:1049F00009238DF8023083F049FDCDF8030004202F
:104A0000CDF807105DF008FD10EE103A1320CDF838
:104A10000B305DF001FD10EE103A4620CDF80F305E
:104A20005DF0FAFC10EE103A1520CDF813305DF071
:104A3000F3FC10EE103A0320CDF817305DF0FCFCCB
:104A400010EE103A1A20CDF81B305DF0E5FC10EEA8
:104A5000103ACDF81F3004F5A0432722D3F8F431E3
:104A6000CDF82330694604F58F504FF03FFC0AB073
:104A700010BD000013B5044600F58F5001904EF0B4
:104A800067FF01984EF0FEFF04F58053019893F9FB
:104A900010330BB14FF09EF8204602B0BDE8104035
:104AA000FFF798BF7047000010B500F5A04304461B
:104AB000D3F8AC0103685B68984704F500530146DE
:104AC00093F8342404F58F504FF0D0FD04F5A05036
:104AD00010300DF0D5FE04F59070BDE810401BF0CD
:104AE0006FBD00009FED020A002245F067BE00BFC7
:104AF0000AD7233C1C4B70B5044640F8043B5BF0DE
:104B000077FF1A4E1A4B6360542560195CF026F942
:104B100066513035B5F5557FF7D104F555705EF027
:104B20006FF8144A04F5EE6002F66C3180F086F9F5
:104B300004F67C15FF2384F88C3984F894390E49E7
:104B4000284646F0D1F90D4B1A6812B10C4883F093
:104B500063FC1D60012320460A4984F8C13946F0F0
:104B6000C3F9204670BD00BF703A0020C4DF0C08B6
:104B7000D8DF0C0884500020901B0E08F89B002002
:104B800064CC0C0888CF0C082DE9F04100F51251D7
:104B90009AB00D22303104464DF094FF0022BF48F8
:104BA000BF4E272145F082FD042100205EF002F86F
:104BB000132101205DF0FEFF462102205DF0FAFF87
:104BC000152103205DF0F6FF5DF060FD46F092FBDD
:104BD000B44A138843F0040313804FF000080AAF6F
:104BE000002110223846AFF0B7F901238DF830309C
:104BF0003388ADF8283005A973680B93384645F023
:104C00005DFCC8B19DF91430002B15DD5CF070F827
:104C10009DF81410036801391B68C9B2984758B150
:104C2000051D284645F0E8FB30B9B368ADF81830EB
:104C300006A9284647F004F808F10608B8F12A0F3B
:104C400006F10C06CCD1984800220DF10B0145F07D
:104C5000BBF906AD064620B345F0CEFB08BB934B2F
:104C60000FCB85E80F0004A9284645F027FC002853
:104C700040F03C814FF004088D4B0FCB87E80F00CC
:104C800005A9384645F01AFC28B105A845F0B4FB43
:104C900008B148F0010803A930468DF80C8046F0B1
:104CA0007DFF844B0FCB85E80F0003A9284645F014
:104CB00005FC002846D00998002204A945F084F993
:104CC000064600283ED045F097FB0546002839D11E
:104CD0009DF80C30013BDBB2032B96BF764A0346AE
:104CE000D35C8DF828303046394646F057FF73487C
:104CF000002205A945F068F9064669F089F878B1FF
:104D000069F084F890F8302090F8281090F8483036
:104D1000114490F840200A44D34214BF01250025D5
:104D200086B130469DF90C8045F066FB50B91DB147
:104D3000B8F1000518BF0125394630468DF82850D6
:104D400046F02CFF04F515500022B7EE000A0121B1
:104D50000C3045F033FD04F513500022B7EE000A85
:104D60000221283045F02AFD012304F50551009366
:104D7000534A002310318E2045F09CFC94F9DCC985
:104D8000BCF1000F1AD14F4E0FCE3D460FC50FCECE
:104D90000FC50FCE0FC596E80F0085E80F006246DD
:104DA0000421384645F082FC9FED470A474846F00B
:104DB00043FC4748B7EE000A46F03EFC012504F5E7
:104DC0000C51444A00950023203140F2051045F073
:104DD00071FC04F5145002211C30FFF783FE04F52A
:104DE000125003210430FFF77DFE04F51250032119
:104DF0000C30FFF777FE04F5145003211830FFF74D
:104E000071FE04F5145002212030FFF76BFE04F50B
:104E1000125002211830FFF765FE04F512500221EE
:104E20001C30FFF75FFE04F5125002211430FFF72B
:104E300059FE04F5C44008307FF0F4FA264A13689E
:104E4000D90709D42549156004F50A5330330B609E
:104E500004F597531433CB6004F515501F49022213
:104E60002030012545F078FC1D4A0095002304F50B
:104E70008F51FD2045F01EFC1A4B1A68D20705D44D
:104E8000194A1D6004F59B5408341460164801212A
:104E900045F07EFC1AB0BDE8F08100BFC4CC0C0820
:104EA00034CF0C083C92002088CC0C08DC810C0824
:104EB000EC810C08FC810C08C0CC0C0893CC0C08CD
:104EC00044F50C080C820C0800000000A0CC0C0873
:104ED000AFCC0C08D4160E08042C002000220020B1
:104EE000E88D0D08082C00201822002004A845F0A9
:104EF00083FA00283FF4BEAE4FF00C08BCE600BFBA
:104F00007047000000207047002070470020704765
:104F10000020704700207047704700000020704755
:104F20000020704784B001A880E80E0004B0002083
:104F30007047000000207047002070477047000055
:104F40001020704700487047D4DB0C0800487047B9
:104F5000E4DB0C0800207047704700000120704718
:104F60000120704700207047002343608360C360C6
:104F700003614361002303767047000010B50446C7
:104F8000FFF7F2FF0023637610BD0000027E531C82
:104F9000DBB2042B037600EB820288BF002382ED94
:104FA000010A88BF0376704710B50446FFF7EEFF8D
:104FB000D4ED017A9FED107A94ED020A637E77EECC
:104FC000877A042B77EE807A94ED030A94BF01333D
:104FD000052377EE807A94ED040A637677EE807A83
:104FE000637E94ED050A77EE807A00EE103AB8EE13
:104FF000C00A87EE800A10BD0000000010B504460C
:1050000012F090FF204610BD03F082BE03F08AB874
:1050100003F0E2BA03F092B801F0C6BC01F072B836
:1050200001F0FAB901F03ABAFDF7B2BBFDF730B8BA
:1050300070B5234B036000F540530446D3F8AC0829
:10504000204AC3F8F02608B112F070FF1E4B23600F
:1050500004F5005393F8EC2042B9D3F8E8502DB191
:10506000284620F0B3FD284612F05CFF04F59A5064
:105070000C3078F07FFD04F5985010305EF0C8FEDB
:1050800004F6E46504F68466B54204D0183D28466B
:1050900020F0F2F9F8E70D4BC4F8C83804F62820E0
:1050A00052F0B2FA04F6FC1052F0AEFA04F65C10BC
:1050B00052F0AAFA04F5136052F0A6FA204670BD29
:1050C000E0C20C08DCA80D08E8860D08E4470D08CE
:1050D00038B54D4B044640F8043B62F00FF804F13C
:1050E000100010F073FE04F168004BF04DFC04F565
:1050F00090701AF01FFE04F58C600FF069FB04F24B
:10510000845012F015FF04F6C80021F017FE04F5D4
:10511000666061F0D1FD04F5736047F0C1F804F5F5
:105120008F504FF017F804F59750143067F0AAFD30
:1051300004F5985010305EF053FE04F59A500C3090
:1051400078F004FD04F59B5008304BF0DFFF04F5C8
:105150009C500C3063F0B0F904F5805300252B4AC5
:1051600083F8B05304F59D53103304F59E5013603B
:1051700041F0C0FE04F5A050294610300BF028FC89
:1051800004F5D350183072F057FD04F5FB501C3075
:1051900075F0FCFC04F50250143077F031FE04F594
:1051A0000350383078F066FA04F5055010300AF0F4
:1051B00073FC04F50A50303073F0B6FA04F50C5065
:1051C0001349083045F090FE04F50C50203068F08B
:1051D000F5F804F50F501C3079F054F804F500533D
:1051E00004F5115083F834540A4D0C3079F06CF901
:1051F0002B6813B1084883F00FF92046074945F0A2
:1052000073FE2C60204638BDE8860D08649B0020A4
:10521000041D0E0890920020ECDB0C08F0850D08B0
:105220002DE9F04F2DED028B04469FB0FFF750FFA4
:10523000DE4B236004F515502030FFF75BFC04F5CE
:105240003C5028307AF0B6FC04F5005504F51353B1
:105250003A33C5F8503F04F53D50062385F8543FD6
:1052600004F511583C3004F5A05704F5C44B5EF02A
:10527000C9F904F5405608F1340810374FF40063BB
:105280000BF1080BC5F8FC3FC5F8F07FC5F8F48FAB
:10529000C5F8F8BF5A2305F57E6586F87C304FF0D7
:1052A0007E53C5F85C31C24BC5F86031C14BC5F8BF
:1052B000643104F54650C04BC5F86831C5F8CC31AF
:1052C0003C3052F0C1FC04F5475004F53F5A083019
:1052D00052F0BAFC4FF00009B84BC6F8D8310AF1C9
:1052E000200A86F8F0910AF5FC70FFF73DFEB44BFA
:1052F000B449C6F8D83186F8F191504645F0F4FD2E
:10530000B14BC6F800A2C6E97E370023C6F82C329E
:10531000C6F8343204F54755012304F5495086F8A0
:105320003C323835103012F0F3F9A84986F8609213
:10533000284645F0D9FD04F54950414624307AF01D
:10534000EFFF04F54E5041463C307AF04DFC04F539
:105350005450414614307BF0ADFB2C22494606F5F3
:10536000D760AEF0F9FD04F55A509949083004F5BC
:105370005B5945F0B9FD09F13009964BC6F8F03696
:1053800009F1140081F04AFF04F55C5304F55E5204
:1053900028330C3218460F920E9357F0EBFA0E9BFF
:1053A0000F9A14339A42F5D10723C6F8B038002378
:1053B000A6F8B4384FF4CB7012F0B2FDC6F8AC08C2
:1053C00004F56250383081F029FF04F563503C3019
:1053D00081F024FF804B1A680AB9C3F800907F4B14
:1053E000C6F8F03604F564504FF48051C6F81859E9
:1053F0001C3010F0EDFD04F566501C3043F040F910
:1054000004F567501C3046F0D1FC04F5675030308D
:105410006AF090FC04F5A04004F5A0450C3004F0BF
:1054200017FB6F4BEB602846143004F011FB6D4BFB
:105430006B6128461C3004F00BFB6B4BEB6128467C
:10544000243004F005FB694B6B62B7EE008A002341
:1054500028466B642B64EB6385ED0E8A4C3004F0B8
:10546000F7FA634BEB642846543004F0F1FA614BD1
:105470006B6528465C3004F0EBFA5F4BEB65284621
:10548000703004F0E5FA5D4B2B672846783004F065
:10549000DFFA5B4BAB6704F5A140103004F0D8FA9B
:1054A000584BC5F8903004F5A140183004F0D0FAFC
:1054B000554BC5F8983004F5A140203004F5A149BA
:1054C00004F0C6FA09F12C09504BC5F8A030484643
:1054D00004F0BEFA4E4BC5F8AC3004F5A1403430B0
:1054E00004F0B6FA4B4BC5F8B43004F5A1403C309B
:1054F00006F086F804F5A140643004F0A9FA464BA2
:10550000C5F8E430454BC5F8EC3004F5A1404FF444
:10551000C0534349A5F840316C3045F0E5FCFE230B
:1055200085F8B831052385F8D4314FF0FF33C5F83D
:10553000DC313C4B119304F5A3403B4B85ED7D8A58
:105540004FF40071C5E96B99224600937830354BD2
:1055500010940FF023FF4FF0FF33C5F89C3705F28E
:10556000AC73144ADA600023C5F8F437C5F8F8378D
:10557000C5F8FC37C5F80038C5F80438C5F8083850
:105580000323C5F8303805F64C0383ED008A274B1A
:10559000C5F87438264BC5F87C3804F5B140254B66
:1055A000C5F88438C5F8704846E000BFE0C20C0872
:1055B000000080BF0000B4420000B4C258DC0C08F8
:1055C00068DC0C08AC580E0820560E08C8550E08AA
:1055D00064500E08DCA80D08D49500203C900C08FF
:1055E00038E60C083CEA0C085CED0C0880E40C087A
:1055F00048E70C08D0E70C08B0E60C08B8E50C0842
:1056000034E50C08C0E90C08C8E80C0850E80C08A0
:10561000A0DC0C0848E90C08D8EC0C0890DC0C085D
:105620003C630E0809500108108D0C080D5001084C
:105630001150010815500108C5F87848C5F8804890
:10564000183012F065F804F5B140343012F060F80B
:1056500004F5B140503012F05BF87E4BC5F8E438E9
:1056600004F5B0494FF0FF33A5F8E83809F1EC0034
:1056700012F04EF809F154094FF0FF32764BC5F89D
:10568000482948467549C3F8009045F02DFC4FF66F
:10569000FF73A5F890384FF0FF33A5F8AC3804F548
:1056A000B2406F4B6F494C30186045F01DFC04F55B
:1056B000B2406C304CF0FAFD6B4BD6F818291294BE
:1056C000CDE91334694BCDE91534694BCDE9173475
:1056D000684BCDE91934684BCDE91B34674B1D93FA
:1056E0001EA911E903000CAB83E80300DDE91A01F0
:1056F0000AAB83E80300DDE9180108AB83E8030087
:10570000DDE9160106AB83E80300DDE9140104AB13
:1057100083E80300DDE9120102AB83E8030004F52E
:10572000C0464946CDE9002853463A46584604F556
:10573000C5497EF07FFC09F11409514BC6F894323B
:1057400009F13C0011F0E4FF4E49484645F0CCFB1E
:105750004D4BD3F80080B8F1000F02D04B4882F0D7
:105760005BFEC3F8009007F51B77494BC6F89432EF
:1057700004F5C640C6F81C7386F8988286F89D82A8
:1057800086F8C182203011F0C3FF04F5C6403030E6
:1057900011F0BEFF04F5C640403011F0B9FF1C22E5
:1057A000414606F55470AEF0D7FB04F5C84704F542
:1057B000C7403C3738305EF061FC384678F03EFF39
:1057C000344B3549C6F83C34384645F08DFB334AF6
:1057D0003349116004F5C843743314271FFA88F065
:1057E00007FB001208F10108127C002AF6D12D4AAD
:1057F00010802D4A17680FB12C48B0E704F5C84057
:105800007830136078F004FF294BC6F87834294BC0
:10581000C6F88834642386F88C34274BC6F8C03425
:1058200004F5C940254BC6F8C4342549083045F075
:105830005BFB244BC6F8883420460123C6F8E87485
:1058400086F8F07485F8DC371FB0BDEC028BBDE83C
:10585000F08F00BF0000FFFF8091002030560D0840
:105860006C9B002094BC0D08195001081D500108C4
:105870002150010825500108295001082D50010828
:1058800040DC0C0844540E087CA3002000DC0C080B
:10589000FCDF0C0870860C0848860C084C9200202F
:1058A00048D10C084A920020089200201CDC0C0809
:1058B000B0860C0878DC0C0898F10C08F0F10C08A4
:1058C00010B00D0870F30C0810B582F0E7F8064C24
:1058D000064B18602046FFF7A3FC2046044A054902
:1058E000BDE81040ABF0F6BD102C00200C2C0020C1
:1058F000D0EF0020315001080069C0F3401070471C
:105900000F299DBF302303FB01005030002070475A
:10591000014B93F9F9047047104C0020014BD3F868
:105920003C0F7047104C002008B503689B689847EF
:1059300030B9044B93F8C601B0FA80F0400908BDB5
:105940000020FCE7107C002008B5044807F072F83E
:1059500010B9034B93F8C00108BD00BF102C002004
:10596000107C0020022A10B50C4605D1BDE810407D
:105970000948352208F076BF084BD3F8AC0103681C
:105980005B689847A04205D15BF0B2F9BDE81040D2
:105990005BF038B910BD00BF102C0020107C002037
:1059A000012910B50C4614D0022907D0D1B90E4BED
:1059B000C3F8E81459F0A8FC0C4A05E00A4BC3F8F8
:1059C000E81459F0A1FC0A4ABDE81040062152F043
:1059D000C3BD59F099FC074A062152F0BDFD024BA8
:1059E000C3F8E84410BD00BF108C0020BBDD0C08DC
:1059F00090DD0C08A4DD0C08012903D0022914BF96
:105A000000210221014BC3F8BC1E7047104C00203E
:105A1000012902D0022900D011B9024BC3F8EC14BD
:105A2000704700BF108C0020622910B400F38880FA
:105A300047291ADC402900F0978008DC162951DC40
:105A4000032904DD504B01248C40234053B95DF8F9
:105A5000044B5BF0C3BFA1F196040123A3404B4C60
:105A60002342F4D05DF8044B7047A1F148031A2B90
:105A7000EDD801A454F823F0655A01084F5A0108E3
:105A80004F5A01084F5A01084F5A0108655A010838
:105A90004F5A01084F5A01084F5A01084F5A01083E
:105AA0004F5A01084F5A01084F5A01084F5A01082E
:105AB0005F5B01085F5B01085F5B0108655A0108D5
:105AC0004F5A01085F5B0108655A01084F5A0108E7
:105AD0004F5A0108655A0108655A01084F5A0108D2
:105AE000655A0108A1F12703112BB0D8112BAED8AC
:105AF00001A454F823F000BF655A01084F5A010869
:105B00004F5A01084F5A0108655A01084F5A0108B7
:105B10004F5A01084F5A01084F5A01084F5A0108BD
:105B20004F5A01084F5A0108655A0108655A010881
:105B30004F5A01084F5A0108655A0108655A010871
:105B4000B02904DC952986DC6B2980D18AE7B52948
:105B500088D0A1F1D003022B3FF679AF82E75DF840
:105B6000044B00235BF00CBF094B012283F8E424B3
:105B7000A3F58043D3F8380F00283FF473AF5DF8E6
:105B8000044B64215BF0FAB810004100A1008004CE
:105B9000108C002038B50B466B2B0446114600F3E1
:105BA000AA80472B14DC382B00F38E80262B5FDC79
:105BB000102B00F0CD80162B00F02281042B00F07A
:105BC000DE800A4620461946BDE838405BF068BCD6
:105BD000A3F14802232AF4D801A050F822F000BF14
:105BE000595D0108C35B0108C35B0108C35B010881
:105BF000C35B0108835D0108C35B0108C35B010847
:105C0000C35B0108C35B0108C35B0108C35B0108F8
:105C1000C35B0108C35B0108975D0108D75D0108FC
:105C20008F5D0108F95D0108C35B0108DF5D0108B4
:105C3000895D0108C35B0108C35B01083F5D010882
:105C40000D5E0108C35B0108675D0108C35B0108C5
:105C5000C35B0108C35B0108C35B0108C35B0108A8
:105C6000C35B0108C35B0108C35B0108335E010825
:105C7000A3F12702112AA4D801A050F822F000BFF6
:105C80003F5D0108C35B0108C35B0108C35B0108FA
:105C9000435D0108C35B0108C35B0108C35B0108E6
:105CA000C35B0108C35B0108C35B0108C35B010858
:105CB000795D0108615D0108C35B0108C35B0108F0
:105CC000735D01086D5D0108402B7FF47AAF931E70
:105CD0005942684C594184F8E31459F015FB664A5F
:105CE00094F8E314654B002908BF1346644A062163
:105CF00052F032FC23E09D2B00F08F800BDC962BC2
:105D000000F089809B2B7FF45CAF022A17D15D489D
:105D100006F09EFD13E0B52B00F09B800ADCAD2B56
:105D20007FF44FAF022A0AD19FED570A5548FCF77E
:105D300007FA04E0A3F1D002022A3FF642AF0124A1
:105D400054E08A1E514B5142514183F8B911F6E794
:105D50000A21FFF707FEF2E70A4601212046F8E78D
:105D60000A460421FAE70A460321F7E70A460C210E
:105D7000F4E70A460F21F1E70A460021EEE70B217E
:105D8000E7E70A460D21E9E70A460521E6E720464E
:105D9000FFF732FED3E7374CD1B102290DD10123F1
:105DA00084F8E034A4F58053D3F8AC0103685B6A4F
:105DB000984710B1334800F085FD59F0A5FA344AF0
:105DC00094F8E014334B002908BF1346324A8EE79B
:105DD00084F8E014E6E72046FFF7E2FDAFE7012490
:105DE00031B1022902D12D4B83F89C42204638BDA7
:105DF0002A4B83F89C12F9E72046FFF709FE9EE73D
:105E0000022A9CD11F4806F0B9FB98E75AF070FFB0
:105E10005AF0F8FE93E707219BE701242AB1022AF2
:105E2000E4D1144B83F8E244E0E7124B83F8E22418
:105E3000DCE7022918D1154DD5F8AC010368DB6BFE
:105E40009847044648B10121A5F5A04002F0D8FCCE
:105E5000CCE7134880F074FB71E759F055FA114A0A
:105E6000042152F079FB6AE70648002102F0C8FCE1
:105E700065E700BF108C0020D0DD0C0873C50C084E
:105E8000D8DD0C08102C002000000000107C002041
:105E9000CFB00C08A8EA0C08E8DD0C08104C002074
:105EA000FC7C0020FBDD0C0810B5084CD4F8AC01DC
:105EB00003689B6B984730B9D4F8AC01B434001B2D
:105EC00018BF012010BD0220FCE700BF107C00209D
:105ED00008B5022103205CF0B7FD022108465CF002
:105EE000B3FD012104205CF0AFFD022115205CF020
:105EF000ABFD132002215CF0A7FD124807F00CF85F
:105F0000A8B1002146205CF09FFD002149205CF0F3
:105F10009BFD00214A205CF097FD002101205CF0F0
:105F200093FD0021BDE8084008465CF08DBD0121CD
:105F300046205CF089FD012149205CF085FD0121AE
:105F4000E8E700BF102C002002490348052208F0B2
:105F5000B1BB00BF887C0020102C002038B5304B2E
:105F600001241C7090F90A302B2B0CD12D487EF0A7
:105F700057FA2D4808F024F9BDE838402B48012293
:105F80000921FBF7FFBC284D9FED290AD5ED460AF4
:105F9000642103205CF022FBD5ED460A9FED240A24
:105FA000642102205CF01AFB9FED220A03205CF0C2
:105FB0001FFA9FED200A02205CF01AFA9FED1E0ADC
:105FC00004205CF015FA9FED1C0A15205CF010FA15
:105FD00013209FED190A5CF00BFA284606F09CFF8F
:105FE000A0B1002146205CF05DFD002149205CF05D
:105FF00059FD00214A205CF055FD002101205CF094
:1060000051FD002108465CF04DFDB2E721464620D7
:106010005CF048FD214649205CF044FD2146E9E75B
:1060200034960020188E0020102C00204C90002068
:10603000000000000000C84200A08C4500F5A04010
:10604000D0F8AC0103681B6C1847000000F514532E
:1060500093ED067A00F5C040B5EEC07AF1EE10FA85
:1060600003F118035DBFD0F81C33DFED086AD3EDF0
:10607000017AD0F834035FBFF8EEE77AE7EE267ACC
:10608000FDEEE77A17EE900A704700BF0000C842A5
:1060900000F5005090F8580528B141F00101084280
:1060A00014BF01200020704713B50346FFF7F0FF2F
:1060B00058B103F5005191F8580FC00705D501F606
:1060C000747191ED000A02B010BD03F5C04412B91D
:1060D00094EDDB0AF7E794F80422022AF8D103F5DD
:1060E000B240012201A96C304CF066FA0028EFD0D2
:1060F0009DED010AE7E7000000F5C04393F858233F
:10610000FFF7D2BF10B54B68516800F5C0448B4211
:10611000D8BF0A46D4F85003CCBF1A46194623F01C
:1061200067FCC4F8500310BD10B504464E4867F034
:10613000A1FA10F0080217BF4C4BDFED4D7A93ED3A
:10614000CB7AD3EDCD7A1FBF77EE877A9FED497A70
:10615000012267EE877A10F0010317BF434B9FEDD2
:10616000447AD3EDCD6A93EDCA7A1CBF37EE667AD6
:10617000DFED406A04F5145118BF27EE267AD1ED01
:10618000086AF5EEC06A18BF0123F1EE10FA34DD9B
:10619000394A9FED386AD2ED006A66EE866A0122BE
:1061A000F4EE676AF1EE10FA58BFF0EE667A04F585
:1061B000C04090F8581329B373B1D0EDD76AF8EE08
:1061C000E66AF4EEC76AF1EE10FA58BFF0EE476ADD
:1061D000FDEEE66AC0EDD76A9AB190EDD77AB8EED7
:1061E000C77AB4EEE77AF1EE10FAD8BFB0EE677A6C
:1061F000BDEEC77A80EDD77A03E0002AD7D1002B15
:10620000D5D110BDB3B1D0F81C33D3ED016AF8EE8F
:10621000E66A76EE876A90EDD47AB8EEC77AF4EE45
:10622000C76AF1EE10FAD8BFB0EE667ABDEEC77A53
:1062300080EDD47A002AE4D0D0F81C3393ED017AB3
:10624000B8EEC77A77EE277A90EDD47AB8EEC77AAF
:10625000F4EEC77AF1EE10FA58BFB0EE677ABDEEF1
:10626000C77A80EDD47ACCE7304F0020104C002064
:10627000000000000000C8423051002000F5C0407E
:106280000023C0F85433704773B516460446002304
:106290006A463046009311F029FB48B1DDED007AE3
:1062A0009FED277A67EE877AFDEEE77A17EE900A80
:1062B00004F5C045C5F8540333785B0718D595F845
:1062C0005833ABB104F5B240012201A96C304CF057
:1062D00073F968B1D5EDD77ADDED016A9FED187AD3
:1062E000F8EEE77AE6EEC77AFDEEE77AC5EDD57A05
:1062F00004F5A043D3F83038042B1FD004F5005424
:10630000B4F95225002A16DDD5F854339FED0D7AE5
:1063100083EAE371A1EBE37107EE901AF8EEE77AF6
:1063200067EE877A07EE102AB8EEC77AF4EEC77ADE
:10633000F1EE10FA02D50023C5F8543302B070BD57
:106340000000C8420AD7233C37B50B785A070446E9
:106350000D461DD500F5B240012201A96C304CF06C
:106360002BF9A8B1D5ED017A2B78DFED1B6AF8EE99
:10637000E77ADB0767EEA67A19D59DED017AB4EED0
:10638000E77AF1EE10FACCBF0120002003B030BD57
:106390002B78D5ED017A13F0010FF8EEE77A04F5CA
:1063A000C0440FD194EDCD7AB8EEC77AE7E704F593
:1063B000C044D4F81C3393ED017AB8EEC77AE7EE07
:1063C000667ADAE7D4F81C3393ED017AB8EEC77A2F
:1063D00077EE877AE6E700BF0AD7233C00F5005343
:1063E000B3F9023500EE103A00F5A0431A46D3F88F
:1063F000AC1178329142B8EEC00A0CD1D3F83028F3
:10640000042A02D093F8DD372BB100F5C040D0ED5F
:10641000827A30EE270A704710B5044604F5C0446E
:10642000FFF7DCFFD4EDCD7A9FED057AF8EEE77A41
:10643000E0EE477AFDEEE77A17EE900A10BD00BF56
:106440000000C84237B500F5C045044695F85833FA
:10645000DBB100F5B240012201A96C304CF0ACF880
:1064600098B1D5EDD77AD5EDD86A9FED0B7AF8EED5
:10647000E77AE6EE877ADDED016AE6EEC77AFDEEB1
:10648000E77A17EE900A03B030BD2046FFF7C4FF4D
:10649000D5F85033181AF6E70000C84210B5044684
:1064A00004F5C044FFF79AFFD4EDDB7A37EEC00A5B
:1064B000DFED047A20EE270AFDEEC07A17EE900A8F
:1064C00010BD00BF0000C8422DE9F04100F5C647ED
:1064D00000F5C6453037403504462946384611F0A8
:1064E00079FC04F5A04804F5C64608F2C4732036CA
:1064F0002A46314683ED000A384611F0A1FB08F523
:10650000F963DFED220A83ED000AB7EE001A762068
:1065100023F0CEF904F53F5383ED790A2046FBF7CB
:10652000B7FDD8F8AC0103685B6898470B280DD01D
:1065300008D80A2811D004F5C0440023C4F8543305
:10654000BDE8F0810E38C0B20128F4D829462046B3
:10655000FFF7FAFE0028EED011E029462046FFF7AB
:10656000F3FE30B90A484FF48041FBF7FFFF0028E3
:10657000E1D12046FFF792FFB0F5FA6FE6DD2A463B
:1065800031462046BDE8F041FFF77EBE0000000026
:10659000102C002010B52DED028B00F5C043D3ED7B
:1065A000D17A93F84033DFED1C8ADA0758BF00F543
:1065B000B452B8EEE78A58BFD2ED007A28EE288AA6
:1065C00058BFF8EEE77A82B058BFA7EEE88A5B07BB
:1065D00004460FD500F5B240012201A96C304BF002
:1065E000EBFF38B19DED010A30EE480A02B0BDEC78
:1065F000028B10BD2046FFF70FFF04F5B45393ED57
:10660000000A07EE900AB8EEC00AF8EEE77A28EE24
:10661000C00AA7EEA80AE7E70AD7233C70B52DED1C
:10662000028B00F5A0463346D6F8AC2154339A428B
:1066300004464DD100F58053D3F8105600F50053B1
:10664000B3F95035002B66DD04F5C05292ED057AA2
:10665000F7EE007AB4EEE77AF1EE10FA5BD404F5C7
:106660004052D2ED027AF6EE006A67EEA67A87EE25
:10667000871AB5EEC01AF1EE10FA4CD907EE905A0F
:106680009FED278AB8EEE70A07EE903A04F5B2408C
:1066900004F5C044F8EEE70A20EE080A6C304CF02E
:1066A00097F8D4F854339FED1F1ADFED1F0A002B23
:1066B000BCBF07EE903AF8EEE77A4FF42970B8BF06
:1066C000A7EE880ABDEC028BBDE8704023F0F0B85D
:1066D00005F0ECFDF8B904F5405306F2C476D3F8A2
:1066E000180903681B69984704F50053DFED0E0A8B
:1066F000B3F9503596ED000A01EE103A0546B8EEB2
:10670000C11A40F27F2023F0D3F8BDEEC00A10EE8C
:10671000103A1BB296E7BDEC028B9FED030A70BDE9
:106720000AD7233C00007A440000000010B504465C
:1067300081F0A4FE04F50053D3F86C2F801A41F2C7
:10674000883290420FD802212046FFF7A1FC50B1B9
:1067500004F5A044D4F83028042A04D103F5766364
:1067600093ED000A10BD9FED010AFBE70000000059
:1067700030B52DED028B00F5C045DFED278A95F889
:10678000583383B004465BB3D5EDD77A9FED230A27
:10679000F8EEE77A00F5B24027EE800A012201A95F
:1067A0006C304BF041FFD8B12046FFF737FFDDEDED
:1067B000017A85EDD80A37EE800A20468DED010A70
:1067C000FFF7B4FFDDED017A30EE270A20EE280A4C
:1067D000BDEEC00A10EE100A03B0BDEC028B30BD56
:1067E000D5F81C23D5F8503352689B1A08EE103A9E
:1067F0002046FFF7F3FDB8EEC88A2046A0EE288AAF
:10680000FFF794FFBDEEC88AB8EEC88AA0EE288ACA
:10681000BDEEC80ADEE700BF0000C8420AD7233C2D
:1068200010B500F5A0430446D3F8AC0103685B6AD9
:10683000984718B104F5C04494F8E00410BD000076
:1068400038B500F5C0440D46D4F850330B44C4F8B5
:10685000503394F858333BB1FFF7E2FF20B9D4F836
:106860005C132944C4F85C1338BD000030B500F552
:106870000050D0F84C25D3070FD4094B08201D78C1
:106880005C688D4204D1224214BF0120002030BD3B
:10689000013803F10803F2D1F9E70120F7E700BF5F
:1068A0004CE00C0810B500F5A0430446D3F8AC0149
:1068B00003685B68984701462046BDE81040FFF733
:1068C000D5BF000037B500F5C0440546D4F83433D1
:1068D000C4F850330023C4F85433FFF7E3FFD0B1BA
:1068E00005F5B240012201A96C304BF065FE90B174
:1068F0002846FFF795FF70B9DDED017A9FED087A24
:1069000067EE877A0123FDEEE77A84F85833C4ED09
:10691000D77A03B030BD002384F85833F9E700BFBD
:106920000000C84238B504460D46FFF7BBFF30B142
:106930000321284610F0B6FF80F00103D8B204F519
:10694000C04484F8590338BD73B500F5C0444A68A3
:10695000C4F850230B780D46D90741BFD4F81C3337
:106960005B689B18C4F8503394F85933064623B13A
:1069700000F5C6414031FFF7D5FF2B785B070FD5F7
:1069800006F5B240012201A96C304BF015FE38B17A
:10699000012384F858336B68C4F85C3302B070BDCF
:1069A000002384F85833F9E7F0B52DED028B044647
:1069B00083B004F5C0450E468DED010AFFF7C4FF14
:1069C000DFED350A9DED010A40F24310B7EE001AE3
:1069D00022F06EFFD5F854335B4207EE903AF8EEA2
:1069E000E77A04F5155767EE807A2046FDEEE77AE0
:1069F000B0EE408A17EE901AFFF722FFD7ED057A26
:106A0000F5EEC07AF1EE10FA07F114073FDDD5F884
:106A10005433002B3BDD2046FFF714FD07EE900AB0
:106A2000DFED1E6AB8EEE77AD7ED007A67EEA67A58
:106A3000B4EEE77AF1EE10FA29D531462046FFF799
:106A400083FF04F5C641324630312046FFF71CFC77
:106A5000D5F854335B4207EE903AF8EEE77A2046D9
:106A600067EE887AFDEEE77A17EE901AFFF7E8FEF8
:106A7000B5EEC08AF1EE10FA09DDD5EDD57AB8EEA3
:106A8000E77AC7EE087AFDEEE77AC5EDD57A03B06E
:106A9000BDEC028BF0BD00BF000000000000C8C2CA
:106AA000F0B500F5C04487B094F8403303F0050317
:106AB000052B07460BD04CF0FFFD4FF4AE724FF4A0
:106AC00080114CF0B1FD0025284607B0F0BD1E48EE
:106AD0006A46032110F0F6FE0028F4D01B4801AAF4
:106AE000032110F0EFFE05460028ECD0184BDFED37
:106AF000190A93ED000A40F26D10B7EE001A22F069
:106B0000D7FE04F550730FCBB0EE401A02AEDFEDA6
:106B1000111ADDED010A9DED000AB7EE002A86E8A4
:106B20000F0022F0F7FDDFED0C7A20EE270A304649
:106B3000FDEEC07A032217EE901A10F0EFFD3146F9
:106B40003846FFF701FFBFE7308F0020508F00204D
:106B5000D8830020000000000000C842F7B50E46B0
:106B600002210446FFF794FA70B304F5A045D5F866
:106B70003038042B28D12046FFF794FE20B304F5CB
:106B8000B2476C3704F5C64101236A4630313846B6
:106B90004BF0FCFBC0B104F5C641012301AA403112
:106BA00038464BF0F3FB78B19DED017ADDED007ACC
:106BB00077EEC77A96ED007A37EE277A05F5FD6510
:106BC00086ED007AC5ED007A03B0F0BDF0B52DED8D
:106BD000048B00F5005489B000F5736694F8221F09
:106BE00003910546304645F02BFC03990746304695
:106BF00045F038FC042F0399B0EE408A20D10023E1
:106C000005A88DED050A0693079325F021FA05F5F1
:106C1000B95005A9103023F027F9DFED9B7A8DEDEF
:106C2000050AB4EEE71AF1EE10FACDED060A8DED85
:106C3000071A05DB05F5805393F88C36DF070CD473
:106C400094F8583F002262F3000384F8702F84F810
:106C5000583F09B0BDEC048BF0BD94F8583F98073D
:106C60005CBF43F0020384F8583F04F6747758BFC2
:106C700004F65C7305F53D5158BF83ED008A34314D
:106C800087ED001A2846FFF769FF94F8703F092B3B
:106C900000F2898004F67873D3ED000A9FED7B9AA9
:106CA000B0EE480A22F0F2FC00BB04F65C7394F8E4
:106CB000221FD3ED008A304645F0F2FB07EE900A22
:106CC0009FED737AF8EEE77A78EEC88A67EE877AF6
:106CD000F0EEE88A67EE897AF4EEE78AF1EE10FAD0
:106CE000C2BF94F8703F013384F8703F04F67873A4
:106CF00094F8221FD3ED008A304645F0D1FB07EE11
:106D0000900AF8EEE77A9FED637A67EE897A78EE7B
:106D1000C88A67EE877AF0EEE88AF4EEE78AF1EE49
:106D200010FA02DD002384F8703F04F6787383EDD7
:106D3000008A94F8583FDA078BD5284605F5C046F7
:106D4000FFF728FC04F6747393ED008A96F8583325
:106D500030EE488A002B4CD005F5B240012205A93F
:106D60006C304BF029FC002849D181F087FBD4F826
:106D70006C2F41F28831821A8A42034604F576620A
:106D800004F6647144D982ED008A284681ED008AB8
:106D90000221FFF77DF918B1D6F81422C6F81022A7
:106DA000C4F86C3F55E794F8583F43F00103590786
:106DB00084F8583FB9D405F5A042D2F83028042A07
:106DC000B3D102212846FFF763F90028ADD043F084
:106DD000040384F8583F3868F9F796FB05F55B56CD
:106DE0003036CDE900012C4A0621304651F0B4FB83
:106DF0009BE72846FFF756FD0028ADD1B5E704F61E
:106E0000747393ED000A9DED058A38EE408AACE775
:106E10009FED200A92ED007ADFED207A28EE008ABD
:106E2000A7EE278A82ED008AC4F86C0FD1ED007AB4
:106E300038EE678AF3EE0E7AB0EEC88AB4EEE78ACF
:106E4000F1EE10FA7FF705AF94F8583F5B070ED5C7
:106E500004F6747405F55B562068F9F755FB303677
:106E6000CDE900010E4A0621304651F075FB05F5CB
:106E70003D5024220021183009B0BDEC048BBDE840
:106E8000F040ADF069B800BF000000340AD7233CE1
:106E9000CDCC4C3DCDCC4C3E0CE00C08CDCC4C3F89
:106EA00029E00C0838B52DED028B0D460446FFF79E
:106EB00071FB002320462B70B0EE408AFFF736FCB2
:106EC0000221204638EE400AFFF7E2F828B104F527
:106ED000005494F8580F00F00100BDEC028B2870AC
:106EE00038BD000070B50B7803F00503042B054690
:106EF0000C46164615D105F5C0454CF0DDFBB2B287
:106F00004FF480114CF090FBD5F81C236368526855
:106F10009B1A13F5FA7FC8BF6360237843F001031F
:106F2000237070BDF8B500F5805300F5A047D3F885
:106F30008066D7F8EC57B542044619D00E4A12685D
:106F4000D26A92F89C209AB100F5C641751B2522A1
:106F50004031FFF7C7FF07EE905AB8EEE70ADFEDC2
:106F6000077A04F53F5020EE270A20307CF0EAFD36
:106F7000C7F8EC67F8BD00BF0C2C00200AD7233CF3
:106F8000F8B500F5A04C00F5C0449CF8DFE70546D5
:106F90000F4604F54876BEF1000F53D004F5507348
:106FA0000FCB86E80F0001238CF8E03797E80F003D
:106FB00004F5507686E80F00D4F8483305F5C64648
:106FC000403693B9D4F84C337BB9D4F83833D4F87D
:106FD0004423C4F84833D4F83C33C4F84C3322B9C2
:106FE000D4F83413304610F099FB31462822284655
:106FF000FFF778FF94F8401311F0040102D13046F6
:1070000010F050FC05F5C64105F5C640324620316A
:10701000303010F04BFE38B104F5487604F54C746E
:1070200094E80F0086E80F00284604F093FD2846F8
:10703000FFF74AFA284605F0FDF82846BDE8F84073
:10704000FEF7FCBF04F54C730FCB86E80F0001235D
:107050008CF8DF378CF8E0E7A8E70000F8B500F51A
:1070600000530446B3F9AA34002B0D4635DB0B78E8
:1070700013F0020F14BF4FF0FF33012304F5C04695
:1070800006F5487786F8F83206F54C730FCB87E89B
:107090000F0095E80F0006F5507787E80F0004F51C
:1070A000C641572240312046FFF71CFF2046FFF71C
:1070B00009FC2046FFF708FA204605F0BBF804F566
:1070C000A042002382F8E037C6F8FC3282F8E537A8
:1070D0002046BDE8F84004F03DBD4FF0FF33CDE75A
:1070E0002DE9F043364B1B6885B00546D86AFAF7A0
:1070F0001BFA002861D105F5005393F9D03E5A1CC4
:1071000054D0002B05F58C6711DD95F871242421EE
:1071100007EE903A01FB027292ED0B7AF8EEE77AF5
:10712000B0EEC77AB4EEE77AF1EE10FA3EDC05F580
:10713000805305F5A05693F88C3613F0010406F140
:10714000100629D0C3F340089B0732D495F81414D5
:1071500095F858444FF0B00909FB015191F8F1310D
:107160004CBB022B18D9684610F0D2FA694630465B
:107170000AF078FE044678B195F8143409FB0353FD
:107180004246D3F80012684610F0C8FA0BF02CF90A
:1071900069460AF055FD044638460DF0EDFB3046D1
:1071A0000AF06CFC2846FBF7B3F9204605B0BDE8B1
:1071B000F0830024F0E74446EEE70020F6E700BF46
:1071C0000C2C002038B50C4B1B680546D86A0C46C1
:1071D000FAF7AAF910B10024204638BD0BF004F9E3
:1071E00021460AF02DFD04460028F4D005F5B040F4
:1071F000543025F01BFDEFE70C2C0020F0B500F516
:10720000A04300F5C046002283F8DF2783F8E0277B
:1072100006F54C73044600EE101A0FCB87B006F546
:10722000487585E80F0002AD04F5C642B8EEC00A05
:1072300028461749303244F0C1FE95E80F0006F5A4
:10724000507787E80F0004F5C64140F257124031ED
:1072500020460191FFF746FE01992046FFF762FBA9
:1072600001992046FFF770FB04F500532046B3F95F
:10727000AA34002BB4BF4FF0FF33012386F8F83255
:10728000FFF722F9204607B0BDE8F04004F0D2BF76
:10729000EC65002010B50349044644F08FFE2046FB
:1072A00010BD00BFEC650020F8B500F5C04505F540
:1072B0004C7304460E460FCB05F5487787E80F0060
:1072C00006F108012046FFF75BFEB28802EB82025E
:1072D00002EB8202920012B204F5A043002AD8BF4A
:1072E0004FF4C872A3F8DA27D5F81C23D5F8441355
:1072F0005068091AC3F8AC1791680A31C5F84813E9
:10730000D2680A32C5F84C230022C3F8C02783F89C
:10731000DC2783F8F027C3F8B02703F2A47200211A
:1073200011604FF0FF32C3F89C2794F8711404F5F4
:107330008C62242000FB012203F2D473D26A1A600B
:10734000F8BD000070B50E4608310446FFF718FE80
:10735000B38804F5A04543B3642213FB02F3C5F8D8
:10736000AC37B5F9DA37002BD8BF4FF47A7304F590
:107370003D50D8BFA5F8DA37242200211830ACF0F0
:10738000EBFD04F5C04304F5C44093EDDB0A314640
:1073900008307CF045FFD5F83038072B0CD120465B
:1073A0000421BDE87040FAF723BED5F8AC37002BB6
:1073B000D7DC40F6B833D2E770BD00000B7A00F599
:1073C000C04013F0020F14BF4FF0FF33012380F8C9
:1073D000F83270477FB501F1080305460E460FCB22
:1073E0006C4684E80F0005F5C6413031204610F0A8
:1073F000F9FA21462846FFF7C3FD31462846FFF734
:10740000DDFF04B070BD00007FB501F10803044644
:107410000E460FCB6D4685E80F0004F5C6413031AE
:10742000284610F0DFFA29462046FFF7A9FD20463E
:107430003146FFF7C3FF337907EE903A337E9B075F
:1074400048BF9FED0B7AF8EE677A04F5C04448BF59
:1074500067EE877A9FED077A67EE877A0123FCEE65
:10746000E77AC4F81033C4EDBC7A04B070BD00BF35
:107470000000803B00A00C477FB501F108030446E3
:107480000E460FCB6D4685E80F0004F5C64130313E
:10749000284610F0A7FA29462046FFF771FD20463E
:1074A0003146FFF78BFFB38804F5C0444FF47A727E
:1074B0005343C4F808330123C4F8103304B070BD3B
:1074C0002DE9F34100F5C6450446403500F5C640B8
:1074D0000E462030294610F045FA04F5A047D0B9F1
:1074E0004FF0FF33C7F89C3706F10807384610F015
:1074F0003FF9032802463CD1F168284610F00EF906
:10750000B28804F5C0432046C3F8102302B0BDE89A
:10751000F041FEF7B3BE19F0E9FFFAF7FBFA0128D4
:1075200012D94FF0FF33C7F89C3719F0DFFF90F8FE
:10753000F432DFED150AB02202FB030090ED3C0AA5
:10754000284610F0BDFCCFE704F58058D8F81006A7
:1075500022F082F908F5C263C7F89C07D3ED007AE0
:107560009FED0A0ADFED080AF8EEE77A27EE800AB7
:10757000E6E701AA0021384610F006F90028BFD03E
:1075800001990022B9E700BF00007A440AD7233CE2
:107590007FB501F1080304460E460FCB6D4685E822
:1075A0000F0004F5C6413031284610F01BFA294679
:1075B0002046FFF7E5FC20463146FFF7FFFE04F5C5
:1075C000C0440023C4F8103304B070BD37B504467E
:1075D0000D4680F053FFE060D5ED027AF5EEC07AFB
:1075E000F1EE10FA15DD9FED127A67EE877AFCEE68
:1075F000E77AC4ED027A57F087FEA2684FF47A73F7
:10760000B2FBF3F30B4A062103B0BDE8304050F063
:10761000A3BF65F07DFE0023009395F90D2095F939
:107620000E3095F90C1065F00FFEA060E3E700BF87
:1076300000007A448CE00C082DE9F0432DED028B1C
:1076400085B004460AF0D0FE09F0FEFF04F5805331
:1076500004F5A04693F808390BB9002877D0D6F87E
:107660009C37013373D1D6F8C037002B4BD080F054
:1076700005FFD6F8C037C01AB0F5FA6F67D394F893
:107680001424DFED607A9FED608A4FF0B00808FBAC
:10769000024292ED840A20EE270A22F0F5F806F263
:1076A000A479D9ED007A30EE670A22F0EDF8DFED2B
:1076B000577A20EE080A04F55B5720EE270A22F0DD
:1076C0008BF8FDEEC07A303717EE905AC6F89C570B
:1076D000D9ED007A67EE887A17EE900AF8F714FF72
:1076E000CDE9020194F8143408FB0343D3F80C02EB
:1076F000F8F70AFF464ACDE900012B460621384635
:1077000050F02AFF23E004F59070FAF703FA0228FC
:107710001DD994F81434B02202FB034393ED837A0D
:10772000F1EE047AB4EEE77AF1EE10FA0FDD394BA0
:107730001B68D86A0368DB699847012803D080F08A
:107740009DFEC6F8C007D6F8C037002B8FD104F5D0
:107750004053D6F89C17D3F818094A1C036848D040
:107760001B6B98472C4807F0C5FD20B104F5B040CD
:10777000543027F0DDFC2046FEF790FED6F8AC37FB
:107780008342054638DA07EE905A9FED247AF8EEE8
:10779000E77A04F55B5767EE877A303717EE900A81
:1077A000F8F7B2FE1E4ACDE900013846062150F036
:1077B000D3FE04F5C0444FF0FF330125C6F89C37D3
:1077C00086F8DC5704F54C730FCB04F5487704F5C5
:1077D000507487E80F0084E80F00124865F014FF2A
:1077E000002386F8DF37284605B0BDEC028BBDE8E4
:1077F000F0835B6B9847B5E7074807F05BFD00280F
:10780000C1D1F1E735FA8E3CE02E65420000C84256
:107810009CE00C080C2C0020102C00200AD7233CE4
:10782000C0E00C08304F00202DE9F04F00F5A049D2
:107830002DED028B4FF0FF3300F5C04AC9F89C379D
:107840000AF550730F4606460FCBBC8897F80480A4
:1078500089B004AD240A85E80F001FD006F5C6479D
:1078600020372946384610F0B5FA29463846B0EE9A
:10787000408A10F07FF9DFED577AB4EEE78AF1EE37
:1078800010FA0BDBE3B200EE903ADFED537AF8EE3C
:10789000600A20EE270A284610F012FB06F5405B2E
:1078A00099F8E027DBF818099FED4C0A036806F504
:1078B000C6479B6A303732B306F5C6412A462031A7
:1078C000984706F50051B1F9DA34002B1EDD07EEBA
:1078D000903A09F2C472F8EEE77A92ED007AB4EECB
:1078E000E77AF1EE10FA11DD06F5C6412A4620319D
:1078F000384610F0DBF900BB0024204609B0BDEC8F
:10790000028BBDE8F08F2A463946D9E7B8F1000F5F
:107910001DD1002C3DD1B1F9D824DBF8180900EEB7
:10792000102A026809F5F763126AD3ED000AB8EE6F
:10793000C00A9047B0EE408A0DE0002CDCD10AF579
:107940004C730FCB0AF5487585E80F00D5E707EEB5
:10795000908AB8EE678A2946384610F03BFAB4EEB2
:10796000C08AF1EE10FA17DBB9F890380393294674
:10797000384610F02FFABCEEC00A06F55B50039BA8
:10798000174A8DED000A0621303050F0E5FD012444
:10799000B3E79FED128ADEE706F5C6412A4620319D
:1079A000384610F083F904460028A5D0B9F890387D
:1079B00003932946384610F00DFABCEEC00A06F5CE
:1079C0005B50039B074A8DED000A0621303050F0D2
:1079D000C3FD92E700000034E02E65420000000085
:1079E000DCE00C08FAE00C0838B500F5005500F5AD
:1079F000C043B5F9DC140029ACBF01224FF0FF32BF
:107A00000029B8BF4942044683F8F82289B204F03D
:107A100033FD04F5AF4393ED117AB5F9D834002B5B
:107A2000CABF07EE903ADFED0E7AF8EEE77AFCEE89
:107A3000E77AF8EE677AB4EEE77AF1EE10FA08D852
:107A400004F55B503030074A062150F085FD0120D7
:107A500038BD204604F02AFC0028F1D1F8E700BF29
:107A60000000000018E10C08F8B500F5C64600F566
:107A7000C645203640350446294630460FF072FF91
:107A800004F5405750B304F5A043D3F89C174B1CA2
:107A900024D0D7F8180903681B6B984704F5C04534
:107AA000D5F81033012B47D0D5F81033022B06D16F
:107AB0002046FEF7B1FCD5F84433984243DD20461A
:107AC000FEF7AAFCD5F84433C01A0028B8BF4042DC
:107AD000B0F5FA7FCCBF0020012035E004F5C640A8
:107AE0002946303010F076F9DFED187AB4EEE70A67
:107AF000F1EE10FA16D53046294610F03BF89FED0E
:107B0000147ADFED140AF6EE007AE0EE077A2846E2
:107B10009FED110AFDEEE77AF8EEE77A27EE800A8C
:107B200010F0CEF9D7F818099FED0C0A03682A4621
:107B30009B6A31469847B1E72046FEF76DFCD5F8C1
:107B400044339842B0DB0120F8BD00BF0000484339
:107B5000A00CB345000096430AD7233C0000000068
:107B600073B5374CD1ED026AD4EDCD7A9FED357AFD
:107B7000F8EEE77A0546D7EE876A0E46F5EEC06A5C
:107B8000F1EE10FA08DD57F0BFFB2F4A062150F046
:107B9000E3FC012002B070BDD1ED037AF5EEC07AAE
:107BA000A4F64404F1EE10FA94ED006A12DDF4EE4E
:107BB000C67AF1EE10FA0DD557F0A6FB05462068FF
:107BC000F8F7A2FC214ACDE900010621284650F031
:107BD000C3FCDEE7DFED1E7A337CB4EEE76AF1EE3C
:107BE00010FA54BFB0EE677AB0EE467A0BB90020B7
:107BF000D0E7B5EEC06AF1EE10FA0CDC86EE876ACB
:107C000003EB830307EE903AF8EEE77AF4EEC67AD8
:107C1000F1EE10FAEBD52C7C002CE8D180F02EFC94
:107C20006B69C01A337C4FF47A7253439842DED9A1
:107C300001232B7480F022FC68612046AAE700BF74
:107C4000108C00200AD7233C30E10C0841E10C08DD
:107C50000AD723BC38B5054677F0A6FF76F038FD85
:107C6000044640B980F00AFCEB68C01AAB68984241
:107C700084BFAC600124204638BD000038B50446FE
:107C80000D4680F0FBFB04F5C0439FED067AC3F878
:107C90001403D5ED027A67EE877AFDEEE77AC3ED3D
:107CA000C47A38BD00007A4410B5044680F0E6FB83
:107CB00004F5C043D3F81423801AD3F8102390425C
:107CC0004FF0000084BFC3F81003012010BD000076
:107CD00000F5C04300F5AF41D3F8102391ED117AC0
:107CE00022EAE27207EE902AF8EEE77A0020B4EE7C
:107CF000E77AF1EE10FA44BFC3F810030120704791
:107D000010B500F5005300F5C040B3F9AA34002BBC
:107D1000B4BF4FF0FF33012380F8F83200F5507400
:107D200000F54C700FC884E80F0010BD38B504464C
:107D30002DED028BF0EE408AB0EE608A09B3012986
:107D40005CD0B5EEC08AF1EE10FA67DDDFED347A73
:107D5000B4EEE78AF1EE10FA60D8FCEEC87A04F5CA
:107D60005B5017EE903A2F4A0621303050F0F4FB6A
:107D7000FDEEC87A04F5005417EE903A84F8773493
:107D80003AE0F8EE000A21F081FC40B104F5A0448D
:107D90004FF0FF33C4F8DC31BDEC028B38BD04F585
:107DA0000053B3F9802407EE902AF8EEE77AF4EE58
:107DB000E87AF1EE10FAC4D8B3F9823407EE903ABB
:107DC000F8EEE77AF4EEE87AF1EE10FAB9DBDFEDDF
:107DD000147A154A68EEA77A04F5A043FDEEE77A17
:107DE00004F55B50C3ED777AFCEEE87A062117EED6
:107DF000903A303050F0B0FB0120CDE7FCEEC07A75
:107E000000F55B5017EE903A084A0621303004F531
:107E1000125450F0A1FBC4ED038AEDE70020BBE74C
:107E20000000C84287E10C0860E10C0874E10C080E
:107E3000D1F80D3000EE903AD1F80930097A00EE11
:107E4000103AFFF773BF000070B58B88012B044612
:107E50000D4611D100F590763046F9F75BFE022809
:107E60000AD994F81414B02303FB01612046DC31D5
:107E7000BDE87040FFF7A6B90AF0B6FA05F10801AF
:107E8000BDE8704009F0DCBEF0B500F5A046002763
:107E9000A24B86F8E57789B0044608460D4683F87C
:107EA000597324F0D5FC50B3012386F8DC3704F570
:107EB0004053D3F818090368DB6B984704F5C043B7
:107EC00086F8E37703A8C3F8FC720FF021FCB6F83C
:107ED00090184FF6FF73994208BF3946013104F5F7
:107EE000B04001AA89B2543026F0A4FC28B1BDF8F4
:107EF0000600A0F115035842584186F8DD076B884B
:107F00005D2B00F0038132D81F2B29D80F2B01D80D
:107F100000202AE0103B0F2BFAD801A252F823F0E0
:107F20001380010829800108338001083D80010881
:107F3000518001081F80010801800108117F01089C
:107F4000117F0108117F0108117F0108117F0108CD
:107F5000117F0108117F0108618001084780010835
:107F6000532BD5D1012086F8E30709B0F0BDBD2B16
:107F700018D8BB2B4BD8B22B7CD00CD8702B74D01C
:107F8000722BC5D1D5ED027AFDEEE77A04F5C04437
:107F9000C4EDC47A3BE0B32BBAD129462046FFF7A3
:107FA00053FF34E0C33B9AB2112AB1D8112BAFD89A
:107FB00001A252F823F000BFAF800108117F010831
:107FC000AF800108117F0108117F0108117F0108AE
:107FD000AF800108117F0108117F0108117F01089E
:107FE000EB800108117F0108117F0108117F010852
:107FF000117F01087F800108117F01089F8001081F
:10800000002386F8193829462046FFF74DF901204C
:10801000ABE705F108012046FEF7B2FFF7E7294676
:108020002046FFF78FF9F2E729462046FFF7D2F9FD
:10803000EDE729462046FFF7E7F9E8E7294620461D
:10804000FFF71AFAE3E729462046FFF7A1FADEE731
:1080500004F5A14129221031204606F02BFBD6E77A
:1080600029462046FFF72CFAD1E729462046FFF79C
:1080700005FECCE729462046FFF7DAFEC7E7AB88C6
:10808000012BC4D803F0010386F8DE3704F55B50FA
:10809000AB88234A0621303050F05EFAB7E7A98852
:1080A000003918BF0121204600F0AAFBAFE704F514
:1080B000C746EB6804F5C044383694F8311473B9F8
:1080C0002B6963B96B6953B930465CF005F8042835
:1080D0009DD194F8311430465CF008F897E705F12B
:1080E000080230465CF040F991E704F5C04304F51E
:1080F000C74095ED041AD5ED020A95ED030A93F8F1
:108100003114002238305CF013F880E704F5A04009
:1081100029467830FFF75AFA79E700BF108C002023
:1081200098E10C0800F5A0421346D2F8AC21783350
:108130009A4201D1FFF7A8BE0120704710B500F5A3
:10814000A0421346D2F8AC2178339A4204460ED1AD
:1081500000F5A1410822103106F0ACFA04F55B509D
:10816000034ABDE810400621303050F0F5B910BD8B
:10817000A8E10C0870B58EB009AD044628460E463D
:108180000FF0C6FA04F5A0434FF6FF72B3F890382B
:10819000934208BF0023013304F5B04007AA99B207
:1081A000543026F047FBB0B104F5C04416B10023AB
:1081B000C4F8F43295E80F0001AE86E80F00D4F859
:1081C0004C33009304F5507494E80E00034802F019
:1081D000ADFD0EB070BD0120FBE700BFA87C002004
:1081E00070B5054605F5C046002104F045F9D6F8FE
:1081F000FC427CB9284604F059F810B90024204606
:1082000070BDD6F8F432012BF8DD80F037F9C6F8EE
:10821000FC02F4E7D6F8101361B180F02FF9D6F81C
:10822000FC32C01AD6F808339842E7D90023C6F8C2
:10823000103301212846FFF79DFF04460028DDD0BA
:1082400005F55B50054A0621303005F5A04550F094
:1082500083F9002385F8E537D1E700BFD0E10C08AA
:1082600038B50A468B88190A137EDB0748BF01EB35
:108270008101044648BF490004F0FEF804F5A0431C
:10828000002583F8E557204604F010F810B90025C2
:10829000284638BD04F5C043D3F8101341B1D3E9E3
:1082A000BC128A42F3DD012AF1DDC3F8105301212B
:1082B0002046FFF75FFF05460028E8D004F55B5035
:1082C000024A0621303050F047F9E1E7E8E10C08B6
:1082D00038B5054605F5C044898804F0CDF8D4F8D2
:1082E000103383BBD4F8F432002BB8BF5B42012BB0
:1082F00002DC0024204638BD94F8F92294F8FA32C2
:1083000072B9002BF5D005F55B50D4F83423642303
:10831000062192FBF3F330300C4A50F01DF901E0D6
:10832000002BF0D10121C4F810132846FFF722FFDB
:1083300004460028DDD005F55B50054A06213030A3
:1083400050F00AF9D6E70021EFE700BF00E20C0881
:108350001EE20C082DE9F0474B881F2B8AB004461B
:108360000A4631D80F2B07D804F55B50984A0421F0
:10837000303050F0F1F888E0A3F110010F29F3D864
:1083800001A050F821F000BF9B8401086985010815
:1083900075850108838501089D850108A984010868
:1083A0008F840108698301086983010869830108D2
:1083B00069830108698301086983010869830108E9
:1083C000A98501088F850108702B00F0FB800CD86F
:1083D000532B00F0EF805D2BC6D100F5A040783024
:1083E0000AB0BDE8F047FFF735BCB32B08D8B12B76
:1083F0004BD8722BB8D10AB0BDE8F047FFF768BC84
:10840000D42B3BD8BB2BAFD9A3F1BC02182AABD8D5
:1084100001A151F822F000BF8B8401088B84010870
:108420006983010869830108698301086983010878
:10843000698301088B840108698301088B84010822
:108440006983010869830108698301088B84010835
:108450006983010869830108698301088B84010825
:108460008B8401088B8401086983010869830108F2
:108470008B840108698301088B840108DF2B04D0F9
:1084800040F6B83293427FF46FAF01202FE02046D0
:108490000AB0BDE8F047FFF7CFB8114620460AB052
:1084A000BDE8F047FFF7C0B904F5A04504F5C446A0
:1084B000D5F8303804F5C64704F5C64804F5C64972
:1084C000072B06F1080607F1200708F1400809F11B
:1084D00030090FD104F5B04428340194D5F8AC37F5
:1084E000009342464B46394630467BF05DFF0AB06A
:1084F000BDE8F0870DF12701002336488DF82730BD
:10850000FEF7D0FC05F5FD63D3ED007AD5F8CCA7D6
:1085100005F2BC73D3ED000A05F5F96330EE670A86
:1085200093ED001A8DED070A04F5C8403C30CDEDFF
:10853000060A8DED051A76F0C1F80546204600F0D2
:10854000A3FE9DF827309DED051ADDED060A9DED91
:10855000070ACDE90203CDE900A54B46424639465C
:1085600030467BF077FEC2E72046918803F084FF17
:108570000020BCE7114620460AB0BDE8F047FFF7EF
:108580006FBE20460AB0BDE8F047FFF729BE11468E
:1085900020460AB0BDE8F047FFF79ABE20460AB071
:1085A000BDE8F047FFF720BA20460AB0BDE8F04723
:1085B000FFF75ABA00F5A04078300AB0BDE8F0479E
:1085C000FFF7CEBA0AB0BDE8F047FFF76DBB00BFBA
:1085D00038E20C08102C002070B500F5A0421346BC
:1085E000D2F8AC2178339A4205460E4602D00024D8
:1085F000204670BDFFF7AEFE04460028F7D005F513
:108600005B503188303054F097F9F1E721F04003A6
:10861000152B04D0A1F15E03584258417047012048
:108620007047000018294ED8DFE801F00D11151928
:108630001D2125292D4D313539453D3D414D4D4DAE
:108640004D4D4D4D490000F5A1403430704700F5C7
:10865000A0400C30704700F5A0401430704700F582
:10866000A0401C30704700F5A0402430704700F552
:10867000A0404C30704700F5A0405430704700F5E2
:10868000A0405C30704700F5A0407030704700F5A6
:10869000A0407830704700F5A1401030704700F5D9
:1086A000A1401830704700F5A1402030704700F518
:1086B000A1402C30704700F5A1403C30704700F5D8
:1086C000A1406430704700207047000000290DDB96
:1086D000074890F8542FCBB29A4207D3D0F8503FB6
:1086E0000122595CA0F5005006F0BCB8704700BFED
:1086F000104C00202DE9F34100F5005300F55B55C7
:1087000093F8203F03F0010603F0020803F004078A
:108710005B07044605F1300535D01F4A062128467F
:108720004FF01AFF26B104F54950243078F04AF88A
:10873000B8F1000F04D004F54E503C3077F0BEFD88
:1087400027B104F55450143078F066FC04F5C044A9
:10875000012384F8E134114A114B1249B8F1000F9A
:1087600008BF1A46002F08BF1946CDE900210E4A5E
:108770000621002E18BF134628460C4A4FF0ECFE87
:1087800002B0BDE8F0810A4A0621284602B0BDE8E1
:10879000F0414FF0E1BE00BF65E20C085AE20C0860
:1087A000C8C20D0861E20C0854E20C0876E20C081D
:1087B00088E20C0810B5044600F54950243078F0E2
:1087C0002DF804F54E503C3077F0A4FD04F55450DC
:1087D000143078F05BFC04F5C04393F8E1245AB1FF
:1087E000002283F8E12404F55B50044ABDE8104000
:1087F000062130304FF0B0BE10BD00BFA8E20C081B
:1088000009B1FFF777BFFFF7D5BF000000F5A04221
:108810000848D2F8AC11814209D092F8B90138B9B0
:1088200013467833994203D192F8DE07704700204F
:10883000704700BFC47C002010B504467FF01EFEC8
:10884000054BD3F8CC31C01A642804D82046BDE8C3
:10885000104058F0C7B910BD107C002010B500F5CD
:108860003C54D4ED047AF5EEC07AF1EE10FA8AB0F9
:108870004FF0000304F1100445D9079308930993BE
:1088800006AB019300F5A05007AB009303AA05AB1C
:1088900004A9103009F05AFA30B3DDED080A9DED55
:1088A000070AA8F0C3FFDDED090AA8F0BFFFD4ED69
:1088B000007A9DED047A77EEA76AB4EEE70AF1EE4E
:1088C00010FAF4EEC76AACBF01200020F1EE10FAF6
:1088D0000CD802309DED037AF4EEC77AF1EE10FA6F
:1088E0000CD8003818BF01200AB010BDF4EEC77ACA
:1088F000F1EE10FA9CBF0130C0B2EBE7012894BF43
:1089000000200120F0E70020EEE7000010B5074B43
:108910001A7A4AB901241C724CF0E0FC224611215B
:10892000BDE810404CF092BA10BD00BF0891002085
:1089300010B5074B1A7A4AB100241C724CF0CEFCD9
:1089400022461121BDE810404CF080BA10BD00BF96
:1089500008910020F0B5054685B005F5A05668469B
:1089600010360EF0D5FE6946304609F043FBA0B143
:108970003248334C334F75F0A1FE40B105F53C53FE
:10898000D3ED047AF5EEC07AF1EE10FA07D80023A1
:1089900028462380FB73FFF7CBFF05B0F0BD2846C8
:1089A000FFF75CFFA0B363787BBB23780133DBB2B6
:1089B000082B237002D1304609F034FA2378092BB2
:1089C00002D1304609F026FA2378092B1DD94FF43D
:1089D000857323804CF082FC022210214CF036FA81
:1089E0007FF04CFD6368C01A47F23053984209D9B2
:1089F00005F55B50144A022130304FF0ADFD7FF099
:108A00003DFD60602846FFF781FF6378FB73C4E794
:108A10002678002EF9D0013E6378F6B22670002B3E
:108A2000F3D0002EF1D166704CF058FC3246102184
:108A30004CF00CFA2846FFF77BFFE6E74C9000204D
:108A400008910020AD910020BCE20C0800F5A04088
:108A5000D0F83038042B14BF90F85C080120704720
:108A600073B500F5A0450192A5F8C41104467FF046
:108A700005FDC5F8C801D5F8AC0103685B689847E7
:108A800085F8C201D5F8AC0103685B6898470F28E8
:108A9000019A0BD80F2827D8DFE800F01C261C1CF1
:108AA0001C1C1C1C1C264E260A260A0A18281BD130
:108AB00004F50056019296F9EC34ABB1D5F8AC014F
:108AC00003685B68984785F8C20196F9EC34019A0F
:108AD000022B29E01F4B93F8E23403B304F5A041C5
:108AE0004C31204605F0E6FDD5F8AC0195F8C261A1
:108AF00003685B68984704F55B54864204F13004D0
:108B000020D0D5F8AC0103689B689847124A034609
:108B10000421204602B0BDE870404FF01DBD04F5B1
:108B2000005393F9EC34022BD8D004F5A041042B68
:108B30000CBF54310C31D4E72046FFF787FF0028E3
:108B4000D2D1B5E7054A0421204602B0BDE8704005
:108B50004FF002BD108C0020CCE20C08EEE20C08B5
:108B6000F0B5044604F5A04685B00F46154657F00B
:108B7000BFFFD6F8AC01A6F8C47103685B689847DC
:108B800018281ED8DFE800F00D0D0D0D0D0D0D0D90
:108B90000D1D53690D0D58581D1D1D1D1D1D1D1D3D
:108BA0000D00314BD3F83028012A21D104F50053B0
:108BB00093F8ED34023B012B1AD904F5405383F8A6
:108BC000EC26D6F8AC01294A294B052D18BF1346CF
:108BD000026803939268904704F55B543034009028
:108BE000039B244A042120464FF0B6FC05B0F0BD9B
:108BF000214B93F8E2343BB104F5A0412A464C31B5
:108C0000204605F057FDDCE704F5005393F9ED34F9
:108C1000032B03D1204603F08BFCD2E7022BEBD0D1
:108C2000042B15D104F5A0412A467831E8E7204607
:108C3000FFF70CFF0028C4D104F5005393F9ED347D
:108C4000032BE7D0022BD7D0042BEBD0012BB8D1CC
:108C500004F5A1412A461031D2E704F5005393F9F7
:108C6000ED34042BADD1DDE7107C002004E30C08CB
:108C7000FDC60C080CE30C08108C002070B500F544
:108C80005B5504463035124A0421284604F5A046B7
:108C90004FF062FC0023A6F8C43104F5005393F8AA
:108CA0003434032B12D196F8C2113022204605F03D
:108CB000D9FDD6F8AC0103689B689847054A03467E
:108CC00006212846BDE870404FF046BC70BD00BF8D
:108CD00020E30C0837E30C0800F5405310B50022E0
:108CE0000529044600F55B5083F8EC2600F13000BE
:108CF0000CBF054A054A042104F5A0444FF02CFCA2
:108D00000023A4F8C43110BD50E30C0861E30C0843
:108D100030B50B4687B00446052A18D8DFE802F0C4
:108D2000172A0350175D00F5A043D3F83038042B01
:108D300020D02C4D95F8D531E3B12B4905F65400E0
:108D400026F04AF928B1274B012283F85C2807B0A6
:108D500030BD254905F6540026F03EFC50B104F51F
:108D6000A04104227831A5F5A04007B0BDE830400D
:108D700005F0A0BC04F5A043D3F83038042BE6D0AE
:108D800004F5005393F9B734022B0AD1154890F833
:108D9000D53133B1144900F6540026F01DF90028EE
:108DA000D1D104F5A14104221031204605F082FC06
:108DB00004F51150373007B0BDE8304042F06AB9D1
:108DC0000A4A112101A87EF0B9FB04F5C54001AAA9
:108DD0000121143078F00CFAB9E707B0BDE8304053
:108DE00003F0A6BB107C0020408F00207CE30C0821
:108DF00070B52DED048B04467FF034FB4F4BB4F877
:108E0000BE101A884E4E8A4205464E4A06D0198038
:108E1000002330601370BDEC048B70BD33684A4989
:108E2000C31A8B4276D90123137057F061FF57F0B4
:108E300019FE356057F05CFF57F014FE04F54053FF
:108E400093F8EB3623B104F5C540143078F024F9DB
:108E500057F030FE0428DED957F04AFE00212046A4
:108E600003F090FE00212046F0EE409A03F094FEBD
:108E700001212046B0EE409A04F054F8002120462B
:108E8000B0EE408A03F092FE04F5C8403C30F0EEAC
:108E9000408A75F01DFCDFED2D7A0028B0EE690ADE
:108EA0004FF0040008BFB0EE678A59F0A1FAB0EEA7
:108EB000490A132059F09CFAB0EE680A152059F0BF
:108EC00097FA04F5C545B0EE680A1A2059F090FAF1
:108ED00014354620B0EE480A59F08AFA284678F050
:108EE00069F908BB0121084659F084FD9FED170A76
:108EF000022059F07DFA9FED150A032059F078FA07
:108F0000204604F02BFABDEC048B2046BDE87040EF
:108F100005F056B91278002A3FF47DAF44F620627E
:108F200093427FF678AF80E72846FDF717F804F5FF
:108F3000C04393F99E322B2BD4D06CE714910020C0
:108F40001891002016910020400D03000000000041
:108F500000F5A0431846D3F8AC217830824202D104
:108F600093F85C08E8B10F4B93F8340403F58043A1
:108F7000A0F12702012A93F8F0340FD92C2809D048
:108F80000A2809D0A0F13102504250410A2B18BFE3
:108F9000002070470120F9E7012070470A3B584242
:108FA00058417047104C002008B500F5005393F865
:108FB000202342B193F85C332BB1FFF7C9FF80F057
:108FC0000100C0B208BD0120FCE700002DE9F04718
:108FD00000F50055A64F95F85C83044600F5C8409F
:108FE0008AB03C3075F06AFBD7F83038042B06465F
:108FF0004FD000284DD0B7F89218A7F5A040FFF742
:1090000005FB014620B197F858184B1E59425941AB
:1090100004F50C57DFF86CA22037384664F05AFE8E
:109020009AF8F0340A2B814603D1A6BB00238AF8B4
:10903000F03495F82033002B39D195F926338D4D36
:10904000012B03D0063BDBB2012B11D895F8343449
:109050000A2B0DD104F5A046D6F8AC0103681B6AB3
:10906000984728B1D6F8B0112B22204605F022FBF4
:109070009AF8F0340A2B04BF37238AF8F03495F8B5
:1090800034340A2B02D1372385F834340AB0BDE8D2
:10909000F0870121BCE740EA0803DBB2002BC8D10E
:1090A000AAF5C04000F0F0F80028BFD0C1E7002EBC
:1090B000ECD004F5C44008307BF042F80028E5D13C
:1090C0002046FFF745FF0028E0D1B9F1000F00F07E
:1090D000BD8069494A46384664F0D4F995F926833B
:1090E000B8F1010F06D040F38380A8F10603DBB28C
:1090F000012B7DD85FFA88F8B8F1010F4BD104F548
:10910000A0421346D2F8AC117833994207D192F8B5
:109110005C3823B195F8B734013B012BB6D904F57F
:10912000A1410A221031204606AE05F0C3FA3046AE
:109130000EF0EEFA95F9392392BBB8F1010F2FD05A
:1091400004F5C048B5F93A33D8F81C13DFED4B5A93
:10915000D1ED017A002BF8EEE77A52DD07EE103AF6
:10916000F8EEC76AE6EEA57A3046FDEEE77A17EE2E
:10917000901A0EF0D3FA00233846CDE9043364F098
:1091800045FE04A965F086FB002859D0049B08938E
:10919000059B099317E004F5A1410A222031C2E79B
:1091A0002046FCF753FF07EE900A6F4604F5C642CF
:1091B000303221463846B8EEE70AFEF76BF897E8FA
:1091C0000F0086E80F0095F92633012B10D03146A9
:1091D0002046FDF7A7FB31462046FDF73FFF95F9F6
:1091E0002633072B04D104F54054012384F8EA36D2
:1091F0004CF074F84A4609210AB0BDE8F0474BF03C
:1092000025BED5EDCA6A95EDCD5A95EDCB7A35EEF2
:10921000076A36EEC57AB4EEC67AF1EE10FA8DBF63
:1092200037EE067A05F5A36393ED007A27EE257AEB
:109230008ABFF6EE006AE7EE257AE7EE267A93E734
:10924000D8F81C339A680892DB68A2E7B8F1000FDF
:109250003FF41CAF95F85C33002B7FF417AF04F597
:109260005B50074A052130304FF076F9C0E700BF68
:10927000107C0020104C002088E30C080000C8423D
:1092800091E30C08108C002010B5044600F5C8408E
:109290003C3075F01DFA04F5A04404F6340494ED56
:1092A000007A48B1DFED067AB4EEE77AF1EE10FA13
:1092B000ACBF0120002010BDDFED027AF4E700BF53
:1092C000CDCCCC3D6666663F10B500F5A04200F5FA
:1092D000A141D2F8AC413C318C42034602D192F814
:1092E000280888B903F5A04378339C420DD192F841
:1092F000280848B1D2F83038032B06D1B2F89208CA
:10930000A0F116035842584110BD0020FCE70000B0
:109310002DE9F84F00F5A0463346D6F8AC21783356
:109320009A42054604D100F5005898F9903433B9B3
:109330000023C6F81C3886F81938BDE8F88F7FF08E
:109340009DF8D6F8D047814634B1041B40F6C313CC
:109350009C4294BF002401242846FFF795FF8346D2
:1093600020B1002486F8184800273FE005F5C840E2
:109370003C3075F0A3F982460028F2D005F5C447C9
:10938000083738467AF0DCFE002840D096F8187886
:10939000C7BB44B305F5805141F27072D1F808366D
:1093A000002BB8BF5B42934206DCD1F80C36002B91
:1093B000B8BF5B42934228DD05F5B14105F5C640D3
:1093C000183130300EF006FDDFED467AC6F81C98F5
:1093D000B4EEE70AF1EE10FA4FF000034CBF01279C
:1093E0000027C6F82038012386F8183805F5907054
:1093F000F8F790FB022835D9002C46D10023C6F897
:109400001C389AE75C465F46EDE73C46EBE738469A
:109410007AF07EFE074638B1002CA5D04FF4FA73DF
:10942000C6F8203854469FE7D6F83038012B03D0D1
:10943000032B0FD03C46D9E708F5A663D3ED007A9D
:10944000F5EEC07AF1EE10FAF4DD96F82838002B2C
:10945000F0D1E3E72846FFF737FF0028EAD1002CD8
:10946000DCD1C3E705F5055A0AF1100A98F89E12F7
:10947000504606F05BFE0028C0D098F89E12504679
:1094800006F04CFF0028B7D1B8E7D6F81C3813B95E
:10949000C6F81C9851E7D6F82028A9EB030393429D
:1094A000FFF44BAF96F81938002B7FF446AF01223A
:1094B00086F8192898F89034DB0705D505F5C840DB
:1094C0000C213C30F8F75EFA05F55B5030302FB1D7
:1094D000054A0221BDE8F84F4FF03EB8034A39462D
:1094E000F8E700BF00009642A8E30C08BEE30C08B2
:1094F0002DE9F04F2DED028B054685B0002305F5D3
:10950000005803937EF0BAFF08F28C43D3ED007A43
:10951000F5EEC07AF1EE10FAC4BF9FEDC07A67EEA7
:10952000877A05F5907BC8BFFCEEE77A0746584678
:10953000CCBF17EE906A9626F8F7ECFA022840F2B4
:10954000FC8095F814349FEDB67AB02202FB0353E9
:10955000D3ED837A67EE877AFCEEE77A17EE903ADE
:109560009E428CBF00260126B8F98034022BB8BF7A
:10957000022307EE903A05F5A050B8EEE78A03A95A
:10958000F6EE087A103028EE278A08F011FD04461E
:1095900040B1DDED037AF4EEC87AF1EE10FAACBF1B
:1095A000012400245846F8F7B5FA05F5C849012802
:1095B00009F13C0905F5A04A18D8484675F07EF82F
:1095C000A0B19CB90AF6340292ED007ADFED957AEB
:1095D000B4EEE77AF1EE10FA08DDDDED037AF4EE91
:1095E000C87AF1EE10FAACBF01240024484675F0A9
:1095F00065F80090002800F0FE8095F8142405EB33
:109600000212D2F8C02172B158460192F8F782FADC
:10961000012800F29480019A41F28731BA1A8A42F5
:109620008CBF00220122DAF8CC1701B11AB9002C44
:1096300040F087803446DAF8AC1105F5A042783264
:1096400091421AD198F9B824002A40F08280002271
:109650008AF81A28DAF83028042A00F0AA80072AA3
:1096600000F0BD80032A08D12846FFF72DFE20B167
:1096700000248AF81948CAF8D0479AF81A2802B183
:109680008CB907EE904A9FED687AF8EE677A0AF691
:10969000340267EE877AD2ED006A9FED647AE6EED7
:1096A000877AC2ED007A2846FFF7EEFD044698B1AE
:1096B0009AF83808CAF8CC7708B9CAF83C78DAF8CA
:1096C000AC1105F5A0427832914205D1DAF8D027E5
:1096D00002B108B9CAF8D0779AF860298AF83848F0
:1096E00064F3C3028AF860296FF022F921466FF013
:1096F000FBF84F4A28465471FFF70AFE2846FBF74D
:109700001FF934B198F836241AB97EF0B7FEC8F8BC
:10971000380488F836442846FFF7B6FD00287BD188
:10972000484674F0D5FF80F00100C0B28AF84008C6
:1097300005B0BDEC028BBDE8F08F002614E70022D7
:1097400071E71FF039FB1EF02DFB00287FF472AF8C
:1097500071E7524207EE902A05F61862F8EEE77AB2
:1097600092ED007AF4EEC77AF1EE10FA13DD0122E1
:109770008AF81A28CAF824780AF63402DFED2D7A1E
:1097800092ED007AB4EEE77AF1EE10FA7FF762AF6D
:10979000C2ED007A5EE79AF81A28002A3FF45AAF21
:1097A000DAF8242840F6B831BA1A8A423FF64FAFA9
:1097B00050E705F5C44008307AF0AAFC00283FF4D1
:1097C0005CAF0AF2BC7292ED007ADFED1A7AB4EE69
:1097D000E77AF1EE10FA7FF750AF009C4DE70AF2FE
:1097E000BC7292ED007AFEEE007AB4EEE77AF1EE0A
:1097F00010FAF2D441E7DAF83028002C18BF3446CA
:10980000012A07D005F5C44008307AF077FC00281B
:109810003FF433AF002430E7002087E70000B44274
:109820000000C8429A99993E9A99193E9A99593FCF
:10983000AD910020CDCC4C3E0020704700207047F9
:10984000012070470020704701207047034BD3F878
:109850003008431E58425841704700BF107C00201A
:1098600030B587B002A80DF053FF3B487AF046FCB4
:1098700020B13A493A48FDF767F81FE036487AF0D8
:1098800047FCE8B1374C04F12405234604F11002EB
:10989000A4F11001A4F5947000957AF05FFCCDE975
:1098A0000045A4F66C3292ED000A2F4904F1100332
:1098B000A4F11002A4F594707AF012FC07B030BD48
:1098C000254802A97AF062FC08B102A9D2E7274C28
:1098D000D4F8B83E002B0CDD94F8583E4BB1A4F5FB
:1098E00000502049FDF730F8A4F50050FCF7C6FC05
:1098F000E4E71B4802F0DAFC0028BAD11C4C94F8CB
:1099000040335B0720D4D4F85433002BB1D0134A32
:10991000A2F12001A2F110000EF0C8F90028A8D190
:10992000144C0F48D4ED007AB7EE000A04F67831F3
:1099300030EE670AFDF738F8094804F6583204F6A5
:109940007831FCF7DFFBB9E7A4F5C040FDF7A8F8D4
:109950000028B3D1D7E700BF188E0020508F002019
:10996000102C0020408F0020685B0020104C00204D
:10997000108C0020D883002008B50A4890F82935BB
:10998000013B012B03D8A0F50050F9F731F9064847
:10999000F9F758F80448F9F7F1F8BDE8084002482B
:1099A000F9F70CBC104C0020102C0020124A9042F9
:1099B00008B50ED002F1080188420AD002F1100168
:1099C000884206D002F13801884202D05C329042CF
:1099D00006D10A4B93F9E104B0FA80F0400908BDC2
:1099E00003681B6A984728B1054B93F8EA0680F094
:1099F0000100F4E70120F2E7247C0020104C002055
:109A0000105C0020104A904208B518D002F10801FD
:109A1000884214D002F11001884210D002F13801BE
:109A200088420CD05C32904209D003681B6A984788
:109A300038B1064B93F8EA0680F0010008BD00201B
:109A4000FCE70120FAE700BF247C0020105C002026
:109A5000024A0260024A4260704700BF10E40C08EC
:109A60002040002008B503681B6E98470648D0F8D0
:109A7000AC2100F170039A4205D0BDE80840A0F582
:109A8000A040FEF797BE08BD107C00202DE9F843EA
:109A9000484C04F2A47300221A6004F17803C11A3E
:109AA0004B42A4F500584B4188F88C3904F2B4734A
:109AB000002584F88857A4F8DE5784F8E25784F824
:109AC000A05784F8195884F81A58C4F80858C4F8EC
:109AD0000458C4F80058C4F810581A60436804F5D4
:109AE0008059D3F8FC31A4F8D83709F54C730646F1
:109AF0000FCB04F5995787E80F0084F8E15784F8F5
:109B0000F057C9F8FC527EF0B9FCC4F8B4013368D0
:109B100030465B6998474FF0FF3384F8E40784F8D8
:109B2000E55788F8EC5689F8595384F8E357C4F898
:109B3000DC3133683046DB6D98470546002836D067
:109B4000336830469B6B984784F82808D8F8180982
:109B50000368DB6B984708F5D16076F09BFFA4F5AE
:109B6000A04002F07BFFA7F5804064F019F994F85B
:109B70005C38CBB1A4F5A040FFF786FBA0B907F590
:109B80008E7074F0A5FD78B9D4F8AC0103685B6BF6
:109B9000984748B955F0B8FB074A06214EF0DCFC5F
:109BA00004F6540025F0C4FA0448F8F771FA284680
:109BB000BDE8F883107C0020D0E30C08102C0020B6
:109BC00070B503685B6E0E4615469847044650B95B
:109BD00095F900303BB90548054B00683246C06A2C
:109BE00029461BF08DFF204670BD00BF0C2C0020C5
:109BF000F4E30C0810B50E4C204676F047FD04F552
:109C0000AC7076F0BFFA04F52C7077F0EDF9094BE3
:109C100003F5A042002182F8A01702F2A4720021ED
:109C200003F540531160012283F8B02110BD00BF3D
:109C3000745E0020102C002008B52DED028B15203D
:109C4000B0EE408A58F0D4FBB0EE480ABDEC028B6F
:109C50001A20BDE8084058F0CBBB000008B5084802
:109C600090F9E1340121A0F5005033B103F05AF925
:109C7000BDE80840462058F0BBBB03F07BF9F7E78E
:109C8000104C0020042070470048704722270E081F
:109C90000048704722270E08037A73B1D0ED037A8B
:109CA000FDEEE77A17EE903A084AC2F84438437A54
:109CB0003BB10369C2F8483870474368D3F8F831BC
:109CC000F2E74368D3F8FC31F4E700BF107C0020D2
:109CD00008B50023038100F11401406808F07EF903
:109CE000012008BDF8B56D4E2DED048B0446012111
:109CF000304606F5A04797ED7D9ADFED699A02F0B0
:109D000041FF0121B0EE408A304602F045FFC8EE27
:109D1000297A06F500556068B5F9043504F1140197
:109D200008EE903AF8EEE88AB5F9063568EEA78AAB
:109D3000C0EE297A08EE103AB8EEC88A28EE278AD3
:109D400008F04CF995F90A355BB39FED567AF0EEC1
:109D5000E87AF4EEC77AF1EE10FA22D5227A636837
:109D6000002A54D1012222720022E26094ED037A8B
:109D7000DFED4D7AD3F8F8314C4867EEC77A9FEDA6
:109D80004C7A67EE877A0122FDEEE77AB0EE490A57
:109D900017EE901A0B44C7F84438002376F006FCFF
:109DA00008E0002341482372F0EE490AB0EE680A49
:109DB00076F0F8FB042058F01BFB95F90A3543B107
:109DC0009FED387AF0EEC87AF4EEC77AF1EE10FA29
:109DD00028D4002337486372F0EE490AB0EE480AEF
:109DE00076F03AF8132058F003FBB5F90835002B4C
:109DF00003DD314E96F92A355BBB28482021F8F760
:109E0000B5FB002842D1254802F0F8FC41E0D3ED33
:109E1000C56A96ED467AD4ED037AE6EE877AC4ED0C
:109E2000037AA3E7637A2BB9012363726368D3F8DB
:109E3000FC3123612169C7F848186368D3F8FC0135
:109E40000023091A1A461B48B0EE490A76F0EAF8D0
:109E5000C8E70121A6F5405002F0A8FE80EE297A5D
:109E6000B5F90835002106F2145007EE903AF8EEE5
:109E7000E77AF0EE490A27EE870A76F0B5FFBDECE7
:109E8000048B2046BDE8F840FFF7D6BE0348F9F73B
:109E900001F807EE900AB8EEE70AF0E7102C002070
:109EA00000A08C4500000034E02E6542745E002066
:109EB0000000C842CC5F0020105C00202DE9F04F6C
:109EC0002DED0C8BDFF8A0A39FEDDCDA9FEDDC9A83
:109ED00097B000F114050AF5A04B04460121504645
:109EE0009BED7DBA02F04EFE01215046F0EE408A15
:109EF00002F052FE01215046B0EE408A02F056FEBA
:109F0000DFEDD07A88EEA77A0AF5005601A8B6F9F7
:109F100004350AEE903AF8EEEAAAB6F90635DFED16
:109F2000CA8A6AEE87AA88EE277A0AEE103AB8EE55
:109F3000CAAAB6F908359FEDC58A2AEE07AA80EEAF
:109F4000277A09EE903AF8EEE99A6AEE8D7A69EE90
:109F5000879AF0EEEACAF4EEC8CACDED017AB0EE07
:109F6000CACA6AEE0D7AF1EE10FAF0EEE9BAB4EE72
:109F7000C8CACDED027A58BF4FF0010969EE8D7A5B
:109F800048BF4FF00009F1EE10FAF4EEC8BA9AEDAE
:109F9000460ACDED037A54BF4FF001084FF0000898
:109FA000F1EE10FA54BF0127002721F057FF01A955
:109FB000284621F05DFA284621F04CFB284621F086
:109FC000C3FA20EE090A284620EE280ABDEEC00A90
:109FD00010EE103ACBF8443821F0D0FA20EE090AFE
:109FE00020EE280ADFED9A8ABDEEC00ACDED0D8A7B
:109FF00010EE103ACBF848380DF1280B4FF07E5395
:10A00000594660680A93CDED0C8ACDED0B8A07F0B6
:10A01000E5FF0021504602F085FFB0EEC00AB4EE25
:10A02000C80AF1EE10FA16D55046FFF72DF990B98F
:10A03000F4EEC8CAF1EE10FA0DD5B4EEC8CAF1EECE
:10A0400010FA08D5F4EEC8BAF1EE10FA44BF9BE856
:10A050000F0085E80F000AA821F060FB294612A82E
:10A060008DED141A8DED120ACDED130ACDED151AF2
:10A0700021F066FB0DF1100A51460EA88DED101A65
:10A08000CDED048ACDED058ACDED068A8DED0E0A63
:10A09000CDED0F0ACDED111A21F024F9B6F90435F2
:10A0A000DFED6C7A01EE103AB6F9063509EE103A9A
:10A0B000B6F9083508EE903AB8EEC11AB8EEC99A6A
:10A0C000F8EEE88A21EE271A29EE279A68EEA78A89
:10A0D000F4EEC8CAF1EE10FA21EE0D1A29EE0D9A2F
:10A0E00068EE8D8A07D594F82430DFED597A002B7D
:10A0F00018BFB0EE671AB4EEC8CAF1EE10FA07D571
:10A1000094F82530DFED527A002B18BFB0EE679A35
:10A11000F4EEC8BAF1EE10FA07D594F82630DFED68
:10A120004C7A002B18BFF0EE678A9AE8070007AE5A
:10A1300086E80700F1EE410AC2209DED070A1FF0F4
:10A14000B7FBC3208DED070AB0EE491AF1EE490ABC
:10A150009DED080A1FF0ACFBB0EE681AF1EE680A3C
:10A160008DED080AC4209DED090A1FF0A1FB5146A0
:10A1700030468DED090A21F007FE12A928468DED23
:10A18000120ACDED130A8DED141A21F071F928464B
:10A1900021F060FA304BDDED076A93ED9A7A9FED7E
:10A1A000280AC6EE877A3046DDED086ACDED077ADB
:10A1B000D3EDF07A86EEA77ADDED096A8DED087AA7
:10A1C00086EEA77A8DED097A21F048FEB9F1000FED
:10A1D00001D0CDED07AAB8F1000F01D08DED08AA8E
:10A1E0000FB1CDED099AF0EE4B0A9DED070A1B4821
:10A1F00076F0D8F9042058F0FBF8F0EE4B0A9DED0C
:10A20000080A174875F028FE132058F0F1F80021CD
:10A21000F0EE4B0A9DED090A124876F0E5FD204666
:10A22000FFF70AFD84F8249084F8258084F82670CE
:10A2300017B0BDEC0C8BBDE8F08F00BF35FA8E3C3B
:10A24000E02E654200A08C450000C84200000034AA
:10A2500000000000CDCC4C3E105C0020745E00205D
:10A26000CC5F002024610020102C002010B5044693
:10A27000FFF7F4FC0B4B93F90A25022A0DD1B3F931
:10A280000825002A09DD03F5805393F92A3523B107
:10A290002046BDE81040FFF711BE2046BDE8104043
:10A2A000FFF720BD104C00200A207047004870477F
:10A2B00031F00C080048704731F00C08012070475D
:10A2C000012070470120704701207047012070472E
:10A2D000034BD3F83008031F58425841704700BF62
:10A2E000107C0020F8B51B4D05F59954234610331A
:10A2F0000FCB05F59A5684E80F0086E80F0000277B
:10A3000005F6540085F8E47725F052F9124B1C68E5
:10A31000E66A336830465B689847A8B196F84D30D6
:10A3200093B1E36A9B8F7BB154F0EEFFE36A0B4A73
:10A330009B8F06214EF010F9E36A05F65400998FC1
:10A3400024F022FFE36A9F8705487AF06FFE012020
:10A35000F8BD00BF107C00200C2C0020E8E40C08A5
:10A36000E058002010B50A4C94F85838012B0AD157
:10A3700004F6540022F0E0F9B4F89238152B02D11B
:10A38000044879F09BFF0023C4F8D03710BD00BF0C
:10A39000107C0020188E002008B508F025F890F8F1
:10A3A0007C32DB0704D5BDE80840024824F09CBF9E
:10A3B00008BD00BF6484002010B52F4C94F85838B5
:10A3C000012B0ED004F190010822A4F5A04004F066
:10A3D00071F954F099FFBDE81040284A06214EF06B
:10A3E000BBB8B4F89238162B05D0152B34D1D4F85D
:10A3F0003038072B0AD1224804F0E6FC204804F04C
:10A400002FFEBDE810401E4804F040BDA4F5A0405A
:10A41000F9F744F8A4F5A040F8F73EFFA4F540533F
:10A42000D4F8441893F94825164864235A4379F020
:10A43000A1FEC4F84408134879F0DEFF30B1BDE84E
:10A4400010409FED110A462057F0D2BFA4F5A0405E
:10A45000BDE81040F8F706BD1E2B18BF4FF0FF33C4
:10A46000074818BFC4F89C37F9F718F80448F8F7FC
:10A4700013FF0348ECE700BF107C002000E50C0848
:10A48000102C0020188E00200000000010B5144B86
:10A49000B3F89238532B04461ED103F035F99FEDE3
:10A4A000110A462057F0A4FF9FED0E0A492057F0ED
:10A4B0009FFF9FED0C0A4A2057F09AFF462058F064
:10A4C00077F8492058F074F84A2058F071F820467F
:10A4D000BDE81040FFF78EBBBDE81040FFF74CBA57
:10A4E000107C0020000000000820704700487047E2
:10A4F0009CE50C0800487047A8E50C08012070474F
:10A5000008B50248FEF7F6F8012008BD102C00201F
:10A51000014800F061B900BF5C7C002010B5044622
:10A52000FFF72AFA2046BDE81040FFF797BB00006E
:10A53000012070470048704720E60C08004870472B
:10A5400028E60C08012070470120704710B5054B24
:10A5500003F5507403F54C730FCB84E80F00012012
:10A5600010BD00BF108C002008B50B4800F5A042BC
:10A5700000F500530321D3F8483F93FBF1F3C2F8F1
:10A580004438F8F7F1FE0448F8F786FEBDE80840C5
:10A590000148F8F767BC00BF102C00200720704767
:10A5A00000487047BAC80C0800487047A0E60C087D
:10A5B000012070470120704701207047704700005C
:10A5C00008B500230372036103487AF02FFD0348A6
:10A5D000FCF778F9012008BDE0580020102C00207D
:10A5E00010B5194CD4F8303FB3F9083023B9D4F87A
:10A5F0003C3FB3F90830F3B1002303720361D4F890
:10A60000300F56F065FC04F64873D3ED007A0F481E
:10A61000F8EEE77A27EE800ABDEEC00A10EE103A97
:10A62000C0F84438A0F5A040F8F79EFEBDE8104001
:10A63000074801F039BD037A002BE0D0A4F50050A3
:10A64000F8F72CFFF2E700BF104C0020107C002030
:10A65000102C002070B54F4DDFED4F7A95F8143473
:10A660009FED4E7A2DED048BB02606FB035393ED40
:10A67000848A9FED4B9A28EE278A05F5B053BDEEEC
:10A68000C88A93ED070AF8EEC87A044667EE897A1D
:10A6900097EE870A1FF0F8F8237AF0EE408A002B35
:10A6A00063D105F50053D3F8303FB3F90830002BE0
:10A6B0005BD1284602F0A2F8002856D195F8143450
:10A6C00095F8581406FB035393F8F12100294CD157
:10A6D000012A4AD993ED837AF0EE087AB4EEE77A4C
:10A6E000F1EE10FA41DBDFED2F7AB0EEE80AB4EEBE
:10A6F000E70AF1EE10FA38D523699BB37DF0BEFE70
:10A700002369C01AB0F5FA7F33D8237A002B3DD0E5
:10A71000254DA5F1200696E80F0085E80F0094ED81
:10A72000038AA5F110013046B8EEC88A0DF052FB3D
:10A7300028EE098ADFED1D0A284670EE200AB0EEE9
:10A74000480A0DF0BDFBA5F54D53BDEC048BD3F8C5
:10A7500018099FED170A03682A4631469B6ABDE82F
:10A76000704018477DF08AFE20612369002BCCD011
:10A77000C4E7104D84ED038A012323720023236173
:10A7800005F110030FCB85E80F00BEE7BDEC048B8D
:10A7900070BD00BF102C00200000C84235FA8E3C6E
:10A7A0000AD7233CDB0FC93F508F002000007A44BA
:10A7B00000000000308F0020C3680B60007A7047F3
:10A7C000052070470048704718E70C08004870479C
:10A7D00028E70C080120704738B52DED028B4D4C51
:10A7E0009FED4D8AD4F8300F56F072FBD4F8483FF5
:10A7F00007EE903AF8EEE77A04F5405527EE800A26
:10A80000A4F50050BDEEC00A10EE103AC5F8443869
:10A81000F8F7AAFDD4F8340F56F05AFBB5EEC00A8B
:10A82000F1EE10FACBBF04F5936304F64C73D3ED4D
:10A83000007AD3ED007A3948CBBF20EE270A20EE0C
:10A84000270A20EE080A28EE400ABDEEC00A10EEE4
:10A85000103AC5F84838F8F751FD04F5936393EDC5
:10A86000007AD5F8480804F64C7327EE087AD3ED41
:10A87000007A27EE888AFDEEC77A17EE902AFDEE61
:10A88000C87A17EE901A1FF0B3F8C5F848082348A5
:10A89000FDF7BCFF20B1D5F848385B42C5F8483811
:10A8A00095F8C03163B194F9EC34022B08D1002340
:10A8B00001214620C5F84438C5F8483858F0F2F868
:10A8C00056F016FA5F2157F045FAF8B157F012FA30
:10A8D00002281BD195F8E137C3B905F2B47304F52A
:10A8E000A76493ED007AD4ED007AB4EEE77AF1EE46
:10A8F00010FA0BD5012385F8E137BDEC028B084A2D
:10A900000848BDE8384004214DF026BEBDEC028B5E
:10A9100038BD00BF104C00200000C842102C0020A1
:10A9200030E70C080063002010B50446FFF724F858
:10A930002046BDE81040FFF791B90000062070479F
:10A9400000487047B0E70C0800487047C0E70C08A3
:10A950000120704701207047012070470120704797
:10A960007047000008B504487AF060FB0348FBF725
:10A97000A9FF012008BD00BFE0580020102C0020D6
:10A9800038B50F4C04F50055D5F8300F56F0A0FA45
:10A9900005F64872D2ED007AF8EEE77A04F5A043A6
:10A9A00027EE800A2046BDEEC00A10EE102AC3F83A
:10A9B0004428F8F7D9FC2046BDE8384001F074BBC4
:10A9C000102C00200F2070470048704738E80C0812
:10A9D0000048704740E80C0801207047012070478C
:10A9E0000120704701207047012070470120704707
:10A9F0007FB50B4D05F54053002283F8EA2605F597
:10AA0000C643303306460FCB6C4684E80F00002364
:10AA10002846B3602146FCF721FB012004B070BD3D
:10AA2000102C002010B53C4CD4F80038002B2CDD45
:10AA30007DF024FDD4F80038C01A40F6B7339842B0
:10AA400023D8A4F54053D4F8F407D3F8482F514243
:10AA50001EF0CEFFC4F84408A4F5A040F8F784FC2B
:10AA6000D4F80438002B14DC2C48F8F715FC2C48DB
:10AA700090F8EA3693B30121A0F5405002F052FA63
:10AA8000BDE81040462057F0B3BC2448F8F706FD57
:10AA9000E6E77DF0F3FCD4F80438C01A40F6B7338B
:10AAA0009842E1D81F4BDFED206A93ED007AD4F88D
:10AAB000F80703F6B423D3ED007A27EE267A67EE83
:10AAC000A67ABDEEC77AFDEEE77A17EE102A17EEEA
:10AAD000901A1EF08DFFC4F84808C8E7A0F5805012
:10AAE00090F97734012B04DCBDE810400B48F8F7EF
:10AAF000B9B9D4F81038002BF6D07DF0BFFCD4F8EB
:10AB00001038C01A40F6B7339842EDD804F60C045A
:10AB100094ED000AB4E700BF107C0020102C002048
:10AB2000105C0020A85000200000C842D0ED027A3E
:10AB30000348FCEEE77A17EE903A99B201F09CBC1C
:10AB4000102C002084B010B503AC84E80E000B4834
:10AB500021466F22FCF7C6F99DF80C1011F0040194
:10AB600002D120460CF09EFE04482146FCF776FAFE
:10AB7000BDE81040012004B0704700BF102C002039
:10AB8000B0EEC00AFDEEC07A38B54FF6FF7205464A
:10AB90000C4617EE900A00211EF02AFF07EE900ADD
:10ABA000002CF8EEE77A054BC5ED027A14BF4FF0A2
:10ABB000FF32012283F8F82238BD00BF108C00203C
:10ABC000FEF74EBE0C20704700487047B8E80C08EE
:10ABD0000048704711270E08012070470120704778
:10ABE00001207047012070470120704708B50C48CC
:10ABF000FDF786F80A480B49FBF794FE0848F7F77B
:10AC0000AFFE40B106484FF48051F7F7AFFC10B1EA
:10AC10000348FBF757FE024800F09CFF012008BDE7
:10AC2000102C0020508F002008B50D48F8F736FC96
:10AC30000B48F7F795FE50B109484FF48051F7F7EC
:10AC400095FC20B1BDE80840054801F02DBA044844
:10AC5000F8F722FBBDE808400148F8F703B900BF48
:10AC6000102C002008B50A484FF48051F7F77EFCFD
:10AC700038B108480022D0F8501300F550700CF09D
:10AC80004DFDBDE808400248002101F0F5BB00BFC2
:10AC9000102C0020108C0020881A10B51EF0D0FD5A
:10ACA000104BD3F8F4220028B8BF4042002AB8BFA6
:10ACB000524248F6A041B2FBF1F24FF47A7102FB26
:10ACC000011188420CDC93F84023D20606D503F527
:10ACD000507403F54C730FCB84E80F00012000E0A3
:10ACE000002010BD108C002013B50446406801916F
:10ACF00000F57F7020F0ECFEDFED0A7A20EE270AE7
:10AD00001EF040FDDFED087A019920EE270A20466B
:10AD1000FDEEC07A17EE902A02B0BDE81040FFF7B2
:10AD2000BBBF00BFE02E65420000C84284B070B5D2
:10AD30002DED048B86B00FAD85E80E004D4CDFED98
:10AD40004E8A0646D4F8180904F5405494EDC30A17
:10AD50000368B0EEC00A5B6A9847B4EEE80AF1EE09
:10AD600010FAB0EE408A07DA012006B0BDEC048B81
:10AD7000BDE8704004B07047404928460CF036FFEB
:10AD800002A8CDED030A8DED020A20F045FF04A8CC
:10AD90008DED040AB0EE480ACDED050A20F036FE2E
:10ADA00013A928468DED000ACDED010A0CF01EFF17
:10ADB00002A88DED020ACDED030A20F0D3FEB4EE19
:10ADC000E80AF1EE10FACFDBB4EEC08AF1EE10FA29
:10ADD0009FED2B9ADFED2B8ADFED2B9A2BD802A863
:10ADE000694620F003FE04A88DED040ACDED050AA6
:10ADF00020F06EFE684620EE098A20F069FE94F984
:10AE0000F83207EE903AF8EEE77A28EE288AA7EEB5
:10AE1000A90A1EF039FD20EE090ABDEEC88A20EE0F
:10AE2000280A18EE101AFDEEC07A304617EE902A66
:10AE3000FFF732FF99E738EE400A38EE088A80EED5
:10AE4000080AA6F05BFE02A8B0EE408A20F040FEA1
:10AE500094F9F832F0EE007AB0EE697AA8EE677AEB
:10AE600007EE903AF8EEE77AA7EE270A1EF00CFDFF
:10AE7000C0E700BF105C002000000034408F0020BD
:10AE8000E02E65420000C842DB0FC93F10B5044602
:10AE90000848F7F765FD20B92046BDE81040FEF7E9
:10AEA000DFBC04484FF48051F7F760FB0028F3D073
:10AEB00010BD00BF102C00200020704700487047D4
:10AEC00030E90C080048704738E90C08002070474A
:10AED0000020704738B5154C05460021204601F08A
:10AEE00051FE042057F084FA0021204601F054FE60
:10AEF000132057F07DFA0021204601F057FE284626
:10AF0000FEF79AFE2046012102F00CF8462057F089
:10AF10006FFA6B6804F5A044D3F8F831C4F84438EC
:10AF20006B68D3F8FC31C4F8483838BD102C0020C9
:10AF3000FEF760BE0B207047004870475EEC0C08BF
:10AF400000487047B0E90C080120704701207047A5
:10AF5000012070470020704770B50B4E06F5C045C4
:10AF600005F54C730FCB05F5487484E80F003046A7
:10AF7000FBF76CF801463046FCF740F9002385F8F2
:10AF8000B033012070BD00BF102C002038B531480F
:10AF9000F8F784FA2F48F8F77FF92E48F7F762FFA1
:10AFA0002C481021F7F7E2FAE0B12B4AD2F83433FB
:10AFB000D2F844239342D4BF00230123264C94F8B3
:10AFC000B02372B973B304F54C730FCB04F5487515
:10AFD00085E80F00A4F5C040FBF776FA012384F85A
:10AFE000B03338BD1D4AB2F9141F0029F9DD02F54E
:10AFF00080429FED1B7AD2F83433D2F824239B1A77
:10B0000007EE903AF8EEE77A67EE877A07EE101AC5
:10B01000B8EEC77AF4EEC77AF1EE10FACCBF01238E
:10B020000023CBE7A4F58043642193F9482512FB64
:10B0300001F2D3F8481FA4F580548A42A8BF0A46FB
:10B04000D4F84408C3F8482F51421EF0D1FCC4F88C
:10B050004408C6E7102C0020108C0020104C002063
:10B060000AD7233C38B52A4DB5F9DC3483EAE371BD
:10B07000A1EBE37189B241B1002B05F58043B4BF68
:10B080004FF0FF32012283F8F822224C224801F0CF
:10B09000F3F994F8E237DBB995F9B734022B18D1FC
:10B0A00094F8D5318BB11D49A1F6DC2024F094FA37
:10B0B00058B101231A49184884F88D38282203F022
:10B0C000F9FA28B9002384F88D38012384F8E2378F
:10B0D00038BD012B0ED1A4F5A04001F0E7F848B12E
:10B0E000A4F5A040FBF7AEF90028B8BF4042B0F588
:10B0F0007A7FD5DB95F9B734042BE9D194F8D531B3
:10B10000002BE2D00549A1F6DC2024F0E1FACFE7DC
:10B11000104C0020107C0020102C0020408F0020BC
:10B12000887C0020022070470048704728EA0C08FD
:10B130000048704706270E08034B0022C3F8442836
:10B14000C3F84828704700BF107C002038B5094D6F
:10B1500004462846F7F776FC2846F7F70FFD204609
:10B16000F7F724FD2846F8F729F82046BDE83840CF
:10B17000FEF774BD102C00200D207047004870476A
:10B18000A4EA0C0800487047ACEA0C08012070479C
:10B1900001207047012070470023C37480F82430D9
:10B1A000012070470148002101F066B9102C0020F1
:10B1B0002DE9F041B44CD4E9CE322DED088B134388
:10B1C000D4F83423134388B005460FD1AF48F8F7BD
:10B1D00065F9AE48F8F760F89FEDAD0A462008B073
:10B1E000BDEC088BBDE8F04157F002B907F0FCF860
:10B1F00090F87C32DB07E9D5B5F90830E97C09EE37
:10B20000103AB5F9103008EE903AB8EEC99AF8EE57
:10B21000E88AA4F58056002940F0D7809FED9DAACA
:10B2200029EE0ABA0122FDEECB7AA4F5C04017EE52
:10B23000903AC6F8AC37FAF737FF686800F57F70C8
:10B240000790B0EE408A20F043FCDFED937A20EEC9
:10B25000270A1EF097FA0798F0EE409A20F082FC39
:10B26000A4F5C040F0EE40AAFEF70EF8002878D111
:10B2700004F54C7797E80F0005F1140C8CE80F00EB
:10B2800097E80F0004F5487C8CE80F0004F5507C2B
:10B290008CE80F00D4EDD17A8048F8EEE77AF0EE32
:10B2A000680A77EE8B7AB0EE690AFDEEE77AC4EDB4
:10B2B000D17A0CF005FE002386F8193895F9123082
:10B2C000724803EB830303EB83039B000121A6F881
:10B2D000DA37F6F78DFE96F82888B8F1000F74D1AA
:10B2E0006F4B9FED707AB3F9803407EE903AF8EE29
:10B2F000E77A67EE877AF4EEE7AAF1EE10FA64DDFA
:10B3000054F002F8074619EE900AF5F7FDF8CDE97A
:10B31000040118EE900AF5F7F7F8CDE9020119EEED
:10B32000100AF5F7F1F8604ACDE900010621384628
:10B330004DF012F97DF0A2F8C6F89887C6F8840798
:10B340007DF09CF80123C6F8940729EE8A0AEB7475
:10B350001EF042FABDEEC00A10EE103AC6F89C3755
:10B3600033E07DF08BF8D6F83C38C01A42F2107307
:10B3700098427FF67DAFF0EE087AF4EEE7AAF1EEA0
:10B3800010FA7FF775AFBCEEC88A04F5507718EE57
:10B39000103A9BB208EE103AB8EEC88AB4EEC89ADA
:10B3A000F1EE10FA47D853F0AFFF404A06214DF0B6
:10B3B000D3F804F54C730FCB87E80F000123EB742F
:10B3C0000321A4F5C040F6F713FE304803F092FFC6
:10B3D00028B12E480321F6F70BFE0023EB74D6F8B4
:10B3E0003038012B40F0B180D4F83433AA699FED96
:10B3F00029AA9B1A07EE903AD6F89C370133F8EE4B
:10B40000E79A5BD0DFED2A7AE9EE0A7AF4EEE79A62
:10B41000F1EE10FA0ADA274905F114000CF0DAFC13
:10B42000F4EEC08AF1EE10FA00F28F801748032183
:10B43000F6F7DEFD89E053F067FF1F4A06214DF065
:10B440008BF804F54C7C9CE80F0005F1140E8EE897
:10B450000F009CE80F0087E80F00D4EDD17A39EE99
:10B46000488AF8EEE77AF0EE680AE8EE0A7A38469B
:10B47000B0EE690AFDEEE77AC4EDD17A0CF020FD5A
:10B480000121E9749DE700BF108C0020102C0020E2
:10B49000000000000000C842E02E6542508F0020EE
:10B4A000104C00209A99993EF5EA0C08B4EA0C0871
:10B4B000000048C3408F0020D0EA0C08B5F90A30DC
:10B4C00007EE903AF8EEE77A05F1140767EE8A7A0C
:10B4D000F4EEE79AF1EE10FA51DB424938460CF0EF
:10B4E00049FBDFED417AB6EE008AA0EE278A97E8A5
:10B4F0000F00BDEEC88A9FED3D0AB8EEC88A04F57C
:10B50000507C28EE008A8CE80F00F0EE680A38487C
:10B51000B0EE480A0CF0D4FCD4EDD17AF8EEE77A1C
:10B5200028EE0A0AE9EE0A7AFDEEE77AC4EDD17A4E
:10B530001EF052F9BDEEC00A10EE103AC6F89C3764
:10B54000D6F83038012B3FF45DAF2A4803F0B2FE45
:10B5500018B128480321F6F74BFDD6F83038012BF7
:10B5600017D1244803F030FC224803F079FD21482C
:10B5700008B0BDEC088BBDE8F04103F087BC194969
:10B5800038460CF027FCF4EEC08AF1EE10FAA4D98C
:10B59000D6E795F824302BB9174862F035F8012327
:10B5A00085F824301348F7F779FF1248F7F774FE4F
:10B5B0001048F7F757FC114890F8EC366BB10023B0
:10B5C00080F8EC3633220221A0F5405008B0BDECE3
:10B5D000088BBDE8F041FDF7C3BA08B0BDEC088B9D
:10B5E000BDE8F081408F0020A00CB3450AD7233C72
:10B5F000508F0020102C0020304F0020105C0020C5
:10B6000010B50446FEF724FA2046054B40F8143BDB
:10B610000CF07EF8204603493FF066FC204610BD42
:10B62000A8EB0C0840EB0C08182070470048704746
:10B6300010EC0C080048704718EC0C08012070470B
:10B64000012070470120704708B50548F7F726FF2D
:10B650000348F7F721FEBDE808400148F7F702BCB0
:10B66000102C002008B5064879F04EFFBCEEC00A49
:10B67000044810EE103A99B2BDE8084000F0FCBE54
:10B68000E0580020102C002010B50D4CD4F8B83E26
:10B69000002B12DDA4F50050FCF732FBA4F500509E
:10B6A00000F058FA04F54D607AF078F804F54D6032
:10B6B000044979F011FC012010BD0020FCE700BF17
:10B6C000104C0020508F002070B5234CD4F8B001EE
:10B6D00003688EB05B689847072830D00A2809D0E5
:10B6E000062805D106F080FE90F87C32DB071DD4D9
:10B6F000012019E004F509660FCE07AD0FC596E8E5
:10B70000070085E8070009AB0FCB04F5805601ADB3
:10B7100085E80F00D6F84C33009304F59A530ECB0E
:10B7200004F19800FFF702FB0EB070BD06F05CFE5E
:10B7300000F51B700FC804F5805601ADE8E707A9B6
:10B7400004F15C00FFF738F80028D1D0079904F124
:10B750009800FFF7C9FAE7E7107C0020F0B585B044
:10B760000E4E0391144653F0CFFD06F5A047054653
:10B77000D7F8B001026892689047039B0090084A8E
:10B78000284606214CF0E8FED7F8B0112246304694
:10B7900005B0BDE8F04002F08DBF00BF102C0020C6
:10B7A00020EC0C082DE9F0472DED028B96B000241B
:10B7B00007466D4879F0D2FE05940694079406F08A
:10B7C00013FE05A906F05AFB70B3684B93ED007A9F
:10B7D000B5EEC07AA3F6B468F1EE10FA08F5405958
:10B7E00027DBDDED067ADDED056A67EEA77A27EE49
:10B7F000077AE6EEA67AF4EEC77AF1EE10FA18DDD3
:10B80000D9F8B00103685B6898470A2811D053F053
:10B810007BFD574A06214CF09FFE262209F190013C
:10B82000A8F5005002F046FF16B0BDEC028BBDE853
:10B83000F087D9F8B0A14F4B01949A450294039434
:10B84000049417D109F509660FCE08AD0FC596E827
:10B85000070085E8070011A80BF05AFFB9F8E818AF
:10B860000FAA0AF2DC7022F0E5FF88BB0294019473
:10B87000049403949FED400A404E01A820F0D2F8B2
:10B8800003A88DED080A9FED3C0ACDED090A20F0D2
:10B89000C9F835488DED0F0AB0EE401AF0EE601A87
:10B8A000CDED100A9DED080ADDED090A79F0B0FD35
:10B8B0000628044619D10023C6F8F4327CF0DEFDD8
:10B8C00006F55071C6F8DC04274879F005FBABE7B4
:10B8D00001A911A80CF0FAF80028C7D003A90AA8FA
:10B8E0000CF0F4F80028C1D0C4E708F561687CF0DA
:10B8F000C5FDDFED237A98ED008AD6F8DC6428EEEA
:10B90000278ADFED207AB4EEE78AF1EE10FA0546D9
:10B91000384658BFB0EE678AFFF7D6FE48B9022C0A
:10B9200016D0BCEEC88AAD1B18EE103A9D42FFF44B
:10B930007BAF013C062C0ED8DFE804F0040A0D0DA5
:10B94000100D1300104924223846FFF707FF6BE75C
:10B950000E492522F8E70E491622F5E70D49262261
:10B96000F2E70D490122EFE7E0580020C45A002019
:10B970003CEC0C08887C00200000C842108C0020A1
:10B9800000007A4400409C4662EC0C0877EC0C08FE
:10B990008CEC0C08A4EC0C08BBEC0C0803207047E2
:10B9A0000048704740ED0C08004870474CED0C080B
:10B9B000F8B52B4D06460027A5F54050A5F8E876CA
:10B9C000F7F7D2FC7368A5F58052D3F8F811D2F8D6
:10B9D000483F994205F5005423DBC4F844387368A6
:10B9E0009FED206AD3ED7F6A02F5936393ED007AB1
:10B9F000F8EEE66A27EE067AF4EEC76AF1EE10FA80
:10BA000018DBBDEEC77A17EE103A1748C4F848386D
:10BA1000FCF7FCFE20B1D4F848385B42C4F8483843
:10BA2000F8BD5B429942D8DD012385F8E836C4F8B9
:10BA30004478D4E702F64C72D2ED007A67EE867A4B
:10BA4000F4EEE76AF1EE10FA93BFFDEEE77A012318
:10BA500085F8E93617EE903A88BF0023D5E700BF96
:10BA6000105C00200000C842102C002070B500219E
:10BA70002DED028B04463448344D01F083F83248F2
:10BA80000021F0EE408A01F087F895F8E836B0EE34
:10BA9000408AD3B1B0EE680A042056F0A9FC95F8AC
:10BAA000E93693B3B0EE480A132056F0A1FC2648BD
:10BAB000002101F07BF82046FEF7BEF8BDEC028BBA
:10BAC0002046BDE87040FEF7C9B805F50056A5F55B
:10BAD0004050F6F7B7FFD6F84438002B0CDCD6F808
:10BAE0004438002BDBDA042056F096FCB4EEE80A6A
:10BAF000F1EE10FACED4D2E7042056F08DFCB4EE6D
:10BB0000E80AF1EE10FAEADDC4E7114D0E48F7F746
:10BB100035F8D5F84838002B0CDCD5F84838002B20
:10BB2000C5DA132056F078FCB4EEC80AF1EE10FA2C
:10BB3000B8D4BCE7132056F06FFCB4EEC80AF1EE9F
:10BB400010FAEADDAEE700BF102C0020105C0020E8
:10BB5000107C002000F5C0400023C0E9BC3380F811
:10BB6000F93280F8FA32704700F5A043D3F8DC319F
:10BB7000002BCBBF07EE903A00F51250B8EEE70A63
:10BB8000DFED037ADCBF90ED010A20EE270A704753
:10BB90000000C8422DE9F0412DED028B00F5A057C1
:10BBA00084B09FEDDB8A1037054603A938468DED3A
:10BBB000038A06F0FDF905F5A044B0B19FEDD57AF2
:10BBC000DDED037A04F5056367EE877AD3ED006A4D
:10BBD0009FEDD17AE6EE877AF4EE487AF1EE10FA2C
:10BBE00048BFF0EE487AC3ED007A2846F6F706FE25
:10BBF000F0EE000AB0EE408A9FEDC50A1DF030FF5E
:10BC0000D4ED7D7A94F8C03138EE678A05F5005698
:10BC1000E0EE087AC4ED7D7A002B40F02681D4F85E
:10BC2000AC2105F5A04354339A4205D005F5A04355
:10BC30005C339A4240F0198108212846F6F796FCB9
:10BC4000804640B106F28443D3ED007A9FEDB37A8B
:10BC500067EE877A04E102212846F6F787FC014661
:10BC6000002800F0E680D6F8383F1B8B2846414676
:10BC700008EE103A01F056F9D6F8380F4369B8EEDD
:10BC8000488AB0EE401A002B00F0B480012B00F07F
:10BC9000B680DFEDA37AF0EE671A06F2844393EDE7
:10BCA000000A9FED9E7AF4EEC17AF1EE10FA20EED2
:10BCB000070A4FF06401C0F2AF80B6F8802412FB8F
:10BCC00001F2B0EE672A07EE902AF0EE400AB8EED5
:10BCD000E70A1DF01FFDBDEEC00A84ED760AD4F818
:10BCE000AC0103689B6B9847002852D094F8EC3164
:10BCF000002B4ED0D4F8AC3105F5A0450C35AB4245
:10BD000047D0D4ED767A9FED877AF8EEE77A384619
:10BD100027EE878AD4ED7A7AF8EEE78A68EE878A8A
:10BD200006F052FBC8EE807A9DED037A77EE877AB3
:10BD3000B6EE007AB4EEE78AF1EE10FA4CBF77EE79
:10BD4000C87ADFED777A77EE877A94ED7C7AFDEE2C
:10BD5000E77AF8EEE77AB4EEE77AF1EE10FA0ADD68
:10BD600037EE676ADFED706AB4EE666AF1EE10FADC
:10BD700048BFF0EE477A94ED767ADFED686AC4ED5D
:10BD80007C7AB8EEC77AA7EEA67ABDEEC77A84EDC4
:10BD9000767AD4F8AC0103681B6B984740B1B4F9CC
:10BDA000E421002AC2BFD4F8D8319B18C4F8D83196
:10BDB000B6F98224B6F98014D4F8D80164235A4322
:10BDC00059431DF015FEC4F8D80106F57E63D6F878
:10BDD000F00F93ED4A8A06F0F7FAC8EE007A9DED6F
:10BDE000037A77EEC77AC4ED787A04B0BDEC028BA3
:10BDF000BDE8F081DFED4A7AF1EE481A4DE78DEDAE
:10BE0000010A54F0D7FF07EE900ADFED451A9DEDC9
:10BE1000011AF8EEE77A40E7B6F8823413FB01F333
:10BE200000EE903AB0EE482AF8EEE00AF0EE671A1B
:10BE30004FE7B6F98024B6F982349B1A07EE903AA0
:10BE40002846B8EEE78A01F06DF8B6F8803464222F
:10BE500013FB02F307EE903AF8EEE77AE8EE007A89
:10BE6000FDEEE77AC4ED767A39E7D6F8B83E002BD6
:10BE700018DD96F8583EABB1D4F8AC2105F5A143D6
:10BE800064339A421AD105F53350103079F056FCDC
:10BE9000B5EEC00AF1EE10FADFED207A1ADD20EEE1
:10BEA000270A18E7D4F83038042B18D105F5C44018
:10BEB000083078F06DF9C4F8D80110E705F5A04313
:10BEC00078339A427FF40BAF05F53350103079F098
:10BED00039FCDDE706F2844393ED000ADFE7D4F88E
:10BEE000AC2105F5A14320339A4206D1D4F8DC31C8
:10BEF000002B02DDC4F8D831F1E605F5A043783314
:10BF00009A427FF49FAE2846FFF72EFEE3E600BF7D
:10BF1000CDCCCC3DCDCC4C3ECDCC4C3F0000C8422E
:10BF2000000000000AD7233C9A99993F30B500F5EC
:10BF3000A05587B010350023044628460393049388
:10BF4000059305F0E3F8002846D003A9284606F03B
:10BF50005DF8002840D004F5B95393ED047ADFED85
:10BF6000236A8DED017AB0EEC77AD3ED077AB4EE8D
:10BF7000E67AF1EE10FACDED027A06D5F0EEE77A28
:10BF8000F4EEE67AF1EE10FA2DD401A81FF03CFE93
:10BF900003A901A81FF080FD04F5125393ED037A65
:10BFA000B5EEC07AF1EE10FAC4BFDFED117A27EEDC
:10BFB000C00A04F5A044C8BFA7EE270A03F10C038A
:10BFC000CABF01230023FDEEC07A84F8EC31CCBF58
:10BFD00017EE903A002304E004F5A044002384F80F
:10BFE000EC31C4F8E83107B030BD00BF00000034C8
:10BFF0000000C8422DE9F04100F5C0472DED028B4D
:10C0000007EE901AD7F8FC3200F5C645B8EE678AFD
:10C010000446403500F54056B3BB00F5A042134638
:10C02000D2F8AC117833994204D000F5A143203303
:10C03000994229D192F8E03733B304F5C640294636
:10C0400030300BF0C7FED6F818090368F0EE408ACE
:10C050005B6AB0EE480A9847F0EE087A60EE277AFD
:10C06000F4EEE78AF1EE10FA0EDDBDEC028BD6F8A5
:10C0700018099FED0C0A036804F5C6412A469B6A1D
:10C08000BDE8F04120311847B0EE480ABDEC028B04
:10C09000D6F8180997F9F82203682946DB6ABDE843
:10C0A000F04118470000000070B504462DED048BE8
:10C0B00004F5C0457CF0D6F9D5F86833534AC31A65
:10C0C0009342064674D907EE903AB8EE670ADFED60
:10C0D000507A9FED501ADFED500A20EE270A40F209
:10C0E00095101DF0E5FBC5F8686304F50056DFED1B
:10C0F0004B7AD6F8343FB3F9083008EE103A96F987
:10C10000DE34B8EEC88AF0EE408A28EE278A0BB1FA
:10C11000B1EE488A9FED427ADFED427AB4EEC78AEB
:10C12000F1EE10FA6ADAD5EDD96AF4EEC76AF1EEEB
:10C1300010FAB4EEE78AACBF01230023F1EE10FA47
:10C1400059D995EDD97AB4EEE77AF1EE10FA52D8D2
:10C150002046FAF7B7FB96F9DF349FED339A00EEED
:10C16000103A04F54053D3ED040A93ED021AB8EEE9
:10C17000C00A40F2A710F1EE600A20EE080A1DF096
:10C1800097FB28EE800A204620EE090AFDEEC07AD1
:10C1900017EE901AFAF754FBD6F8B83E002B05DDDF
:10C1A00096F8583E8BB12046FAF78CFB85EDD98A7C
:10C1B0002046F9F7B9FF2046F6F754FEBDEC048B94
:10C1C0002046BDE87040F7F767B8184BDFED187AE6
:10C1D00093ED007AE7EE097AF0EE678A06F004F94B
:10C1E000D0ED9C7AF8EEE77A77EEA87AFDEEE77A62
:10C1F000C5EDD47ADAE7002BAAD1ACE7B4EEE78A32
:10C20000F1EE10FAA7D900239BE700BF9F8601003B
:10C21000BD3786359A99193ECDCCCC3D530469394A
:10C2200000000034000000B40000C842AC5A0020F6
:10C2300000007A4470B5054600F5B0404FF0FF317C
:10C24000543022F04DFB431C064605F5A04404D1B2
:10C2500004F5F764124B236070BD05F5C64105F582
:10C26000C640403120300BF085FC9FED0E7AF6EE93
:10C27000007AE0EE077A04F5F764FDEEE77A17EE50
:10C28000900A301A1DF0DCFA07EE900A9FED067A4C
:10C29000F8EEE77A67EE877AC4ED007ADCE700BF54
:10C2A0000000B442A00CB3450AD7233C00F540502F
:10C2B000D0F8180903689B6B18470000F7B500F524
:10C2C00040530546D3F8180903681B699847074689
:10C2D0002846FFF7EBFF05F5C0440646D4F8F40204
:10C2E000002860D13EB1D4F83433C4F800333D4B5C
:10C2F000C4F804330120C4F8EC721DF0A1FAD4F89C
:10C30000F43294F9F82200FB0230C4F8F4022EB3A0
:10C310000023019394F85833002B48D094F804324A
:10C32000022B44D105F5B240012201A96C3046F040
:10C3300043F900283BD0D4EDD77ADFED2B6AB8EE75
:10C34000E77ADDED017AE7EE667AB1EE047AF0EE97
:10C35000E77AF4EEC77AF1EE10FA33D494F8F932B2
:10C36000002B3DD1D4F8F432D4F80423002BB8BF0D
:10C370005B42934234DBD4F83413D4F80033C4F86E
:10C380000013CB1A03F2F31340F2E630834202F5B6
:10C39000D2328CBF0023012302F5F07284F8FA3206
:10C3A000C4F804231CE0D4F8EC32F81AA3E7D4F85C
:10C3B0005023D4F834339B1A03F2F31340F2E632DD
:10C3C0009342CBD8012384F8F932002384F8FA325F
:10C3D000D4F8F43203F5D23303F5F073C4F8043320
:10C3E00003B0F0BDE0A501000AD7233C2DE9F041E0
:10C3F00000F5A045044695F8D531C3B300F5C04318
:10C40000D3F8482312B9D3F84C3383B304F5C646A6
:10C4100004F5C647204630364037FAF783FD3946E3
:10C4200030460BF0D7FC05F2C47304F5C6413A461A
:10C430002031304683ED000A0BF002FC05F5F9636C
:10C44000DFED0C0A83ED000A7620B7EE001A1DF02E
:10C450002FFA04F53F53204683ED790AFFF72EFFAC
:10C46000D5F8AC010368BDE8F041DB6A1847BDE8C8
:10C47000F08100BF00000000012970B5044600F5FE
:10C48000C04512D800F5005395F84023B3F9AA34FB
:10C4900083EAE371A1EBE37189B2012998BF3C21E2
:10C4A000920731D5FF2385F8F83207EE901AF8EE9F
:10C4B000677A2046C5EDC37AFFF79CFDD5F8FC32BC
:10C4C00043BB2046FFF7F2FE04F5A04650B906F53F
:10C4D000F96393ED007AF7EE007AB4EEE77AF1EEC5
:10C4E00010FA17DD7BF0CAFFC5F8FC02D6F8AC01E4
:10C4F00003681B6A984768B104F55B500021BDE8EA
:10C500007040303050F018BA002BB4BF4FF0FF33FA
:10C510000123C8E770BD000010B500F5B2444C34EB
:10C5200020465CF03FFC2046BDE810405CF0AABC11
:10C5300010B500F5A043044693F860399A0717D464
:10C540005B0700F55B504FF002014CBF094A0A4AF5
:10C5500030304CF001F804F5B2404C305CF0F6FBA2
:10C5600004F53B500121BDE810401C3063F00EB8CB
:10C5700010BD00BFC4ED0C08DEED0C0870B500F571
:10C58000A046054696F94C499CB196F86039C3F32C
:10C5900080045B0729D4B6F95239002B0BDC2846FE
:10C5A000FFF7C6FF05F53B5001211C3062F0EEFF9E
:10C5B0000124204670BD2146F9F79EFDB6F9523997
:10C5C00007EE903AF8EEE77AB4EEE70AF1EE10FAE9
:10C5D000E5D5D6F8CC37002BE1D005F55B50044A01
:10C5E000042130304BF0B8FFE3E70024E1E700BF5F
:10C5F000F4ED0C0808B52DED028B08EE901A30B35F
:10C60000F2B1B0F9083008EE103AB8EEC88AF8EE88
:10C61000E88A9FED100ADFED100A28EE800ADFEDB0
:10C620000F8A4FF4D470B7EE001A1DF041F9C8EE2E
:10C63000280A1DF099F820EE280ABDEC028B08BDEF
:10C6400054F03CFC07EE900AB8EEE78ADFE79FED76
:10C65000020AF2E70AD7233C0000000000A08C4544
:10C6600037B500F50054054694F90B35002B52D030
:10C6700054F03EFB54F032FBC4F8300F54F038FB5A
:10C6800054F018FBC4F8340F54F032FB54F01CFB88
:10C69000C4F8380F54F02CFB54F020FB41F29411F5
:10C6A000C4F83C0FD4F8300F54F06CFBD4F8340FBE
:10C6B00041F2941154F066FBD4F83C0F41F294110E
:10C6C00054F060FB284600F027FC48BBD4F8380F34
:10C6D000642154F053FB54F00BFBD02155F03AFB8E
:10C6E000C4F8400F54F004FBD22155F033FBC4F8DA
:10C6F000440F05F5225034304921019056F0B8F826
:10C7000001984A2156F0B4F80198462103B0BDE8DB
:10C71000304056F0ADB854F0EBFA54F0C1FAABE744
:10C7200005F5C043D4F8380F93F8E434642173B1AD
:10C7300054F024FB6421462055F092FF64214920E7
:10C7400055F08EFF64214A2055F08AFFC3E754F06C
:10C7500019FBEFE710B500F500541E21D4F8300F97
:10C7600054F014FBD4F8340F1E2154F00FFBD4F80E
:10C770003C0F1E2154F00AFBD4F8380F1E21BDE8EF
:10C78000104054F003BB000007B500F0C5FB0146A4
:10C7900058B90190462055F085FE0199492055F081
:10C7A00081FE01994A2055F07DFE0021042056F0BB
:10C7B0004BF90021132056F047F90021462056F08E
:10C7C00043F90021492056F03FF900214A2056F054
:10C7D0003BF90021152003B05DF804EB56F034B9A5
:10C7E00010B5044656F076FB55F0C6FF204601F022
:10C7F000E7FCBDE8104056F075BA000038B500F50A
:10C800000055044695F90B350BB1002038BD0121C8
:10C81000F5F7ACFE90B104F5A043D3F8AC2104F5D4
:10C82000A14334339A4209D004F5A04314339A4209
:10C8300004D004F5A04324339A42E6D12046F6F70B
:10C840008FF80028E1D0D5F83C3FB3F90800DDE7C8
:10C8500038B52DED028B00F5A04393F8C031002BC5
:10C8600040F0B9805D4A00F5A143D2F8AC213433E1
:10C8700000F55B549A4204F1300408D0584A032171
:10C88000BDEC028B2046BDE838404BF065BE00F59C
:10C8900000559FED546AD5F8302FB2F90830002BBF
:10C8A000B8BF5B429BB207EE903A138B06EE903A0C
:10C8B000F8EEE66AF8EEE77A66EE866AF4EEE67A75
:10C8C000F1EE10FA17DCD5F8342FB2F90830002B4E
:10C8D000B8BF5B429BB207EE903A138B07EE103A5B
:10C8E000B8EEC77AF8EEE77A27EE067AF4EEC77A62
:10C8F000F1EE10FA01DD3C4AC1E700F5B950043011
:10C900001FF0BAFEDFED397A20EE270AF3EE0E7A39
:10C91000B4EEE70AF1EE10FA01DD354AAFE7042084
:10C9200056F04AF8132056F047F8152056F044F810
:10C930004D2056F041F84E2056F03EF84F2056F06C
:10C940003BF8502056F038F8152055F065FD9FED66
:10C95000298AB0EEC00AB4EEC80AF1EE10FA0BD57F
:10C96000102056F029F8562056F026F8112056F0DF
:10C9700023F8572056F020F8032055F05DFDB0EE67
:10C98000C00AB4EEC80AF1EE10FA0FD5022055F035
:10C9900053FDB0EEC00AB4EEC80AF1EE10FA05D5A8
:10C9A000182056F009F8192056F006F8D5F8300F7F
:10C9B000811D0C303FF05EF9D5F8340F811D0C302D
:10C9C0003FF058F9D5F83C0F811D0C303FF052F97B
:10C9D000094A052154E7BDEC028B38BD107C0020CC
:10C9E00008EE0C08CDCC4C3E28EE0C08E02E65423B
:10C9F00050EE0C08000000346CEE0C0810B500F589
:10CA0000005494F9E2349BB1D4F8380F54F0CCF9C7
:10CA1000D4F8382FB4F9E43430B1B2F906009842B2
:10CA2000ACBF0020012010BDB2F906008342F7E739
:10CA30000120F8E710B50446FFF7E0FF60B104F508
:10CA4000A0447BF01BFDD4F8CC31C01AB0F57A7F3E
:10CA500094BF0020012010BD0120FCE770B5054601
:10CA6000FFF7E8FF05F5005408B3D4F8303F9A8982
:10CA7000DA80D4F8343F9A89DA80D4F83C3F9A8936
:10CA8000DA80D4F8303F00261E81D4F8343F1E816E
:10CA9000D4F83C3F1E8105F5A043D3F8AC01C3F8A0
:10CAA000E46103685B689847D4F8383F1E8105F558
:10CAB000C8403C3071F002FE80B3002654F018F9F3
:10CAC000437A13B954F014F9837A94F9E224012AD1
:10CAD00023D106B10BB32846FFF7ACFF05F5A04400
:10CAE00094F8C63138B30133DBB20A2B84F8C6316F
:10CAF0000CD105F55B501F4B1F4A042130304BF021
:10CB00002BFD1E4A012384F8C031937294F8C6317C
:10CB10000A2B02D90A2384F8C63170BD2846FCF7D7
:10CB2000B3FB0028C9D154F0E3F854F0A5F8061E71
:10CB300018BF0126C2E7002BEFD0013BDBB2032B6D
:10CB400088BF032384F8C63194F8C631012B09D17C
:10CB500005F55B500A4B084ABDE8704004213030AF
:10CB60004BF0FABC002BD8D1044A84F8C031937240
:10CB7000D3E700BF134C0E087CEE0C08AD910020EB
:10CB800087F00C0800F500500A4690F9161FD0F8FF
:10CB9000300FFFF72FBD000000F500500A4690F956
:10CBA000171FD0F8340FFFF725BD000000F5005027
:10CBB0000A4690F9181FD0F83C0FFFF71BBD000084
:10CBC00010B54FF480610446F5F7D0FC04F500532E
:10CBD00028B1BDE81040D3F8380F54F06BBABDE867
:10CBE0001040D3F8380F54F06FBA00002DE9F0412F
:10CBF00000F500530546D3F83C3FB3F9088000F533
:10CC0000C044B8F1000F02D1012384F8803405F547
:10CC1000C8473C37384671F051FD0646F8B9B8F5BB
:10CC20007A6F2EDD7BF02AFCD4F87C34804693B1F9
:10CC3000C31A40F6B73293420FD905F5A045012239
:10CC400031463846F4F778FEC4F87C6484F8806492
:10CC5000C5F8748701E0C4F87C04BDE8F08118F5DC
:10CC60007A6F0EDA7BF00AFCD4F87C346BB1C01A10
:10CC700040F6B7339842F0D9012200213846F4F744
:10CC800081FE0023C4F87C34E7E7C4F87C04E4E7C1
:10CC900070B52DED028B044654F02AF853F0E2FEF5
:10CCA00030B9BDEC028B2046BDE87040FFF7D6BE20
:10CCB00004F5A04595F8C0311BB97BF0DFFBC5F842
:10CCC000D0012046FFF79AFE18B17BF0D7FBC5F8DC
:10CCD000CC012046FFF7C2FE2046FCF765F904F5BB
:10CCE00000560023C5F8E43196F9E63473B3D6F85C
:10CCF000383FB3F90830322B28DD38B3323B1BB252
:10CD000007EE903A04F5A050B8EEE78ADFED217AFD
:10CD1000103028EE278A04F033F948B3B6F982348C
:10CD200007EE903A06F2844696ED007AF8EEE77A3E
:10CD300077EEC77A27EE888ADFED177A28EE278A02
:10CD4000BDEEC88A18EE103AA5F8E4312046FFF788
:10CD50004DFFD5F8AC0103685B689847BDEC028BCA
:10CD6000014604F5C9400830BDE8704056F030BBBC
:10CD700096F9753496F977249B1A07EE903AF8EEF7
:10CD8000E77A27EE888ABDEEC88A18EE103AA5F831
:10CD9000E631DBE70AD7A33C0000C84270B500F5D6
:10CDA0000054D4F8E8340BB9002042E094F974340C
:10CDB000002BF9DA00F5A045D5F8AC0103685B68F3
:10CDC00098470138172833D801A353F820F000BF43
:10CDD000C9CE010805CF010831CE0108FBCE0108FC
:10CDE000F1CE0108DDCE0108D3CE010831CE010815
:10CDF00031CE010835CE0108BFCE0108B5CE0108FD
:10CE0000A9CD0108E7CE0108E7CE010831CE01081F
:10CE100031CE010831CE010831CE010831CE0108F2
:10CE200031CE010831CE010831CE01080FCF010803
:10CE3000012070BDB5F89268162EB5D0D4F8E8146C
:10CE400011F0020301F0010205D0A6F1150CDCF18E
:10CE5000000343EB0C0311F0040043EA020303D088
:10CE6000A6F11F046042604143EA000211F008008D
:10CE700007D01F2E1AD0A6F1110002288CBF002067
:10CE8000012011F0100340EA020005D0102E0FD04F
:10CE9000A6F1520253425341034311F4006014BF00
:10CEA00095F85C18014643EA0100C2E70120E8E773
:10CEB0000123F1E7D4F8E804C0F34010B9E7D4F84F
:10CEC000E804C0F38010B4E7D4F8E804C0F3C0105D
:10CED000AFE7D4F8E804C0F30020AAE7D4F8E804E8
:10CEE000C0F34020A5E7D4F8E804C0F38020A0E711
:10CEF000D4F8E804C0F300309BE7D4F8E804C0F3AA
:10CF0000403096E7D4F8E804C0F3803091E7D4F8D5
:10CF1000E804C0F3C0308CE700F5005090F87404CA
:10CF2000C009704738B504460D4653F0E1FE03686A
:10CF3000DB689847C8B104F50053D3F8380F6DB1DA
:10CF400053F0BCFF07EE900AB8EEE70A04F5C044C0
:10CF500094F8E3340BB1B1EE400A38BDB0F90830B3
:10CF600000EE103AB8EEC00AF0E79FED010AF4E7D0
:10CF70000000000038B52DED028B04460D4653F03D
:10CF8000B7FE0368DB68984700283FD0214BD3F8F1
:10CF9000383F5B69012B07D0BDEC028B2946204648
:10CFA000BDE83840FFF7BEBF4FF480612046F5F77B
:10CFB000DDFA0028F0D004F50053DFED177AD3F83E
:10CFC000380F93F97734028B08EE903A00EE102A6E
:10CFD000F8EEE88AB8EEC08A68EEA78A53F078FFC8
:10CFE000B6EE001AA0EE011A04F5C044DFED0B0AFC
:10CFF000B0EE680A1CF08AFC94F8E33428EE000ACC
:10D000000BB1B1EE400ABDEC028B38BD9FED030AB7
:10D01000F9E700BF104C00200AD7233C00000000B5
:10D0200073B500F5C046044696F80432022B00F5AD
:10D03000736512D100F5B240012201A96C3045F0B0
:10D04000BBFA50B1019BC5F89C3228463FF09EFACE
:10D050002046F9F7BBFD02B070BD04F5A043D3F83C
:10D060003038042B05D12046F9F794FA8DED010AEA
:10D07000E8E7D6F86C330193E4E7000070B500F5FB
:10D08000A0450446D5F8AC0103689B6B0E46984753
:10D0900048B9D4ED460A9FED1B0A64213046BDE82D
:10D0A000704055F09BBAD5F8AC0104F5A04104F5E9
:10D0B00000527831884292F8763492F940251DD199
:10D0C00095F8DC1741B93AB1D3B2D5F83018013927
:10D0D000012998BFD3B209E004F5C04191F9841247
:10D0E00061B1D5F83008042808D1CBB207EE903AE8
:10D0F000D4ED460AB8EE670A6421CFE7002AF5D0DE
:10D10000E3E700BF000000002DE9F04100F5A04575
:10D11000044604F5A143D5F8AC013433984203D159
:10D1200000263046BDE8F08103689B6B984740B10C
:10D1300095F8606916F0010603D0012385F82838B8
:10D14000EFE704F5C440083077F056F9064608B119
:10D150000126E6E795F82838002BE1D0D5F8AC0198
:10D1600003689B6B984708B90023E7E794F81434E9
:10D1700094F85874B02202FB034393F8F121BFBB2B
:10D18000012A0AD993ED837AF1EE047AB4EEE77AB4
:10D19000F1EE10FAACBF01270027D5F8AC2104F559
:10D1A000A04378339A4202D195F8DC3723B104F5D5
:10D1B000A1433C339A4241D104F50053204693F9F0
:10D1C0003485FCF761F8A8B9204601F081FC0028FD
:10D1D000BED0002385F8283894F8712404F58C63B8
:10D1E000242101FB023305F2D475DB6A2B6098E73A
:10D1F0003746D2E77BF042F9D5F83C384FF4FA6273
:10D20000C01A642313FB082341F28832934238BFCB
:10D2100013469842D8D92046F9F740F9B0F5FA7F7D
:10D22000D2DD04F5805341F26E72D3F80C3603F66A
:10D23000B7339342C8D8002FC6D095E704F5C04352
:10D24000D3EDDB7AB2EE047AF0EEE77AF4EEC77A49
:10D25000F1EE10FA88DA002F3FF47AAF04F5A0500F
:10D26000103003F08DFE00283FF47EAF04F500532C
:10D2700004F5055093F89E12103003F091F8F1EE8A
:10D28000047AB4EEE70AF1EE10FAFFF661AF6BE74D
:10D29000F8B52DED048B0446084617461D46BDF92A
:10D2A000286055F0B9F804F500543846B0EE408ACD
:10D2B00055F0B2F8B4F91025002AF0EE408A39DAB8
:10D2C000C2F1640307EE903A9FED217AF8EEE77A17
:10D2D00067EE877A60EE278A04F20C54D4ED007A68
:10D2E0009FED1C1ADFED1C0A38EEC80ABC2020EEA8
:10D2F000270A1CF0DDFA38EE288AB0EE409A94ED49
:10D30000000A9FED141ADFED140A28EE000ABD2072
:10D310001CF0CEFA2846B0EE408AB0EE490A55F02D
:10D3200067F8B0EE480ABDEC048B3046BDE8F84023
:10D3300055F05EB8D0D002F1640307EE903A9FED4D
:10D34000047AF8EEE77A67EE877A28EE278AC3E751
:10D350000AD7233C00A08C4500A08CC500B52DED5C
:10D36000048B042083B055F057F80320B0EE408AB8
:10D3700055F062F8DFED189A9FED181ADFED180AE4
:10D380008DED011AF0EE408AB0EE480AA8EEA90A27
:10D39000CF20CDED000A1CF08BFAB0EE409AB0EE33
:10D3A000480A9DED011ADDED000AA8EEE90AD02039
:10D3B0001CF07EFA1820B0EE408AB0EE490A55F013
:10D3C00017F8B0EE480A192003B0BDEC048B5DF8E5
:10D3D00004EB55F00DB800BF0000344200A08C45AE
:10D3E00000A08CC5F8B52DED088B00F5005600F5B2
:10D3F000C04596F9FE3E13F0040F03F0010203F05E
:10D40000020440F0F580D5F8E8747B1E5F425F416E
:10D41000002A00F0EF804D2054F0FEFF4E20F0EE89
:10D42000409A54F0F9FFB0EE408AB6F91235DFEDBC
:10D4300087AA0AEE103A1520B8EECAAA54F0ECFFFB
:10D440002AEE2AAA20EE0AAA002C00F0DB80F0EED9
:10D45000488AB0EE699AB5EEC0AAF1EE10FA40F330
:10D46000D6809FED7B1ADFED7B0A38EE0A0A4FF477
:10D4700080701CF01DFA9FED761ADFED760AB0EE93
:10D48000408A40F2011038EECA0A1CF011FAF0EEA0
:10D49000408A96F9FF3E632B15DC07EE903A9FED2C
:10D4A0006E7AF8EEE77AB4EEC79A67EEAA7AF1EEF2
:10D4B00010FAF4EEC78A98BF29EE279AF1EE10FA17
:10D4C00098BF68EEA78AD5F8E83496F9FC4E96F92D
:10D4D000FD6E022B00F0B48024B2002C01DC002E83
:10D4E0006EDD032054F0A8FFDFED5C7AB4EEE70AAE
:10D4F000F1EE10FAB0EE40AA62DB002F00F0A2803D
:10D500009FED571ADFED570A40F2271030EE000A60
:10D510001CF0CEF99FED541ADFED520AB0EE40BA7E
:10D520004FF494703AEE410A1CF0C2F970EE007AA2
:10D53000B0EE4BAA07EE104AF8EEC7AA9FED4BBA21
:10D540009FED431ADFED430A6AEEA7AAB0EE690A1F
:10D5500040F22B10AAEE8B0A1CF0AAF907EE906A93
:10D56000F0EE409AB8EEE70A9FED391ADFED390A7E
:10D570002AEE40AAB0EE490A4FF49670AAEE0B0AC2
:10D580001CF096F9B0EE409AB0EE480A9FED301AC2
:10D59000DFED300A40F22D10AAEE8B0A1CF088F95C
:10D5A000B0EE408AB0EE680AAAEE0B0A4FF497700C
:10D5B0009FED271ADFED270A1CF07AF9F0EE408A7A
:10D5C000B0EE690A102054F013FFB0EE490A56205D
:10D5D00054F00EFFB0EE480A112054F009FFB0EEEF
:10D5E000680ABDEC088B5720BDE8F84054F000BF36
:10D5F00001270DE7042054F00FFFB0EE408AF1EE52
:10D60000409A12E7DFED178AB0EE689A23E79FEDA4
:10D61000101ADFED100A39EECA0A4FF482701CF0BE
:10D6200047F99FED0B1ADFED0B0AF0EE409A40F23E
:10D63000051039EE0A0A1CF03BF9B0EE409A28E7D3
:10D6400000244CE7F0EE407A74E700BF0AD7233C91
:10D6500000A08C4500A08CC5000000B40000003480
:10D660000000C84200000000000048426666E63E36
:10D6700038B52DED028B00F500550446D5F8440F62
:10D68000A0B304F5A04393F8C0217ABB93F8C63148
:10D6900063BB53F0D9FC07EE900AB8EE678A4620C8
:10D6A00095F9745454F0B8FE002DF0EE408A20DA5B
:10D6B00004F5C440083076F021FDE8B99FED101A5A
:10D6C000DFED100A40F25110B1EE680A1CF0F0F8DC
:10D6D000B4EE408AF1EE10FAC8BFB0EE480ABDECD5
:10D6E000028B6E20BDE8384054F082BE9FED058A63
:10D6F000D5E79FED040AEBE79FED010AE8E700BFDD
:10D700000000C8420000000010B52DED028B4369F7
:10D71000002B4AD0037C0BB101330374037C002B34
:10D7200041D0182B1FD803EB4303C3EB03139B001B
:10D730001CB2002307EE903AB8EEE78A0420B0EE60
:10D74000480A54F055FE07EE904A1320B8EEE70A57
:10D7500054F04EFEB0EE480ABDEC028B1520BDE839
:10D76000104054F045BE4A2B02D8C3F13203DAE729
:10D77000632B01D8643BD6E77C2B08D8643B03EBD2
:10D780004303C3EB03139B001BB20024D2E7AE2B71
:10D7900002D8C3F19603F2E7C72B01D8C83BEEE7E6
:10D7A00000230374F1E71C46C4E7BDEC028B10BDF7
:10D7B00010B59FED1C7AD0ED017AF4EEC77A002304
:10D7C000F1EE10FA044643722BDB90ED007AB4EED2
:10D7D000E77AF1EE10FA24D908F0E8FA217A07F096
:10D7E00039FFD4ED010AF5EE007A60EEA77AB4EEC7
:10D7F000E70AF1EE10FA14D494ED001A40F2A510E5
:10D800001CF056F8F7EE007AB4EEE70AF1EE10FAE3
:10D8100007D494ED007AC7EE007A01236372C4ED59
:10D82000037A10BD00000034437A7BB391F90030D5
:10D8300090ED037A07EE903AF8EEE77A67EE877A92
:10D840009FED137AF4EEC77AF1EE10FAD8BFF0EE3E
:10D85000477AFDEEE77A17EE903A0B7092F90030B6
:10D8600090ED037A07EE903AF8EEE77A67EE877A62
:10D870009FED087AF4EEC77AF1EE10FA58BFF0EE99
:10D88000477AFDEEE77A17EE903A1370704700BFC3
:10D890000000C8C20000C842437AF0EE407A5BB193
:10D8A00090ED030A9FED051ADFED050A27EE800AC9
:10D8B0004FF4E6701BF0FCBF704700BF0000C84289
:10D8C0000000C8C2F8B504460E4617467AF0D6FDE9
:10D8D000054604F5A340783008F046F804F5A04466
:10D8E000D8B3462054F098FDDFED3D7AB4EEE70A58
:10D8F000F1EE10FA10DB97F9002094F92938193A63
:10D90000934209DAD4F82C28AA4205D0C4F82C583E
:10D91000013384F8293844E0462054F07DFDDFEDE2
:10D92000317AB4EEE70AF1EE10FA3AD896F900200F
:10D93000002A36DAC2F1FF2294F92A3802F57F0272
:10D94000E73293422DDAD4F82C28AA4229D0C4F821
:10D950002C58013384F82A3823E0D4F82C38EB1AF9
:10D96000B3F57A7F1DD3462054F056FD94F929383B
:10D9700007EE903AF8EEE77AB4EEE70AF1EE10FA25
:10D9800001DD002B22DC462054F046FD94F92A38B4
:10D9900007EE903AF8EEE77AB4EEE70AF1EE10FA05
:10D9A00018D497F9000094F929280021821A1CF054
:10D9B0002FF8387096F90000002806DA94F92A1832
:10D9C000002201441CF024F83070F8BDC4F82C5833
:10D9D000013B9EE7002BE4DDC4F82C58013BB9E77E
:10D9E00000000034000000B410B52DED028B00F5EE
:10D9F000005282B092F9743492F875248DF8063092
:10DA0000002B0446B0EE408A8DF8072004DAFFF7B9
:10DA1000C5F908B98DF8060004F5A043D3F83028FD
:10DA2000012A4BD0072A49D004F5C440083076F0CB
:10DA300065FB002857D10DF106010DF1070204F531
:10DA40003C50FFF7F1FE2046FFF73CFF9DF9063002
:10DA50009DF90720DFED258A9342A8BF134607EE04
:10DA6000903A04F53F54B8EEE70A203420EE280A35
:10DA700020468DF8063075F039FD9DF9073000EE2F
:10DA8000103AB8EEC00A204620EE280A75F038FD9C
:10DA90009DF9073001EE103A9DF9063000EE903AFC
:10DAA000B8EEC11AF8EEE00A40F24D20B0EE480A96
:10DAB0001BF0FEFE02B0BDEC028B10BD03F28C72B7
:10DAC000D2ED007AFDEEE77A03F5F26317EE902AC5
:10DAD000D3ED007A8DF80720FDEEE77A17EE903A45
:10DAE0008DF80630A7E70023FAE700BF0AD7233CEA
:10DAF00070B5044600F53C5604F5A0453046FFF7E6
:10DB000057FED5F8AC0103685B6D984740B14620DD
:10DB100054F082FC3046FFF7BFFE462054F068FC0C
:10DB2000D5F8AC0103681B6D984740B1462054F00E
:10DB300073FC2046FFF758FF462054F059FC20465E
:10DB4000FFF7E2FA10B304F5005595F9E03443B15C
:10DB500001212046FFF7E6F9BDE87040462054F069
:10DB600047BC04F5C4440834204676F0C7FA50B1E7
:10DB7000204676F04BFC30B195F9743400EE103A43
:10DB8000B8EEC00AE8E79FED020AE5E770BD00BF06
:10DB90000000000010B504462DED028B462054F025
:10DBA0003BFC2046B0EE408AFBF76EFB80BB04F5E1
:10DBB000C8403C3070F082FD50B304F5A053D3ED63
:10DBC0009A8A1BF0F9F890F8EC349FED137A0C2246
:10DBD00002FB0300D0ED807AE8EEC77AF4EEC77A54
:10DBE000F1EE10FA0CDC04F5005494F9773407EEEA
:10DBF000903AF8EEE77AF4EEC87AF1EE10FA07D52B
:10DC0000BDEC028B0548BDE81040012104F060BE68
:10DC1000BDEC028B10BD00BF0AE81C412040002073
:10DC20002DE9F34100F500550646D5F8403F002B9D
:10DC300042D1002706F5A048D8F8AC0103689B6BD9
:10DC400098470446002860D006F5A050103003F035
:10DC500097F900283DD0D8ED767A9FED487AF8EE16
:10DC6000E77A67EE877AFDEEE77A17EE903A1BB215
:10DC700095F927250AB19A422EDA95F9254574BB04
:10DC8000D8F8AC2106F5A14364339A4209D105F5D1
:10DC90006B63D3ED007AFDEEE77ACDED017A9DF965
:10DCA0000440D8F83038013B062B2ED8DFE803F0CB
:10DCB0001E2D24612D2D1E0053F01AF80368DB6819
:10DCC00098470028B5D0D5F8400F53F0BDF947B2BA
:10DCD000B0E795F97734CBE795F92645D0E724B23C
:10DCE0009C42ACBF95F924450024C9E795F9283535
:10DCF000002B18BF1C4608E095F928352BB130469B
:10DD0000FBF7E2FA08B195F9284587EAE773A3EB38
:10DD1000E773DBB2A342C8BF3C4607EE904A03203C
:10DD2000B8EEE70A54F064FB07EE907A0220B8EEF2
:10DD3000E70A54F05DFB95F95935D6ED460A00EE39
:10DD4000103A6421B8EEC00A032054F047FC95F95C
:10DD50005935D6ED460A00EE103A6421B8EEC00AF5
:10DD6000022054F03BFC304602B0BDE8F041FFF722
:10DD7000F5BA06F5C04393F98332B9E70AD7233CD5
:10DD800070B504462DED048B462054F045FB5B4BEB
:10DD9000DFED5B7A93F9C83E08EE903AF8EEE88A38
:10DDA000152068EEA78AB0EE408A54F035FB9FED4F
:10DDB000557A20EE280A04F5C045C0EE077A05F52D
:10DDC0009B6604F5C5401430C6ED007A73F0F2F995
:10DDD00008B100233360B5EEC08AF1EE10FA46D5E3
:10DDE0002046FFF799F8002800F083802046FEF7D0
:10DDF000D5FF00287DD005F59B65D5ED007A9FED18
:10DE0000429A9FED421ADFED420AB0EE480AA7EEB1
:10DE1000890A4FF43B701BF04BFDD5ED007A9FED66
:10DE20003B1ADFED3B0AF0EE408A40F2ED20B0EE07
:10DE3000480AA7EEC90A1BF03BFDB0EE408A04F584
:10DE4000C8453C35284670F043FCE0BB284671F0DD
:10DE500005FD022829D10321492054F023FEBDEC01
:10DE6000048B0321BDE870404A2054F01BBE40D90A
:10DE700005F59B65D5ED007A9FED239A9FED251A58
:10DE8000DFED220AB0EE480AA7EE890A40F2F2203E
:10DE90001BF00EFDD5ED007A9FED1E1ADFED1B0A7B
:10DEA000F0EE408A40F2F320C1E79FED180A4920C6
:10DEB00054F09EFABDEC048B9FED140ABDE870404F
:10DEC0004A2054F095BAB0EE680A492054F090FA0E
:10DED000B0EE480A4A2054F08BFA20464921FFF759
:10DEE000CDF8BDEC048B20464A21BDE87040FFF719
:10DEF000C5B89FED068AF0EE488AA0E7104C0020D6
:10DF00000AD7233C00A08C450000484200000000D6
:10DF10000000C8C20000C842F8B52DED028B00F524
:10DF2000C046044696F98132002B31DD00F5A0424F
:10DF30001346D2F8AC2178339A4229D196F980322F
:10DF4000002B25DD00F5C440083076F049F9F8B122
:10DF500004F5C8403C3070F0B1FBC8B9124F9FEDDA
:10DF6000138A04463D682D190ED0B5F9080054F007
:10DF700065F848B196F98132012B0CD1B5F908004A
:10DF8000B0EE480A54F034FA1434B4F5A07FE9D165
:10DF9000BDEC028BF8BD022BF6D1B5F908000321C8
:10DFA00054F080FDF0E700BF3C9600200000000028
:10DFB00037B500F5A043044693F888370BB39FEDBF
:10DFC000120A15204F2554F013FA204600955023CD
:10DFD00013221521FFF75CF9152054F0ABFC80B932
:10DFE000284654F0A7FC60B99FED070A4E2054F074
:10DFF000FFF99FED050A4D2003B0BDE8304054F015
:10E00000F7B903B030BD00BF00000000704700004A
:10E01000F8B52DED048B00F5A0440546D4F8AC010D
:10E0200003689B6B984730B9D4F8AC2123464C3336
:10E030009A4240F0C08005F5C8403C3070F048FB83
:10E04000002800F0B8802846FBF71EF9002800F0F1
:10E05000B280D4F84438002BB8BF5B42B3F52F7FB1
:10E0600000F3A980D4F84838002BB8BF5B42B3F561
:10E070002F7F00F3A08005F5C0477AF0FFF9D7F8AD
:10E08000A833C31AB3F5FA7F0646C0F0948005F5AD
:10E09000C05393ED057AF2EE007AB4EEE77AF1EE32
:10E0A00010FA00F1888004F5056494ED007AB4EE6E
:10E0B000E77AF1EE10FA7ED405F5405393EDE78A46
:10E0C00005F5225403F59D63D3ED048A3434B0EE94
:10E0D000480A0421204654F001FAB0EE680A1321E0
:10E0E000204654F0FBF978EEC89A4D21B0EE690A4B
:10E0F000204654F0F3F938EE289A4E21B0EE490A42
:10E10000204654F0EBF9B0EE680A4F21204654F057
:10E11000E5F9B0EE680A5021204654F0DFF905F524
:10E120000055B0EE480A1821204654F0D7F9B0EE59
:10E13000480A1921204654F0D1F995F9FE3E03F022
:10E140000202DB075CBFF1EE489AB0EE489A6AB370
:10E15000B0EE498AF0EE698AB0EE690A10212046D5
:10E1600054F0BCF9B0EE680A5621204654F0B6F9D6
:10E17000B0EE490A1121204654F0B0F9B0EE480A39
:10E180005721204654F0AAF9D7F8AC33C7F8A86352
:10E19000F31A42F2107293420DD9C7F8AC63BDEC8A
:10E1A000048B2046BDE8F84054F07EBD9FED038A05
:10E1B000F0EE488AD0E7BDEC048BF8BD000000000B
:10E1C00073B5044654F086FE054654F019FE204609
:10E1D000FFF7D6FD4E23009313224D230421204642
:10E1E000FFF756F84F2315211322009320465023A2
:10E1F000FFF74EF82046FFF7F5F82046FFF78CFEB4
:10E200004FF400512046F4F7B1F910B12046FFF762
:10E21000CFFE04F50056D6F8CC0E50B104F5A0425E
:10E2200004F5A143D2F8AC2134339A4201D154F021
:10E23000B9F854F07BFD53F0CFFF284654F0E8FDC9
:10E2400096F9A03C2BB1204602B0BDE87040FFF724
:10E25000DFBE02B070BD000073B5044604F5C545CD
:10E2600054F038FE143554F0CBFD284672F0A2FF6E
:10E27000002866D104F5A046D6F83038042B04D126
:10E2800004F5C440083075F065FF2046FFF730FC08
:10E29000D6F8AC2104F5A143343304F5C8459A42BD
:10E2A00005F13C0523D0284670F012FAF8B99FED2D
:10E2B000320A462054F09CF89FED2F0A492054F072
:10E2C00097F89FED2D0A4A2054F092F8284671F0F5
:10E2D000C5FA02280BD10321462054F0E3FB0321A9
:10E2E000492054F0DFFB03214A2054F0DBFB204699
:10E2F000FFF750FC2046FFF793FC2046FFF7B8F9E4
:10E3000020464621FEF7BAFE284670F0D7F990B9AC
:10E310000190284671F0A2FA68B102281CD1019937
:10E32000462054F02BFB0199492054F027FB01991A
:10E330004A2054F023FB204602B0BDE87040FFF7AE
:10E340003FBF2846F7F70AFE04F5C04393F99E3213
:10E350002B2B8FD002B070BD9FED070A462054F0E2
:10E3600047F89FED050A492054F042F89FED020A54
:10E370004A2054F03DF8DEE700000000F8B500F553
:10E38000A046054696F85C18214876F015FF05F57D
:10E390000053D3F8B83E002B39DD05F53354103463
:10E3A000204676F0F9FED6F8AC7105F5A146643644
:10E3B000B74208D12046012176F03CFF3846BDE83F
:10E3C000F840FDF7EFB93B6838469B6A984701462D
:10E3D0002046C1B176F0A0FDC8B1204676F03CFEE3
:10E3E000204676F0DBFD90B105F55B50094B0A4AFB
